:020000040800F2
:1000000000000110017E03080525030835130108CF
:10001000057F0308057F0308057F03080000000033
:100020000000000000000000000000004D2B03084D
:10003000492B030800000000452B0308C9C4000831
:10004000057F0308057F0308057F0308057F030874
:10005000057F0308057F030831D000085DD1000843
:1000600021D10008E5D00008A9D00008C1BA0008D5
:10007000B1BA0008A1BA000891BA000881BA000814
:100080006DBA000859BA0008057F0308057F030808
:10009000057F0308057F0308057F03086DD000086E
:1000A000057F0308057F0308057F0308057F030814
:1000B000057F0308851F0108057F0308057F0308E6
:1000C000057F0308057F0308057F0308057F0308F4
:1000D000057F03086DC70008D1C6000835C60008B3
:1000E000F5CF0008057F0308692B0308057F030887
:1000F000551F0108057F0308651F010845BA000860
:10010000057F0308057F0308751F0108057F0308A5
:1001100099C50008FDC4000839B601081DB60108DC
:1001200031BA00081DBA000809BA0008F5B900087C
:10013000E1B90008057F0308057F0308057F030870
:10014000057F0308057F0308057F030809250308C9
:10015000CDB90008B9B90008A5B90008057F0308A2
:10016000057F0308057F0308057F0308057F030853
:10017000057F0308057F0308057F0308057F030843
:08018000057F0308057F030859
:1001880016000800D0270020D82700200000000013
:10019800D405000827000400F4280020FC290020CA
:1001A80000000000DC05000801010400182B0020F5
:1001B800FC410020000000000000000008020900C7
:1001C800D6410020004200200000000019BD0008B0
:1001D80002000C00E04100200C420020000000005A
:1001E80000000000F7010600D0410020184200205E
:1001F80000000000E00500080A020A00A82B002001
:100208002042002000000000E605000815007000EC
:1002180058460020284B0020000000000000000085
:100228000300010054460020984B00200000000005
:10023800000000002A006000644500209C4B00205C
:10024800000000003DF001082C0010000C4C0020BC
:10025800FC4B00200000000075EF01082B00240073
:10026800404C00201C4C00200000000045EF010815
:1002780003123300D74D0020A44D002000000000D9
:10028800F005000825005A00F04C00204A4D0020D7
:100298000000000000000000F6110C00E44C0020F3
:1002A800D84C0020000000002406000801200800A7
:1002B800504F00209C4F002000000000300600082E
:1002C8001A000800384F0020A44F0020000000004A
:1002D80038060008290050002052002074520020DF
:1002E8000000000000000000140002001C52002062
:1002F800C45200200000000040060008100003005F
:1003080010520020C85200200000000042060008D9
:1003180028000C0004520020CC52002000000000ED
:100328004606000823001000F4510020D85200208F
:100338000000000065BA020819000500EC51002011
:10034800E85200200000000052060008F8110100E1
:10035800E8510020F0520020000000005806000874
:1003680000010400E4510020F452002000000000C5
:100378005A0600082F001100D0510020F852002022
:10038800000000005E0600081B00F40094560020E0
:100398008857002000000000B9F1020826000E006E
:1003A8008C5800207C58002000000000957102083D
:1003B8000B2010002C5500209C5800200000000045
:1003C800700600081F000E00C85900209C5B002022
:1003D800000000008006000805020100B059002056
:1003E800AC5B0020000000008E0600080301060038
:1003F800E65B0020085C0020000000009006000872
:1004080001020500305E00202C7100200000000071
:1004180015A5020800020500105C002034710020B8
:1004280000000000000000001E0004007C620020A4
:100438003C710020000000009606000804008000BF
:10044800748A0020F48B00200000000000000000E7
:10045800F9010400E0870020748C002000000000EF
:1004680009BD0008FD011E00C0870020788C00200F
:100478000000000099BC000822000C00F48D002048
:10048800788E0020000000009A06000818102C0042
:100498001C90002048900020000000006DF2010828
:1004A800FB010100E48F0020749000200000000090
:1004B80075010108FC010900B08E00207890002029
:1004C80000000000390101080A101200848E002083
:1004D8008490002000000000A60600080600160010
:1004E80098920020F895002000000000750A020884
:1004F8003400100004910020109600200000000035
:1005080065F001080D003400D090002020960020EE
:1005180000000000F9BF010812100C00B490002080
:100528005496002000000000B80600080C020100E4
:10053800B09000206096002000000000C40600086B
:1005480002020300C490002064960020000000000E
:100558000000000005000600F2A900203CAA0020C7
:1005680000000000C80600080C002400BAA90020FA
:1005780044AA00200000000091AD01080E20EA0006
:10058800B2A8002068AA002000000000550A02084E
:100598001300040024AA002054AB0020000000002F
:1005A800D00600080201030099A8002058AB0020DB
:1005B80000000000B9AD0108F5116200DEA70020B7
:0C05C8005CAB002000000000A5820008D1
:1005D400C4090000190128282003000012010000AA
:1005E400000000004A01B400D60100000000000031
:1005F40000000000000000000000000000000000F7
:1006040000000000000000000000000000000000E6
:1006140000000000000000000000000000000100D5
:10062400000000000000000000000000E803640077
:10063400040A00017E05EA05B40532000300000146
:1006440005000000000100000000000000000000A0
:1006540028010000040090010000000000000000D8
:100664000000000000000000000000002B21231EF9
:1006740064000200000001000A01290000000000DB
:10068400000001000000000500000000040101005A
:10069400000000000100C800141E010064002C01C9
:1006A400280000300100005A0000000090012C01D5
:1006B400C8006400000000010005415746340000F2
:1006C40001000000200003000100000018200000C9
:1006D4000000803F0000803F0000803F01010000D7
:1006E40050010000070000000200000000000000AC
:1006F40000000000010203040607080901010000CC
:100704006CDA0308C00A04080000000000000000BE
:100714007CDA030884DA03080000000001200000EA
:1007240088DA0308B8D9030800000000014000007B
:1007340090DA030814E90308000000000120000017
:100744009CDA0308A8DA0308000000000400000093
:10075400ACDA0308500D0408000000000400000097
:10076400B8DA030860E70308000000000100000095
:10077400020100000000803F0000803FFF000000F5
:1007840000AF03080508040000000000C0D70308F8
:100794005CD70308ECAE0308000000002CAF03088C
:1007A40005080A0000000000C0D703085CD703084E
:1007B4000CD6030800000000A123030859230308F2
:1007C400A922030800000000991F03081D21030843
:1007D4009D2103088520030800000000000000009C
:1007E4008D1F0308711F03086D1F0308691F030889
:1007F4005D1F0308591F0308651F0308611F0308D1
:10080400811F0308751F03085D2003087120030876
:100814004920030835200308212003080000803FF5
:10082400303030302D30312D30315430303A30309A
:100834003A303000FFFFFFFF2808040800000000E2
:1008440000000000C9BF0108A086010004000000E8
:100854000000000000000000000000000000000094
:100864000000000000000000000000003010040838
:100874008807040800000000293C01087D000000EE
:10088400060000000000000000000000000000005E
:100894000000000000000000000000000000000054
:1008A4004009040800000000000000007D33030834
:1008B400E803000003000000000000000000000046
:1008C4000000000000000000000000000000000024
:1008D40000000000480904080000000000000000B7
:1008E400790B02081027000003000000000000003C
:1008F40000000000000000000000000000000000F4
:100904000000000000000000A80E04080000000021
:10091400F1C102081D8B0108204E000005000000F3
:1009240000000000000000000000000000000000C3
:1009340000000000000000000000000030E0030898
:100944000000000000000000392E030810270000FA
:100954000100000000000000000000000000000092
:100964000000000000000000000000000000000083
:1009740054090408000000000000000005010108FB
:10098400E803000005000000000000000000000073
:100994000000000000000000000000000000000053
:1009A40000000000600904080000000000000000CE
:1009B40071B00108204E0000030000000000000098
:1009C4000000000000000000000000000000000023
:1009D400000000000000000070090408000000008E
:1009E40000000000A5AE0108204E00000300000036
:1009F40000000000000000000000000000000000F3
:100A0400000000000000000000000000800904084D
:100A14000000000000000000C92B0308400D030083
:100A240003000000000000000000000000000000BF
:100A340000000000000000000000000000000000B2
:100A4400DC08040800000000000000004DD6010886
:100A5400102700000100000000000000000000005A
:100A64000000000000000000000000000000000082
:100A74000000000038E0030800000000000000004F
:100A84007DB10208102700000300000000000000F0
:100A94000000000000000000000000000000000052
:100AA400000000000000000090090408000000009D
:100AB4000000000031720308A0860100010000005C
:100AC4000000000000000000000000000000000022
:100AD40000000000000000000000000044E00308E3
:100AE4000000000000000000B9D70008A00F0000BB
:100AF40001000000000000000000000000000000F1
:100B040000000000000000000000000000000000E1
:100B1400980904080000000000000000D1EB02085E
:100B24001027000001000000000000000000000089
:100B340000000000000000000000000000000000B1
:100B440000000000901404080000000000000000F1
:100B540029A500081A41000001000000000000005F
:100B64000000000000000000000000000000000081
:100B74000000000000000000C0E0030800000000C6
:100B8400000000001D820208102700000100000080
:100B94000000000000000000000000000000000051
:100BA40000000000000000000000000080070408AE
:100BB4000000000000000000593C03081A41000036
:100BC4000100000000000000000000000000000020
:100BD4000000000000000000000000000000000011
:100BE400A409040800000000000000005570030878
:100BF400400D0300000000000000000000000000A1
:100C040000000000000000000000000000000000E0
:100C140000000000AC09040800000000000000000F
:100C240011700308400D03000000000000000000E4
:100C340000000000000000000000000000000000B0
:100C44000000000000000000B409040800000000D7
:100C5400000000009DC00108A08601000300000000
:100C64000000000000000000000000000000000080
:100C740000000000000000000000000000FFFF0072
:100C840000000000AA5503009FAA5505010000AA10
:100C9400550701000001AA550B010000AA550902DD
:100CA4000000000001000000C0120000000000006D
:100CB400010203040102030406070809E001080015
:100CC40001010000E5BF0208000000000000000070
:100CD400000101010100000000000101FFFF00000C
:100CE4000000803F01000000080000000060024096
:100CF4001060024000000000000B00000000200013
:100D04000000000000000000006002402860024073
:100D140000000000060C000000002000000000009D
:100D2400000000000060024040600240000000003B
:100D3400100D000000002000000000000000000072
:100D4400006002405860024000000000160E0000DF
:100D540000002000000000000000000000600240CD
:100D64007060024000000000200F0000000020001E
:100D740000000000000000000060024088600240A3
:100D84000000000026100000000020000000000009
:100D94000000000000600240A0600240000000006B
:100DA40030110000000020000000000000000000DE
:100DB40000600240B860024000000000362F0000CE
:100DC4000000200000000000000000000064024059
:100DD40010640240000000000038000000004000E1
:100DE400000000000000000000640240286402408B
:100DF4000000000006390000000040000000000070
:100E04000000000000640240406402400000000052
:100E1400103A000000004000000000000000000044
:100E2400006402405864024000000000163B0000C9
:100E340000004000000000000000000000640240C8
:100E44007064024000000000203C000000004000EC
:100E540000000000000000000064024088640240BA
:100E640000000000264400000000400000000000D4
:100E74000000000000640240A06402400000000082
:100E840030450000000040000000000000000000A9
:100E940000640240B86402400000000036460000CE
:100EA40000004000000000000000000004030904EA
:100EB40012010002020200408304405700020102B2
:100EC4000301000009024300020100C032090400CA
:100ED40000010202010005240010010524010001A3
:100EE400042402020524060001070582030800FF0A
:100EF40009040100020A0000000705010240000085
:100F04000705810240000000FF0000008924030857
:100F1400C9210308F59A0208DD1F030835240308D4
:100F2400ED1F030809200308CD1F0308BD1F030894
:100F34000000000000000000F41404080F0000008A
:100F4400000000000000000000000000F41B00206E
:100F5400FFFFFFFFFA000000010000000100000095
:100F6400380D0408400D04086C0D0408000000004E
:100F74000000000000000000000000002F0D040825
:100F8400040000004D5B03080000000000000000A6
:100F9400740D0408010000000000000000000000BF
:100FA40000000000000000000E000000000000002F
:100FB4000000000000000000168D00200100C4099C
:100FC40000000000148D00200100C409000000008E
:100FD400128D00200100C40900000000108D0020C3
:100FE4000100C409000000000C8D00200100C409A8
:100FF400000000000E8D00200100C4090000000064
:101004000A8D00200100C40900000000088D0020A2
:101014000100C409000000004AA800200100C80023
:101024000100000048A800203200307532000000A2
:1010340046A80020055A050041A8002000FF010031
:1010440045A80020010000009008002043A80020CB
:101054000200000000D6030840A8002000FF0100A1
:1010640044A80020010000009008002042A80020AD
:101074000200000000D60308A00D04080F000000C1
:10108400000000000000000000000000980800209C
:10109400E25B00209CFF2C0100000000BE1C00202D
:1010A4000A0000000CD60308C8A70020E0150C179E
:1010B40000000000BD1C0020080000005CD70308ED
:1010C400BC1C002005000000C0D70308CAA70020EC
:1010D4000200000024D60308F8A900200100FF7FC5
:1010E40001000000F0A900200200000030D603082F
:1010F400A2A800200300000040D60308A1A80020F5
:101104000300000040D60308A4A900200000F40155
:1011140001000000A2A900200000F4010100000069
:10112400A0A900200000F401010000009EA90020F5
:101134000000F401010000009CA9002000FF010050
:10114400B8A90020E803D0070A000000B6A90020CF
:10115400006401000A000000B7A900200064010037
:101164000A000000B0A90020006401000A00000089
:10117400B5A90020006401000A000000B4A9002001
:10118400006401000A000000B3A90020006401000B
:101194000A000000AFA9002000FF01000A000000BF
:1011A400AEA9002000FF01000A000000AEA8002044
:1011B4000000F40101000000ACA800200000F401CC
:1011C40001000000AAA800200000F40101000000B2
:1011D400A8A800200000F40101000000ABA9002031
:1011E40000C80100AAA9002000C80100A9A9002084
:1011F40000C80100A8A90020006401000A00000042
:10120400A7A9002000FF01000A000000E7A90020B0
:1012140000C80100E6A9002000C80100E5A90020DB
:1012240000C80100E4A9002000C80100E3A90020CF
:1012340000C80100E2A9002000C80100E1A90020C3
:1012440000C80100E0A9002000C80100DFA90020B7
:1012540000C80100A80D0408000000000000000000
:101264000000000000000000B80D040809000000A0
:10127400000000003C09002004000000C00D040828
:1012840009000000000000003009002004000000F4
:101294005413040809000000000000002409002081
:1012A40004000000C4D80308090000000000000086
:1012B4001809002004000000C80D040809000000FB
:1012C400000000000C09002004000000D00D0408F8
:1012D40009000000000000000009002004000000D4
:1012E400D80D04080900000000000000F4080020E4
:1012F40004000000E00D04080900000000000000E4
:10130400E808002004000000740D04080100000037
:1013140000000000000000000000000000000000C9
:101324000E000000000000000000000000000000AB
:10133400B80E0408000000000000000000000000D7
:1013440000000000B0D903080700000000000000FE
:101354006009002000000000C80E04080800000016
:10136400000000005409002000000000D40E04080E
:1013740008000000000000004809002000000000F0
:10138400740D0408010000000000000000000000CB
:1013940000000000000000000E000000000000003B
:1013A4000000000000000000DC0E04080000000043
:1013B400000000000000000000000000EC0E040823
:1013C4000D000000000000009C0900200000000047
:1013D400F40E04080D000000000000009009002035
:1013E40000000000FC0E04080700000000000000DC
:1013F4008809002000000000040F04080D0000000C
:10140400000000007C090020000000000C0F04080C
:101414000D00000000000000700900200000000022
:10142400140F0408070000000000000068090020F1
:1014340000000000740D040801000000000000001A
:101444000000000000000000000000000E0000008A
:101454000000000000000000000000001C0F040851
:101464000000000000000000000000000000000078
:10147400B0D903080C000000000000004CA80020B4
:1014840000000000300F04080C0000000000000001
:101494004EA8002000000000400F04080C000000CB
:1014A4000000000084A8002000000000500F040881
:1014B4000C0000000000000078A8002000000000DC
:1014C400640F04080C0000000000000050A8002075
:1014D40000000000D00B04080C0000000000000015
:1014E40052A8002000000000700F04080C00000047
:1014F4000000000054A8002000000000840F04082D
:101504000C0000000000000056A8002000000000AD
:101514008C0F04080C0000000000000058A80020F4
:1015240000000000940F04080C00000000000000FC
:101534005AA8002000000000A00F04080C000000BE
:10154400000000005CA8002000000000340704082C
:101554000C000000000000005EA800200000000055
:10156400A80F04080C0000000000000060A8002080
:1015740000000000B40F04080C000000000000008C
:1015840062A8002000000000C8D903080C00000075
:101594000000000064A8002000000000C00F040840
:1015A4000C0000000000000066A8002000000000FD
:1015B400CC0F04080C0000000000000068A8002004
:1015C40000000000D80F04080C0000000000000018
:1015D4007CA8002000000000E00F04080C000000BC
:1015E400000000007AA8002000000000E80F0408B2
:1015F4000C0000000000000088A80020000000008B
:10160400F40F04080C000000000000008AA8002069
:1016140000000000001004080C000000000000009E
:1016240090A8002000000000E4D903080C0000008A
:10163400000000006AA80020000000000C1004084C
:101644000C0000000000000072A800200000000050
:10165400141004080C000000000000006CA8002016
:1016640000000000201004080C000000000000002E
:101674006EA80020000000002C1004080C000000DC
:101684000000000070A800200000000034100408CE
:101694000C0000000000000074A8002000000000FE
:1016A400FC0704080C000000000000007EA80020D5
:1016B40000000000401004080C00000000000000BE
:1016C40076A80020000000003CD903080C000000AC
:1016D4000000000086A80020000000004C10040850
:1016E4000C0000000000000080A8002000000000A2
:1016F400541004080C0000000000000082A8002020
:10170400000000005C1004080C0000000000000051
:101714008CA8002000000000641004080C000000E5
:10172400000000008EA8002000000000740D0408D2
:1017340001000000000000000000000000000000A4
:10174400000000000E000000000000000000000087
:10175400000000006C1004080000000000000000FD
:1017640000000000000000007C10040805000000D8
:1017740000000000A0A8002000000000740D040870
:101784000100000000000000000000000000000054
:10179400000000000E000000000000000000000037
:1017A4000000000084100408000000000000000095
:1017B4000000000000000000C00A0408000000004F
:1017C40000000000AC1E002004000000C0D8030884
:1017D4000D000000955B0308FC09002000000000D8
:1017E4002C1604080D000000DD550308F009002044
:1017F40000000000AC0F04080D000000A955030808
:10180400E409002000000000901004080800000013
:1018140000000000D8090020040000000C10040897
:101824000D00000095550308CC09002000000000BD
:10183400981004080900000000000000C0090020FE
:1018440004000000A010040803000000313B03085A
:10185400A809002000000000740D04080100000025
:101864000000000000000000000000000000000074
:101874000E00000000000000000000000000000056
:10188400A410040800000000000000000000000094
:1018940000000000B41004080D0000000000000067
:1018A400140A002000000000BC1004080A00000014
:1018B4000000000009AA002000000000C81004086D
:1018C4000A0000000000000011AA0020000000002F
:1018D400D01004080A0000000000000019AA00202B
:1018E40000000000D81004080800000000000000F8
:1018F400080A002000000000740D04080100000024
:1019040000000000000000000000000000000000D3
:101914000E000000000000000000000000000000B5
:10192400E0100408000000000000000000000000B7
:1019340000000000F41004080D0000000000000086
:101944002C0A002000000000041104080400000018
:10195400815E030800000000000000000C11040870
:101964000D00000000000000200A0020000000001C
:1019740020110408040000005D5E0308000000005C
:1019840000000000740D04080100000000000000C5
:101994000000000000000000000000000E00000035
:1019A40000000000000000000000000028110408EE
:1019B4000000000000000000000000000000000023
:1019C4003C1104080700000000000000680A002021
:1019D4000000000048110408080000000000000096
:1019E4005C0A0020000000005411040808000000F4
:1019F40000000000500A00200000000060110408EC
:101A04000800000000000000440A0020000000005C
:101A14006C1104080800000000000000380A0020CF
:101A240000000000740D0408010000000000000024
:101A34000000000000000000000000000E00000094
:101A440000000000000000000000000078110408FD
:101A54000000000000000000A71E0020000000009D
:101A6400841104080B00000000000000D00A0020CC
:101A7400000000008C1104080B00000000000000AE
:101A8400C40A002000000000981104080B000000A4
:101A940000000000B80A002000000000A41104089F
:101AA4000B00000000000000AC0A00200000000051
:101AB400B01104080B00000000000000A00A002080
:101AC40000000000BC1104080B000000000000002E
:101AD400940A002000000000C41104080B00000058
:101AE40000000000880A002000000000D011040853
:101AF4000B000000000000007C0A00200000000031
:101B0400DC1104080800000000000000700A002036
:101B140000000000740D0408010000000000000033
:101B24000000000000000000000000000E000000A3
:101B3400000000000000000000000000E81104089C
:101B44000000000000000000000000000000000091
:101B5400FC1104080800000000000000000B002035
:101B64000000000008120408080000000000000043
:101B7400F40A002000000000141204080800000009
:101B840000000000E80A0020000000002012040801
:101B94000800000000000000DC0A00200000000033
:101BA400740D0408010000000000000000000000A3
:101BB40000000000000000000E0000000000000013
:101BC40000000000000000002812040800000000CB
:101BD40000000000A41E00200000000038120408C9
:101BE4000B00000000000000300B0020000000008B
:101BF400441204080B00000000000000240B002025
:101C0400000000005012040807000000000000005B
:101C14001C0B0020000000005C12040807000000F8
:101C240000000000140B00200000000068120408EB
:101C340007000000000000000C0B00200000000062
:101C4400740D040801000000000000000000000002
:101C540000000000000000000E0000000000000072
:101C640000000000000000007412040800000000DE
:101C740000000000A41E00200000000080120408E0
:101C840007000000000000007C0B002000000000A2
:101C9400881204080700000000000000740B0020F4
:101CA400000000009012040807000000000000007B
:101CB4006C0B0020000000009812040807000000CC
:101CC40000000000640B002000000000A0120408C3
:101CD40007000000000000005C0B00200000000072
:101CE400A81204080700000000000000540B0020A4
:101CF40000000000B012040807000000000000000B
:101D04004C0B002000000000B8120408070000007B
:101D140000000000440B002000000000C012040872
:101D240007000000000000003C0B00200000000041
:101D3400740D040801000000000000000000000011
:101D440000000000000000000E0000000000000081
:101D54000000000000000000C81204080F0000008A
:101D640000000000B958030800000000840B0020A4
:101D74009EA800201700000050D603089DA800204C
:101D84000A3201009CA8002001FA010098A8002052
:101D940000C8010096A80020E803D0070100000055
:101DA400414C49454E57484F4F50463400000000BF
:101DB400DCA7002000030100DBA7002000030100D2
:101DC400D01204080F000000DD570308B9570308B8
:101DD40000000000600C0020DC1204080F0000006A
:101DE400795703083157030800000000D80C00207D
:101DF400E81204080F0000001958030801580308EA
:101E0400000000008C0D0020F41204080F000000F4
:101E1400CF580308000000002D5E03088410002042
:101E2400FC1204080F000000F55403080000000031
:101E340000000000D4100020041304080F00000068
:101E4400FD5B0308255B0308215B0308B011002038
:101E54000C1304080F000000F558030800000000EC
:101E64000000000050120020141304080F000000AA
:101E7400955903086559030800000000DC1200208E
:101E84001C1304080F000000115A0308595A0308D0
:101E9400000000007C130020ACA900200103010015
:101EA400281304080F0000003159030809590308D6
:101EB400000000006C140020301304080F00000020
:101EC400C5590308A55E030800000000F8140020AB
:101ED4003C1304080F000000855A0308ED5E030854
:101EE4000000000098150020A6A9002001030100AD
:101EF400441304080000000000000000000000007B
:101F04000000000050130408080000000000000056
:101F1400C416002000000000581304080700000045
:101F240000000000BC160020000000006813040834
:101F34000700000000000000B416002000000000AC
:101F4400741304080700000000000000AC16002011
:101F540000000000801304080D00000000000000D1
:101F6400A0160020000000008C13040803000000E9
:101F7400313B03088816002000000000740D04089B
:101F8400010000000000000000000000000000004C
:101F9400000000000E00000000000000000000002F
:101FA400000000009413040800000000000000007A
:101FB4000000000000000000A41304080A00000050
:101FC40000000000C4DA030800000000AC13040899
:101FD4000A000000000000001CDA030800000000F2
:101FE400B41304080A00000000000000E8A900205F
:101FF40000000000BC1304080A00000000000000F8
:10200400D016002000000000740D04080100000038
:1020140000000000000000000000000000000000BC
:102024000E0000000000000000000000000000009E
:10203400C4130408000000000000000000000000B9
:1020440000000000D013040803000000313B030823
:102054002017002000000000E01204080300000024
:10206400313B03080817002000000000D4120408C4
:1020740003000000313B0308F016002000000000BC
:10208400DC1304080500000000000000DAA70020AB
:1020940000000000E4130408070000000000000032
:1020A400E816002000000000F013040807000000F8
:1020B40000000000E016002000000000740D040879
:1020C400010000000000000000000000000000000B
:1020D400000000000E0000000000000000000000EE
:1020E40000000000FC1304080000000000000000D1
:1020F4000000000000000000F8D9030803000000FD
:10210400313B030868170020000000001014040885
:1021140003000000313B0308C01C00200000000045
:102124001814040803000000313B03085017002072
:10213400000000002014040803000000313B0308E1
:102144003817002000000000740D0408010000008E
:10215400000000000000000000000000000000007B
:102164000E0000000000000000000000000000005D
:102174002C1404080000000000000000000000000F
:10218400000000003814040807000000395F030849
:10219400181800200000000030100408030000009C
:1021A400313B030800180020000000004414040818
:1021B40003000000313B0308E81700200000000082
:1021C4004C14040803000000313B0308D01700201E
:1021D4000000000054140408070000001D5F0308F9
:1021E400C81700200000000048160408030000007F
:1021F400313B0308B01700200000000060140408FD
:1022040003000000313B0308981700200000000081
:102214006C14040803000000313B030880170020FD
:1022240000000000740D040801000000000000001C
:102234000000000000000000000000000E0000008C
:1022440000000000000000000000000078140408F2
:102254000F000000755803083158030800000000FF
:1022640020180020801404080F000000F55A030809
:102274000000000000000000D41800208C140408A2
:102284000F00000015570308F9560308000000006A
:1022940060190020941404080F00000000000000DE
:1022A4000000000000000000141A0020A414040818
:1022B4000F000000CD5A0308555F0308000000001A
:1022C400A01A0020AC140408000000000000000064
:1022D4000000000000000000B8140408030000001F
:1022E400313B0308DC1B00200000000098140408A4
:1022F40003000000313B0308C41B00200000000061
:102304009014040803000000313B0308AC1B0020B8
:1023140000000000C014040803000000313B03085F
:10232400941B002000000000CC14040803000000EB
:10233400313B03087C1B002000000000D414040877
:1023440002000000453A03080000000000000000FD
:10235400DC14040802000000453A030801000000F0
:1023640000000000E814040802000000453A0308D5
:102374000200000000000000000000000E00000049
:102384000000000000000000000000000101010046
:10239400CC1604080F0000003156030800000000AA
:1023A40000000000401E0020A016040800000000E9
:1023B400000000000000000000000000C00A040843
:1023C4000000000000000000CC1E002004000000FB
:1023D4002C1604080D000000855D0308E02200208F
:1023E40000000000AC0F04080D000000555D030858
:1023F400D42200200000000090100408080000000F
:1024040000000000C8220020040000000C10040892
:102414000D0000006D5C0308BC22002000000000D9
:10242400A010040803000000313B0308A42200208C
:1024340000000000B016040803000000313B03084C
:102444008C22002000000000740D0408010000002C
:102454000000000000000000000000000000000078
:102464000E0000000000000000000000000000005A
:10247400A016040800000000000000000000000096
:1024840000000000C00A0408000000000000000072
:10249400CC1E002004000000D8150408030000002E
:1024A400BD5B030874220020080000000C1004081F
:1024B4000D0000006D5C0308BC2200200000000039
:1024C400A010040803000000313B0308A4220020EC
:1024D40000000000B016040803000000313B0308AC
:1024E4008C22002000000000740D0408010000008C
:1024F40000000000000000000000000000000000D8
:102504000E000000000000000000000000000000B9
:10251400B8160408000000000000000000000000DD
:1025240000000000C00A04080000000000000000D1
:10253400CC1E002004000000E01504080300000085
:10254400313B0308EC22002000000000740D040855
:102554000100000000000000000000000000000076
:10256400000000000E000000000000000000000059
:102574000000000020700020702D72002D202D2DF1
:10258400202D2D2D2D202D2D2D2D0000000000009F
:102594000000000000000000000000002D202D2D90
:1025A400202D2D2D2D202D2D2D00000000000000AC
:1025B400000000000000000000000000D6A700207A
:1025C40088130C1701000000D8A7002088130C17EB
:1025D40000000000301504080000000000000000A6
:1025E400000000000000000040150408080000007E
:1025F40000000000F81E0020040000004C15040830
:102604000800000000000000EC1E00200000000094
:10261400A010040804000000515C0308000000003E
:1026240000000000740D0408010000000000000018
:102634000000000000000000000000000E00000088
:10264400000000000000000000000000D4A70020EB
:1026540088130C1701000000D2A7002088130C1760
:1026640000000000881504080F00000089560308C4
:102674000000000000000000041F002022AA002027
:102684000100000080D70308D1A70020010000004A
:102694008CD70308AC5900200200000094D703082B
:1026A4002A8B00200000000000000000288B00207E
:1026B4000000000000000000268B00200000000045
:1026C40000000000248B0020000000000000000037
:1026D400228B00200000000000000000208B00205E
:1026E4000000000000000000D805002000000000E9
:1026F40000000000D0A7002002000000A0D70308BB
:102704009015040800000000000000000000000014
:10271400000000004015040808000000000000004C
:10272400881F0020040000004C1504080800000065
:10273400000000007C1F002000000000A01004081E
:1027440004000000695603080000000000000000B7
:10275400740D0408010000000000000000000000E7
:1027640000000000000000000E0000000000000057
:102774000000000000000000A01504080000000094
:10278400000000000000000000000000B015040874
:102794000D000000F55C0308C41F002004000000C5
:1027A400BC1504080D000000AD560308B81F002036
:1027B40004000000C81504080D000000B55C0308FF
:1027C400AC1F002000000000D41504080300000022
:1027D400DD5B0308941F002008000000E0150408D6
:1027E40003000000313B0308EC220020000000003D
:1027F400740D040801000000000000000000000047
:1028040000000000000000000E00000000000000B6
:1028140000000000000000006C0D0408000000002F
:10282400000000000000000000000000E81504089B
:1028340004000000B55D0308000000000000000073
:10284400740D0408010000000000000000000000F6
:1028540000000000000000000E0000000000000066
:10286400000000000000000034160408000000000E
:1028740000000000000000000000000054E1030814
:102884000D000000000000002420002004000000CF
:10289400441604080800000000000000182000206E
:1028A40004000000501604080800000000000000A6
:1028B4000C20002004000000581604080800000042
:1028C400000000000020002004000000601604083E
:1028D4000800000000000000F41F002004000000B5
:1028E400681604080800000000000000E81F00202B
:1028F4000400000070160408080000000000000036
:10290400DC1F002004000000781604080800000002
:1029140000000000D01F002004000000740D040813
:1029240001000000000000000000000000000000A2
:10293400000000000E000000000000000000000085
:1029440000000000801604080F00000079560308F8
:102954000000000000000000302000208816040859
:102964000F00000000000000000000000000000054
:10297400A8200020901604080F00000000000000AA
:1029840000000000000000004821002021AA0020CF
:1029940004000000ACD70308CCA70020E0150C17F6
:1029A40000000000CFA70020080000005CD7030847
:1029B400CEA7002005000000C0D70308981604081D
:1029C4000F000000000000000000000000000000F4
:1029D40098210020010000004300000000000000D6
:1029E40000000000000000000000000000000000E3
:1029F4000000000000000000430000000000000090
:102A040000000000000000000000000000000000C2
:102A1400000000000000000043000000000000006F
:102A240000000000000000000000000000000000A2
:102A3400000000000000000043000000000000004F
:102A44000000000000000000000000000000000082
:102A5400000000000000000043000000000000002F
:102A64000000000000000000000000000000000062
:102A7400000000000000000043000000000000000F
:102A84000000000000000000000000000000000042
:102A940000000000000000004300000000000000EF
:102AA4000000000000000000000000000000000022
:102AB400000000000000000089830308C9810308A6
:102AC40000000000591704082A0D040809DE030851
:102AD40009DE030809DE030809DE030809DE03082A
:102AE40009DE030809DE030809DE030809DE03081A
:102AF400FFFFFFFFFFFFFFFFFFFFFFFFFFFF0000E0
:102B04000100415343494900000000000000000057
:102B140000000000000000000000000000000000B1
:102B24000000415343494900000000000000000038
:102B34000000000000000000000000000000000091
:102B440000000000782400200000000000000000C5
:102B54000000000000000000000000000000000071
:102B64000000000000000000000000000000000061
:102B74000000000000000000000000000000000051
:102B84000000000000000000000000000000000041
:102B94000000000000000000000000000000000031
:0C2BA40000000000000000000100000024
:10800000002870B51EDB0928044620DD012303EBA0
:1080100083035B00B0FBF3F2092AF8D87BB10E4E64
:10802000B4FBF3F00928CCBF57223022A6FB03E5AE
:10803000024403FB1044EB0801F8012BF0D10023AC
:108040000B7070BD2D230B7040420131DBE73030E7
:1080500001F8010BF3E700BFCDCCCCCC884230B4A3
:108060004FF001042ED301FB04F4B0FBF4F58D4274
:10807000F9D284B1AAB901E0B0FBF4F5092DCCBF67
:10808000572230222A4404FB150003F8012BB4FBCD
:10809000F1F4002CF0D100221A7030BC7047B0FB14
:1080A000F4F5092DCCBF372230222A4404FB1500F9
:1080B00003F8012BB4FBF1F4002CF0D100221A706C
:1080C00030BC70470546002AEBD1D7E703685A1C3D
:1080D00002601970704700BF2DE9F047089C2578B1
:1080E000002B804689460CBF4FF0200A4FF0300A23
:1080F000661C35B3002A29DD334601E0024698B1FB
:1081000013F8011B501E0029F8D1971E60B13D469F
:10811000013D51464046C8476B1C002BF8DC2578D2
:1081200027EAE770013055B1041B29464046C8478D
:10813000301916F8015B002DF7D1BDE8F087BDE8D6
:10814000F087002A04DC2846BDE8F0870020EBE732
:10815000571EDCE783684268D0ED037A00EB8301A9
:108160000133934281ED040A836004BF00238360DE
:1081700000EB830393ED047A036870EE277A9A424A
:10818000C0ED037A77EEC77AC0ED037A0CDA0133DB
:1081900007EE103AF8EEC76AB7EE007A87EEA60A45
:1081A000036030EE070A704707EE102AB8EEC77A70
:1081B00087EE870A704700BF90ED057A90ED004A80
:1081C000D0ED066AD0ED014AD0ED047A90ED035A65
:1081D000D0ED025AA4EE007AB0EE406AB0EE470A43
:1081E000B0EE667AA6EE247A67EEC07AA0EE457A03
:1081F000E6EE257A80ED057AC0ED067A704700BF7D
:10820000D0ED057A90ED013AD0ED003AD0ED064A76
:1082100090ED024A90ED077A90ED035A90ED086ACE
:10822000D0ED045AC0ED067AF0EE406A27EE830ADC
:10823000C0ED056AA3EEA60A80ED087AA4EE240A32
:10824000A5EE470AA5EEC60A80ED070A704700BFF3
:10825000D0ED007A90ED017A30EE670AE7EE007A11
:10826000B0EE670AC0ED007A704700BF704700BFEC
:108270000A44914214D030B40139551E41F2210212
:1082800011F8014F082380EA042004044CBF82EA5D
:1082900040004000013B80B2F7D18D42F0D130BCAC
:1082A000704700BFF0B540F6280340F62C0240F6B8
:1082B000360540F6210440F64D1140F66A1740F6A7
:1082C000E1060380428040F6791340F68112458131
:1082D000848140F6611540F6DA04C18140F633012D
:1082E0000782468240F6F70740F6A7168382C282CD
:1082F00040F6C71340F6E7120583448340F6411564
:1083000040F65914818340F64911C783068440F62C
:108310004C0740F601064384828440F6011340F680
:108320002112C584048540F6410540F62F1441858D
:1083300040F62E118785468640F60A1740F68816C5
:108340008386C28640F6C80340F652020586C4877B
:1083500040F68A0540F63714818740F61711A0F8D9
:10836000447006878380C380038140F6530CC28526
:1083700014234FF0013E4FF0011745874FF00126BF
:10838000A0F846200125A0F84040A0F842100B4C70
:108390000B49A0F848C02822C0F84AE0C0F84E7047
:1083A000C0F8526080F85B50C465C0F8561080F881
:1083B000612080F85A3080F86030F0BD000A010A70
:1083C000980864004FF40063838270474FF40063A1
:1083D0008382704750F8043C012280F84520103811
:1083E00003B11847704700BFBFF34F8F0549064BD5
:1083F000CA6802F4E0621343CB60BFF34F8F00BF43
:10840000FDE700BF00ED00E00400FA0570B4037B57
:1084100004681F2B08D9203B2021626801FA03F36E
:108420001A421CD170BC70472021226801FA03F364
:108430001A42F7D042691449582000FB02125168D1
:108440005689CD680868296821F001012960828970
:1084500092B222EA06028281A36070BC7047426930
:108460000949582000FB021251685689CD680868F6
:10847000296821F001012960828992B222EA06026C
:108480008281E36070BC7047C092002030B4094B19
:108490001C786CB1084A002502EBC404116893886B
:1084A0004D628889083203439BB2A2428B81F5D189
:1084B00030BC7047809500208495002010B4037B69
:1084C00001681F2B09D9203B20224C6802FA03F3D4
:1084D0001C4214D15DF8044B704720220C6802FA4C
:1084E00003F31C42F6D00C4A406800241470026862
:1084F0005DF8044B22F0010202608B607047064A6F
:1085000040680024147002685DF8044B22F00102F8
:108510000260CB60704700BFE08C002070B504465D
:1085200082B01430E56D06236A464321A847B0B1F6
:108530009DF804009DF800609DF801109DF8025020
:108540009DF803209DF8053041EA062143EA002307
:1085500042EA0522A187E287A4F84030012002B058
:1085600070BD00BF70B5044682B00830656A06234E
:108570006A463B21A847A8B19DF804009DF8006019
:108580009DF801109DF802509DF803209DF80530DC
:1085900041EA062143EA002342EA0522E1822283DE
:1085A0006383012002B070BD2DE9F0410446164DF1
:1085B000084616460F462EF045FF2A68023011681D
:1085C0009072D4723B4610464F6922460221B8474A
:1085D00028680E4B0268C4721521817257691421F4
:1085E0002246B84730462EF02DFF296816300D6818
:1085F0008872CC7222466C6933460846A44616211E
:10860000BDE8F041604700BFDC240020DCD7030850
:10861000014B186804F05CB9C496002008B503F05B
:108620000FFE044B5B68C01AC0F5FA5020EAE070F8
:1086300008BD00BFCCA1002000B5002183B00A20F6
:108640002CF07CFA0F210A202CF078FA01AA0321E1
:1086500010202CF09BFA9DF90430DFED277ADFED36
:10866000275A06EE103A9DF9053006EE903A9DF92C
:10867000063007EE103AB8EEC66AF8EEE66AB8EED3
:10868000C77A76EEE76A36EE676A37EE677AF7EE14
:10869000007AB0EE675AA6EE255A194B0021B0EECB
:1086A000456AB0EE675AA6EEA55A0A20E7EE257A8B
:1086B000F3EE0E5A26EE256A25EE257A67EEA57AA8
:1086C00083ED006A83ED017AC3ED027A2CF036FA6D
:1086D0000DF10302012102202CF058FA0DF10302E2
:1086E000012109202CF052FA01210A202CF026FA4F
:1086F000012003B05DF804FB000000430000803B54
:108700000000002038B50B4C2378054653B90A4ABF
:108710006378106849212A460025257004F0FCFD85
:10872000012038BDFFF77AFF0028F0D003F0D4FD18
:10873000EDE700BFCCA10020C8A10020F0B54A4C55
:108740002579012D83B013D028D3022D0DD1474BAD
:108750001B780646002B77D16846FFF7D3FF20B180
:108760009DF8063013F0030022D0002003B0F0BDC6
:108770003E4E3378002B62D16846FFF7C3FF9DF869
:10878000003008B1DB0764D40023237133784BB188
:10879000002301330020237103B0F0BD334E337842
:1087A000002BF5D1012102202CF01EFA2379F0E7ED
:1087B0009DF801E09DF800109DF803709DF80220DF
:1087C0009DF805509DF80430207141EA0E2142EADF
:1087D000072243EA052309B212B21BB249425242B0
:1087E0005B42234806EE901A07EE102A07EE903AF5
:1087F00090ED005AD0ED015A90ED026AF8EEE66A6B
:10880000B8EEC77AF8EEE77A66EE856A27EE257A43
:1088100067EE867AFDEEE66ABDEEC77AFDEEE77A90
:1088200016EE901A17EE102A17EE903A31807280E9
:10883000B38001210A202CF081F903B0F0BDFFF7CD
:10884000EDFE002898D090E7FFF7E8FE00288CD1D5
:1088500082E7337823B9072103202CF0C5F9257965
:108860000135257181E700BFDC240020CCA1002068
:108870000000002038B5044690F8590000285AD16D
:1088800004F11405236E80226B212846984764204A
:1088900003F07CFD236E0722682128469847642058
:1088A00003F074FD236E00226B2128469847642054
:1088B00003F06CFD236E01226B21284698470F20A0
:1088C00003F064FD94F85320236E032A8CBF1A2210
:1088D00018221B21284698470F2003F057FD236ECE
:1088E00018221C21284698470F2003F04FFD236EC5
:1088F00094F852201A21284698470F2003F046FD8D
:10890000236E94F85420192128469847642003F0D8
:108910003DFD236E10223721284698470F2003F093
:1089200035FD2846236E0122382198470F20BDE8E7
:10893000384003F02BBD04F0BBF80546F0B10368E6
:1089400081881B6919409BD12023C171837104F078
:1089500041FA21460F4B41F8103F28462BF02AFFE1
:10896000AB88B3FA83F3C3F11F03012212FA03F3B6
:1089700086D009490A6813430B6081E7014604F079
:1089800029FA2146034B41F8103F28462BF012FFED
:1089900076E700BFD5830008003C014010B5802178
:1089A0000446806904F03EFC012003F095FC20465B
:1089B000FFF760FF10226A2104F1140003F0C0F9F0
:1089C000642003F0E3FCA069042104F02BFC0120E7
:1089D000BDE8104003F080BCF8B5057B466903682C
:1089E0001F2D29D9A5F120045F682021A1400F4245
:1089F0002A4613D01022A240D960DA605A68E240B9
:108A0000D10703D5012202FA04F4DC6004463046A3
:108A100003F0FAFE227B23681F2A20D9A2F120004E
:108A200008215A688140114200D0D9600422596857
:108A300082400A4221D1F8BD20211C68A9400C4285
:108A40002A460CD01022AA4099609A601A68EA401F
:108A5000D207DBD5012202FA05F59D60D6E7082191
:108A600018689140014200D099600421186801FA09
:108A700002F2024203D09A60F8BDDA60F8BDF8BD98
:108A800070B582B00446694614302BF0FFFEB0B1D9
:108A90009DF805009DF801609DF802109DF80350B7
:108AA0009DF804209DF8063041EA062143EA0023A0
:108AB00042EA0522A187E287A4F84030012002B0F3
:108AC00070BDF8B5174D2B78A32B28D16B78BE2B32
:108AD00025D1022229464FF6FF70FFF7C9FB124F3E
:108AE000AC1C22884AB1A618BE4218D2052A16D953
:108AF0002146FFF7BDFB3446F3E721460222FFF78C
:108B0000B7FB0222A118FFF7B3FB0634074B641B27
:108B10001C8041F60F53C31A58425841F8BD00203B
:108B2000F8BD00BF0040000800800008A0530020EE
:108B30000378202B024600F10100F9D0092BF7D071
:108B40002D2B2CD02B2B03BF5378B7EE000A0246F7
:108B5000B7EE000AA3F13001C8B209289FED467AAA
:108B600010D8F2EE046A07EE901AF8EEE77A12F8DF
:108B7000013FE7EE267AA3F13001C8B20928B0EE32
:108B8000677AF0D92E2B4CD003F0DF03452B0BD0A6
:108B9000F7EE007A67EE276A20EE260A70475378D0
:108BA000BFEE000A0246D5E710B451782D2959D0FE
:108BB0002B290ABF9178501C901C0024A1F130038E
:108BC000092B53D8002303EB830301EB430310F875
:108BD000011FA1F13002092AA3F13003F3D9B3F543
:108BE0009A7F28BF4FF49A73072B42D9DFED236A8F
:108BF0001A46F7EE007A083A072A67EEA67AFAD8FC
:108C000003F007032BB1F2EE046A013B67EEA67A8C
:108C1000FBD124B3C7EE276A5DF8044B20EE260A89
:108C200070475378A3F13001C8B2092802F101025C
:108C3000AAD8F2EE046AF0EE665A07EE901AF8EE41
:108C4000E77A12F8013F87EEA66AA3F13001C8B2B5
:108C5000092866EEA56A37EE067AEED994E767EE44
:108C6000276AD9E7901C91780124A7E7F7EE007AEC
:108C7000CFE7F7EE007AC5E70000000020BCBE4C4D
:108C8000B5EEC00ADFED317AF1EE10FACCBF30EE6E
:108C9000270A30EE670ADFED2E7A20EE270A30B57C
:108CA000FDEEC07A87B017EE904A054684EAE4707C
:108CB000002303A9A0EBE4700193009302932BF02F
:108CC000E1FF002CACBF20232D2303A88DF800303A
:108CD0002EF0B8FB012803A924D002282DD00328A8
:108CE00005BF3023684668468DF8013031F0BBFD82
:108CF00068462EF0A7FB0338C4B2224669462846D0
:108D000031F00FFE00232B5528462EF09BFB2E2220
:108D1000431C2A540DEB0401E81831F0C1FD28462C
:108D200007B030BD302368468DF801308DF8023031
:108D30008DF8033031F097FDDAE7302368468DF87F
:108D400001308DF8023031F08EFDD1E76F12033A19
:108D500000007A442DE9F041064615460846B6FB68
:108D6000F2F43CB905FB1464124B1B5D00F8013BA7
:108D7000BDE8F081B4FBF2F767B90E4B05FB17476E
:108D800005FB1464DA5D00F8012B1B5D00F8013B64
:108D9000BDE8F081B7FBF2F8B8F1000F02D0404611
:108DA000FFF7D8FF05FB1878024B13F8082000F8EE
:108DB000012BE3E7E0D703080368591C1A4601605A
:108DC00012F8021B0260587841EA0020704700BF89
:108DD00003685A1C02601878704700BF38B5044613
:108DE000006815462FF002FA22682A44226038BD36
:108DF000036810B40A0E5C1C04601A7003680A0C45
:108E00005C1C04601A7003680A0A5C1C04601A7017
:108E100003685A1C026019705DF8044B704700BF6C
:108E2000036810B40A0A5C1C04601A7003685A1CB8
:108E3000026019705DF8044B704700BF03685A1C4C
:108E4000026010B4197003680A0A5C1C04601A708E
:108E500003680A0C5C1C04601A700368090E5A1C33
:108E6000026019705DF8044B704700BF03685A1C1C
:108E7000026019700368090A5A1C02601970704771
:108E80002DE9F047002488B080460F461E46A146D3
:108E900005AD531C0393117839B3252933D1931CA5
:108EA000CDF810900393507830284ED04FF0000A40
:108EB000A0F13003DBB2092B42D96C2819D0642809
:108EC00000F0938024D825281CD063D9582876D068
:108ED00063281BD131784046B847039A531C03934B
:108EE0001178043601340029D7D1204608B0BDE8F6
:108EF000F087039B5A1C03921B78642B7CD02AD8E2
:108F0000252B54D1252140460134B847039AC0E7A8
:108F1000732833D044D975284FD106F1040E306838
:108F20002B4600220A217646FFF798F8049A00950E
:108F3000534639464046FFF7CFF8039A0444A8E762
:108F400004AA03A92BF07AFEB7E7D31C0393907809
:108F50004FF0010AACE7732B10D05BD9752B3AD0D8
:108F6000782B96D1A3F15802B2FA82F230685209F6
:108F70002B4610210436FFF771F8D7E73368049ABF
:108F80000093394600234046FFF7A6F80436044410
:108F9000039A7EE70028B9D1204608B0BDE8F087E3
:108FA0006E28B3D1039A336804361C6071E72AD95E
:108FB000582BD7D0632B8DD06BE77828A6D1A0F1A2
:108FC0005802B2FA82F2306852092B461021FFF79C
:108FD00045F80436AAE706F1040E30682B46002255
:108FE0000A217646FFF73AF8A0E7331D3068294694
:108FF0001E46FFF705F899E7331D306829461E46DF
:10900000FEF7FEFF92E7002B7FF443AF204608B047
:10901000BDE8F0876E2BC6D03BE700BF0EB400B5AD
:1090200084B005AB019053F8042B0649039301A8C3
:10903000FFF726FF019B00221A7004B05DF804EBD5
:1090400003B07047CD8000080FB430B583B006ABD5
:109050000A490B4853F8042B096800680193FFF78D
:109060000FFF084C0546206803F022FC0028FAD0C8
:10907000284603B0BDE8304004B07047AC41002042
:10908000B0410020C4960020DFED2B7AB4EEE70A51
:10909000F1EE10FA4ADDDFED296A9FED297A01E051
:1090A000B0EE670AB4EEC70AF1EE10FA70EE667A17
:1090B000F6DC9FED247AF4EEC77AF1EE10FA38D59B
:1090C000DFED1E6A9FED207A01E0F0EE407AF4EECB
:1090D000C77AF1EE10FA37EEA60AF6D4DFED1B7A66
:1090E000B4EEE70AF1EE10FA14DDDFED137A37EE95
:1090F000C00A60EE006A9FED166A9FED167ADFEDFA
:10910000167AA6EE867A20EE266AE6EE877AA6EE34
:10911000270A7047DFED117AB4EEE70AF1EE10FA94
:1091200044BFDFED087A37EEC00AE2E7F0EE407A9E
:10913000BFE7B0EE670AD1E7DB0F4940DB0FC9405C
:10914000E4CB1641DB0F49C0E4CB16C1DB0FC93FAE
:1091500092E741B99730083C15A82ABEDB0FC9BF7A
:1091600009B909E0194690FBF1F301FB1303084626
:10917000002BF7D1084670470146FBE7F0EEC07AB6
:10918000B0EEE07AB4EEE77AF1EE10FAB4BFB0EEEA
:10919000676AB0EE476AB5EE406AF1EE10FA46D063
:1091A000B4EEE77AF1EE10FA8CBFF0EE675AF0EE0B
:1091B000475AC5EE866A9FED1F3A9FED1F6A9FEDE5
:1091C0001F4A9FED1F5ADFED1F3ADFED1F4ADFED0B
:1091D0001F5AA6EEC36AE6EEA34AA6EE864AB7EE8B
:1091E000006AA6EE845AA6EEA46AE6EE855AC5EE9B
:1091F000866AB4EEE77AF1EE10FA48BFDFED147A32
:10920000F5EEC00A48BF77EEE66AF1EE10FA48BF05
:10921000DFED107AB5EEC00A48BF77EEE66AF1EEF0
:1092200010FA48BFF1EE666AB0EE660A7047DFEDED
:10923000076ADEE739094E3DE3B59E3E88FA163EE1
:1092400045FE7F3F99FB243F69A2163EA7DFA83465
:10925000DB0FC93FDB0F4940DFED317A30EE277A73
:10926000FDEEC76A16EE903A2033402B02D99FEDEF
:109270002D0A7047B4EEE70AF1EE10FA4DDD9FEDCE
:109280002A6ADFED2A6A01E0B0EE677AB4EEE67A88
:10929000F1EE10FA77EE467AF6DC9FED257AF4EEE1
:1092A000C77AF1EE10FA35D5DFED1F6A9FED217A0E
:1092B00001E0F0EE407AF4EEC77AF1EE10FA37EE04
:1092C000A60AF6D4DFED167AB4EEE70AF1EE10FA4C
:1092D0001BDCDFED197AB4EEE70AF1EE10FA44BFB9
:1092E000DFED137A37EEC00A60EE006A9FED136A75
:1092F0009FED137ADFED137AA6EE867A20EE266ACA
:10930000E6EE877AA6EE270A7047DFED0F7A37EE92
:10931000C00AE9E7B0EE670AD4E7F0EE477ABCE7A7
:10932000DB0FC93F00000000DB0FC940E4CB164152
:10933000DB0F49C0E4CB16C1DB0FC9BF92E741B9CF
:109340009730083C15A82ABEDB0F4940FDEEC07AD5
:1093500017EE903A2033402B51D8DFED2D7AB4EE42
:10936000E70AF1EE10FA50DDDFED2A6A9FED2A7A66
:1093700001E0B0EE670AB4EEC70AF1EE10FA70EE43
:10938000667AF6DC9FED257AF4EEC77AF1EE10FAF4
:1093900038D5DFED206A9FED227A01E0F0EE407AC9
:1093A000F4EEC77AF1EE10FA37EEA60AF6D4DFED46
:1093B0001D7AB4EEE70AF1EE10FA1BDCDFED1A7A43
:1093C000B4EEE70AF1EE10FA44BFDFED147A37EE9F
:1093D000C00A60EE006A9FED156A9FED157ADFED19
:1093E000157AA6EE867A20EE266AE6EE877AA6EE53
:1093F000270A7047DFED067A37EEC00AE9E79FEDEE
:109400000E0A7047B0EE670AD1E7F0EE407AB9E78E
:10941000DB0F4940DB0FC940E4CB1641DB0F49C0ED
:10942000E4CB16C1DB0FC93FDB0FC9BF92E741B9DF
:109430009730083C15A82ABE0000000010B507EEC2
:10944000901A2DED028BB8EE678ADFED217A28EEB7
:10945000008A044628EE278AB0EE480A2FF01CF94D
:10946000F0EE408AB0EE480A2FF078F8F7EE007A76
:109470009FED187AF0EE675AE8EE875A0023A36151
:10948000B0EE676AC7EEA56A63612362E361A8EE86
:10949000C76ABDEC028B77EEC07AB6EE007AF8EEC2
:1094A000005A27EE877A20EE250A27EE267A26EE46
:1094B000266A67EEA67A20EE260A84ED046AC4EDD9
:1094C000017A84ED007A84ED027A84ED030A10BDFE
:1094D00027D4D236F304353F10B44C09012250F89A
:1094E000243001F01F0102FA01F10B4340F824304F
:1094F0005DF8044B704700BF4B0901F01F0150F8A5
:109500002320012303FA01F1114214BF1846002061
:10951000704700BFAA4B33F81020110513D52DE971
:10952000F043A8490446400904F01F0551F8200003
:109530000121A940014291B006D0A349097B19B18C
:1095400011B0BDE8F083704702F01F07C2F3441565
:10955000242CF5D8DFE814F0430055009000A20059
:109560005201960196019B044A036A037002A0020D
:10957000BA02C502D802E302F402FD02C901CB041B
:10958000BD040A05D9010D020D0237024A024A0242
:109590008E03EF03FC030D041E048F0451048004AA
:1095A0002500DFF85482D8F820200AB1B2F908204B
:1095B000864908AE3046FFF731FD30462DF042FFB8
:1095C000D8F800403844A0722068E5722A46334635
:1095D000456939462046A84711B0BDE8F0837C4B69
:1095E0007C491A88DFF81082642303FB02F39B1284
:1095F00008AE632BA8BF632330460122FFF70EFDA0
:10960000DBE7754B754A1B781088022B00F0078545
:10961000734B744C5A781978247802EB820252000A
:1096200000EB800301EB81015B0093FBF4F39B1AD9
:10963000C3EBC303C2EB410293FBF2F3062BA8BFBB
:10964000062323EAE373C3F19603DBB2664A8DF87F
:109650002030A2FB0032D20802EB8203A0EB4303CE
:10966000624906209BB200900DF12100FFF7D6FC65
:1096700008AEDFF88481A0E7DFF87C81D8F800002D
:1096800003681B69984710AEB0F5F07F584B46F859
:10969000203D0CBF072506250D278EE793F8612096
:1096A000544993F86060B1F9000002EB8202530064
:1096B0005F4206EB8606B8424FEA460603DB83426A
:1096C000A8BF03461F46B1F902307542AB4203DB27
:1096D000B342A8BF33461D46DFF81C81D8F800000E
:1096E00003681B699847B0F5F07F05EB850518BF47
:1096F0000224BB0048BF3F3305EB850595FBF6F61A
:10970000293EC6EBA313512B40F22A8607EB4705EF
:10971000002D2B46B8BF05F13F03C6EBA313512B19
:1097200040F20186ED1B002D2B46B8BF05F13F032B
:10973000C6EBA313512B40F2D985ED1B002D2B4610
:10974000B8BF05F13F03C6EBA313512B40F28A8546
:10975000ED1B002D2B46B8BF05F13F03C6EBA3134D
:10976000512B40F2E184ED1B002D2B46B8BF05F1D3
:109770003F03C6EBA313512B40F2B984ED1B002D20
:109780002B46B8BF05F13F03C6EBA313512B40F2A4
:109790009184ED1B002D2B46B8BF05F13F03C6EBAE
:1097A000A313512B40F26984ED1B48BF3F35C6EB34
:1097B000A516512E40F2FA840420FFF7ABFEBFE657
:1097C000DEA70020205E00200000002058D80308FB
:1097D000B28C002028D80308B58C0020C059002086
:1097E0002C550020D6590020CDCCCCCC30D8030845
:1097F000267E270024550020DC240020DFF8E883A3
:10980000D8F8000003681B699847B0F5F07F0CBFDB
:109810000727062707F1040614BF0324042408259C
:10982000D8F800000368C4728572D3F818902246F5
:1098300013230721C847D8F8000016220368C47212
:10984000827222460134D3F8189015211323E4B212
:10985000C847A642E4D1D8F8000009220368C772BD
:1098600082729C693A4603230821A047D8F8000079
:1098700015220368C77282729C693A46022314213A
:10988000A0475DE603EB4403B3F8523013F00F0238
:1098900000F0DC83022A8CBF20219C21012AC3F323
:1098A00003148DF8201000F0D685C0F0D483022A6E
:1098B00000F0BE850023DFF830831A461846012CDD
:1098C00040F0B083A74EA84CA849A6FB0060400B0F
:1098D000A4FB00646409642606FB140000900DF1EB
:1098E0002100FFF79BFB08AE67E6A14BA14A186871
:1098F000A149047A83790194C079009008AE30467A
:10990000FFF78CFBDFF8E08257E69C4B9C4A1B88F4
:1099100012789C4903EB8303022A09784FEA430338
:1099200093FBF1F300F07983974A5178127801EBB9
:109930008101490002EB82005A1AC2EBC202C1EB5C
:10994000400192FBF1F2062AA8BF062222EAE27247
:10995000C2F19602D2B284488DF8202080FB032009
:10996000DA17C2EB601264248849062004FB123324
:1099700079E6874A874B8849DFF86C8292E8410094
:10998000182C08BF064683FB06234FEAE672C2EB9B
:10999000A35203A814BF602364238DF82030FFF77F
:1099A0003DFB32467C4905A8FFF738FB03A82DF0A4
:1099B00049FD05AB034403AA78490DF12100FFF7E7
:1099C0002DFB08AEF9E576487649B0F90230B0F9DA
:1099D0000020B0F90640B0F90400009008AE0194F0
:1099E0003046FFF71BFBDFF80082E6E56E4B6F4861
:1099F0006F49DFF8F4811A2C0CBFB3F90220B3F9D8
:109A0000002080FB0230D317C3EBA00404EB8400DA
:109A1000A2EB400383EAE370002AA0EBE37008AEF8
:109A200084EAE4730090ACBF20222D22A3EBE47300
:109A30003046FFF7F3FAC0E55E4E316800248DF83A
:109A40000B408DF80C40002900F02D850A68D26982
:109A5000002A00F00A8503A90DF10B009047316838
:109A60008DF8144031B10B68196A19B105A88847FF
:109A70009DF814109DF80C404F489DF80B204F4B5B
:109A8000825C009108AE53F824304D49DFF85881CC
:109A90003046FFF7C3FA90E54A4B33481B684A4902
:109AA000DFF8448183EAE37EAEEBE37E80FB0E3099
:109AB0004FEAEE72C2EB601208AE64209A2400FBFB
:109AC00012E300943046FFF7A9FA76E53D4B3F4993
:109AD0009A68DFF8148108AE30460723FFF79EFA34
:109AE0006BE52B4B3A4ADB893A49DFF8FC8003EB04
:109AF000C3039B0082FB030208AEDB17C3EBA21279
:109B00003046FFF78BFA58E5214B33491B7DDFF8D0
:109B1000D88008AE30461F22FFF780FA4DE593F853
:109B20005B302E49DFF8C080002B0CBF0F220C22C7
:109B300008AE0023009230461A46FFF76FFA3CE564
:109B40000B4B274A18680C498478037801944078B5
:109B5000D3E6074B234A186807494479C378019430
:109B60000079CAE65917B7D11F85EB5184D803088D
:109B7000A4A80020C4D80308B0D80308C059002006
:109B8000B58C0020D65900202C55002010D9030890
:109B9000485500206BCA5F6B58D803085CD803088F
:109BA000FC5800201CD9030824550020676666660F
:109BB00030D903086864002054D703085CD7030831
:109BC000A0D80308B85400203CD8030848D803089C
:109BD000D34D621050D8030828D803086CD8030866
:109BE000ACD80308C0D80308DC240020C54B1A7881
:109BF000002A00F0B6825C1E03F10F080DF11F0968
:109C000066782EF0D3FA30443246437803F00303EB
:109C1000022B14F8013F08BFA6F1200209F8012F1A
:109C2000002B00F08480A045EAD180E0B64BB74A13
:109C3000B3F90630B649DFF81C83B3F5FA6FA8BF55
:109C40004FF4FA63B3F57A7FB8BF4FF47A73A3F594
:109C50007A7382FB0302DB17C3EBA2020424052301
:109C60000DF122008DF820408DF8213008AEFFF76D
:109C7000D5F9A2E4A74BA84A1B899268A7499A1A6A
:109C80009A42A8BF1A4622EAE27207EE902AA1FB86
:109C90000313DB08B8EEE77A07EE903AF8EEE77ABE
:109CA000C7EE276A16EE900A2DF038FD41EC100B36
:109CB0002EF07AFB51EC100B2EF01EF88A23C0B266
:109CC0008DF82030002840F09E818D238DF82130C2
:109CD0008D238DF82230022800F26B818D238DF8C0
:109CE00023308D238DF824308D238DF825308D235E
:109CF0008DF826308D238DF827308D238DF8283070
:109D00008D238DF829308D238DF82A308D238DF801
:109D10002B30431E8F22092B8DF82C2004D810AB3A
:109D200018448E2300F81F3C00238DF82D3008AE18
:109D3000DFF8208241E47A4B1B78DB073FF500AC6B
:109D400008AE30467749DFF80C82FFF767F934E454
:109D5000754B1B7803F00303032B00F019832D23AD
:109D60008DF8203000238DF8213008AEDFF8E48133
:109D700023E46D4A127802F00302032A00F03B83C9
:109D80002D2200238DF820208DF8213008AEDFF839
:109D9000C48112E4654B5D4AB3F9043064486549F7
:109DA000DFF8B08182FB0342DB17C3EBA2031BB2D7
:109DB000162404EB430480FB04621619E217C2EB7D
:109DC00066224FF4347606FB124280FB02401044B8
:109DD000D217C2EB6012D2B2C2F11802504200F0A8
:109DE0000F0002F00F0258BF4242603208AED2B2FA
:109DF0003046FFF713F9FFF7E0BB4C4B434CB3F988
:109E000004304B484C49DFF84C8184FB0324DA17BB
:109E1000C2EBA4021623022412FB043280FB02438D
:109E20009C18D317C3EB64234FF4347404FB13233F
:109E300080FB03021A44DB17C3EB621351FA83F36E
:109E400008AE186859681C7A334603C300221C7098
:109E50008DF82920FFF7B1BBDFF8F880D8F8202073
:109E60000AB192F90120354908AE30460E23FFF7BA
:109E7000D5F8FFF7A2BB08AE002330460093682256
:109E80002F49DFF8D080FFF7C9F8FFF796BB2D4BBD
:109E90001B68DC0040F1CE802B4B03222B49098844
:109EA000480500F18380CE0700F1BF8201F0020176
:109EB000274800291CBF03220346264908683A4464
:109EC00004688272C57239462A466469A047FFF762
:109ED00037BB214A214953781278DFF8788008AEE1
:109EE000013301323046FFF799F8FFF766BB1C4A91
:109EF000094B10881B681B4A1B49DFF8588003FB7D
:109F000000F3F7E5D0510020088D002067666666F3
:109F100058D803082C550020B8540020A38B2EBA23
:109F2000045C00203CD9030844550020245500203F
:109F3000B7600BB648D9030884A9030864D803089E
:109F400050D903084450002008D80308308D002061
:109F500024D80308DC240020B4900020D0D80308C3
:109F6000C0590020D34D6210C8D803080021CC4846
:109F7000FFF7C2FA002840F03281CA4B1B7813F079
:109F8000020FC94B1B7802D1002B00F07882012B05
:109F900000F00381022B40F0F28008AE3046C34946
:109FA000DFF84483FFF73AF8FFF707BB0422C04B02
:109FB00083E78B2303288DF823307FF692AE0428A5
:109FC0008DF824307FF690AE05288DF825307FF689
:109FD0008EAE06288DF826307FF68CAE07288DF8D9
:109FE00027307FF68AAE08288DF828307FF688AEB5
:109FF00009288DF829307FF686AE0A288DF82A3098
:10A000003FF685AE82E68B2301288DF8213018BFFC
:10A010008DF822307FF45FAE5AE697229BE49723B7
:10A02000FFF714BBA3490DF12100FEF7F7FF08AEBF
:10A03000FFF7C3BAA04AA1491268A14B02F48002FB
:10A04000002A0ABF0B460322042227E79B22C3F300
:10A0500003148DF8202002F0F3F89A4B9A4ADFF8A7
:10A060008882A3FB00139B0C82FB03121A4452113B
:10A07000C2EB0211A3EB810321E49449D8F800005C
:10A0800081FB0321DA17C2EB610204EB020E02EB43
:10A09000C2015B1A5FFA8EF20168C2724FF0120EB3
:10A0A00080F80AE0803BD1F81890DBB21121C84754
:10A0B000FFF77ABB8549D8F8000081FB0321DA1746
:10A0C000C2EB610204EB020E02EBC2015B1A5FFA03
:10A0D0008EF20168C2724FF0110E80F80AE0803BE8
:10A0E000D1F81890DBB21021C847FFF752BB77496F
:10A0F000D8F8000081FB0321DA17C2EB610204EB00
:10A10000020E02EBC2015B1A5FFA8EF20168C272A4
:10A110004FF0100E80F80AE0803BD1F81890DBB2C7
:10A120000F21C847FFF72ABB6849D8F8000081FB18
:10A130000321DA17C2EB610204EB020E02EBC2014B
:10A140005B1A5FFA8EF20168C2724FF00F0E80F850
:10A150000AE0803BD1F81890DBB20E21C847FFF728
:10A1600002BB5B4BDFF8808193E8070008AE334603
:10A1700003C323F8022B120C1A70FFF71EBADFF884
:10A18000688198F81C30002B3FF4DAA908AE3046FD
:10A190005049FEF743FFFFF710BA08AE30464E496C
:10A1A000DFF84481FEF73AFFFFF707BA474AD8F8CD
:10A1B000000082FB0632F317C3EB6203E21803EBE5
:10A1C000C3031324D2B2F61A0168C272A6F1800347
:10A1D00084728C69DBB21221A047FFF7EDBA3F4BC6
:10A1E0001B88002B3FF4C9AEDC0700F16081C3F38C
:10A1F00040025ABB580700F17481190700F16F81C2
:10A20000DA0600F16A819E0600F165815C0600F1C4
:10A210006081180600F15B81D90500F156819A052D
:10A2200000F151815E0500F14C811C0500F1478170
:10A23000D80400F14281990400F13D815A0400F1F3
:10A240003881DB0B18BF0F223FF471AD244B254939
:10A2500053F82220DFF8908008AE3046FEF7DEFE8D
:10A26000FFF7ABB91949D8F8000081FB0321DA17D1
:10A27000C2EB610204EB020E02EBC2015B1A5FFA51
:10A280008EF20168C2724FF00E0E80F80AE0803B39
:10A29000D1F81890DBB20D21C847FFF759BA00BFBB
:10A2A00044500020045C0020B58C0020F8D803083E
:10A2B00014D8030878D80308A88E00200CD8030807
:10A2C00008D8030883DE1B4389888888398EE338E1
:10A2D00094D8030804D90308ECD80308DC8C0020C8
:10A2E000D0B70308D8D80308DC2400207E49D8F86A
:10A2F000000081FB0321DA17C2EB610204EB020EBE
:10A3000002EBC2015B1A5FFA8EF20168C2724FF073
:10A310000D0E80F80AE0803BD1F81890DBB20C21DA
:10A32000C847FFF70ABA7049D8F8000081FB03213B
:10A33000DA17C2EB610204EB020E02EBC2015B1AF8
:10A340005FFA8EF20168C2724FF00C0E80F80AE0DC
:10A35000803BD1F81890DBB20B21C847FFF7E2B978
:10A360006149D8F8000081FB0321DA17C2EB6102D2
:10A37000A51802EBC2015B1AEAB20168C2720B2592
:10A38000803B85728D69DBB20A21A847FFF7BEB911
:10A39000564B1B88002B6CD0554B5648B3F90430F4
:10A3A000554A5649B2F9002080FB0340DB17C3EB46
:10A3B000A0031BB2D21A5200163281FB0203981876
:10A3C000D317C3EB60234FF4347000FB132381FBDE
:10A3D00003121A44DB17C3EB6213DBB2C3F1180399
:10A3E0005A4202F00F0203F00F0358BF534260338A
:10A3F0008DF82030B6E43D4A93F85B301288002B8C
:10A400003BD14FF4A4733E4903FB02F281FB0213DC
:10A41000D217C2EB63120F2308AE30463949DFF87A
:10A420000481FEF7FBFDFFF7C8B8374B042244E573
:10A43000DFF8F0803549D8F81800354AA1FB003123
:10A44000890C82FB01320A445211C2EB0213A1EBC8
:10A450008303FFF734BADFF8CC802C4BD8F8080020
:10A460002B4AA3FB0013990CEBE78DF81420FFF7A0
:10A47000FABA05238DF8203074E40C23CCE7254A82
:10A48000254B2649927B1B88097893FBF1F39A426E
:10A490007FF675AE08AE30462149DFF88880FEF7BA
:10A4A000BDFDFFF78AB88DF81410FFF7E3BA00225C
:10A4B000CCE60E22CAE60D22C8E60C22C6E60B2226
:10A4C000C4E60A22C2E60922C0E60822BEE6072246
:10A4D000BCE60622BAE60522B8E60422B6E6032266
:10A4E000B4E60222B2E600BF398EE338A48D002024
:10A4F0002455002067666666A68D0020B7600BB6FF
:10A500001F85EB5164D803081CD8030883DE1B4366
:10A51000898888882C550020C0590020D6590020F1
:10A52000DCD80308DC2400202DE9F04F714B724C7D
:10A530001B788DB005460BB101232377626A6F4B00
:10A54000A3FB02139B0803EB8303511CD31A616224
:10A5500040F0B3806A4F94F8281097F8008008F014
:10A560000108414500F09281B8F1000F40F0E88009
:10A57000D4F80090634ED9F8003048469B6898475D
:10A580002068FF2389F80D300122036889F80C2028
:10A59000112102228172C272D3F814905A4B1146D3
:10A5A000C84796F85230002B40F09E830A23079349
:10A5B00009230693082305930623049305234FF0EC
:10A5C000070A03934FF0040B4FF0030896F853303B
:10A5D000002B40F03A8396F84A30DFF8589123B1C7
:10A5E00099F800309B0700F14D8496F85430CBB1B8
:10A5F00096F85B30B4F91620002B00F0C7830C23CB
:10A60000424909A8FEF70AFD404609AA4049FDF75C
:10A61000CBFF049BCDF810A0DDF814A0D846DDF8E0
:10A620000CB0039396F84B30002B40F0B68296F8AE
:10A630005130DFF804A1002B40F0E98296F84C304D
:10A64000002B40F0CD82334B9B79002B40F04082B1
:10A65000DFF8E8B096F84F30002B40F0638296F8B0
:10A66000503093B12C4B9B7803B3032B1ED00022A8
:10A670002A4909A8FEF7D2FC08F10103404609AABD
:10A6800027495FFA83F8FDF78FFF96F855306BB1D5
:10A69000214B9B7853B1032B08D009A900202AF045
:10A6A000F1FA09AA40461F49FDF77EFF1E4A1F4ED8
:10A6B0002A4400233260A3616AE020680368DB68F3
:10A6C0009847236863B193F90E30002B08DD184AD0
:10A6D000138843F480439BB213800DB0BDE8F08F24
:10A6E000134A138823F480439BB213800DB0BDE856
:10A6F000F08F00BFDE8C0020DC240020CDCCCCCC41
:10A70000045C0020DEA7002064D9030864D8030895
:10A7100080D903082C550020F2A90020F0D90308A5
:10A72000F8D9030804DA030800879303285E0020A1
:10A73000DC8C002044550020C0590020B854002073
:10A74000266863613068A3614FF0FA714FF4C60266
:10A750008368E1603046226198472068DFF86093A3
:10A76000DFF860A3DFF860B3FF237373012203688F
:10A770003273112107228172C272D3F81480C04B48
:10A78000C04E0C21C04705F5F42202F590723260EC
:10A79000397801F0010184F82810BB4BDFF82CE375
:10A7A000DB89BA4803EBC3039B008EFB03CEDB17A8
:10A7B0000788B4F90C00C3EBAE131BB29842B8BFC4
:10A7C000A381B4F90E00BAF800309842C8BFE38103
:10A7D000AF48DBF800304FF0640E80FB03C0DB179E
:10A7E0000EFB07F7C3EB6013B4F910E01BB29E45F4
:10A7F000B8BF2382B4F91230C7F38727BB42B4F93C
:10A800001430C8BF6782002BBCBF0023A38299F815
:10A81000003084F8297003F00303032B2ED039B1E4
:10A82000E36AA068A169EB1A18440B44A060A36115
:10A83000E5626AB1AA1A002A31DB27683B6838460C
:10A840009B6898470121FF22002339737A73336094
:10A850009049914F914A3B68AD09A1FB0515C5F39D
:10A86000801515731D0100F10581236853B393F919
:10A870000E20002A26DD0022227723E7884BB4F938
:10A8800016001B889842B8BFE382C8E77D4EDFF808
:10A8900030923268DFF82CA2DFF82CB27DE7814AD3
:10A8A000B2F9061040F2D663994203DCB2F90220F5
:10A8B0009A4201DD00233360206803681B6A9847D1
:10A8C0002368D8E7784E94F8293096F85A209A42AF
:10A8D00040F22381754D2B6843F00103744A1278CE
:10A8E000002A40F0158123F4C00323F0020399F8F5
:10A8F0000020900700F1098143F48043B6F85C80A2
:10A900002B6008F00F02012A00F0BA82C0F0B48276
:10A91000022A00F048820020664A4FEA182802FB0B
:10A9200008F2002A00F07182824200F26E8243F047
:10A930002003B6F85E802B6008F00F02012A00F0B9
:10A940006A82C0F06C82022A40F06782A069594A8C
:10A950004FEA182802FB08F2002A00F053828242D4
:10A9600000F2508243F04003DBF80820B6F856109E
:10A970009142B6F85820D4BF43F0102323F010239F
:10A98000002A00F0458223F4004326682B603368D8
:10A9900030469B6898470122FF233273737313215B
:10A9A0004548FEF7A9FD002886D1444D2B6899073C
:10A9B00000F1B5820120FEF7ADFD0020FEF7AAFDF3
:10A9C0000220FEF7A7FD0520FEF7A4FD0620FEF7F6
:10A9D000A1FD0720FEF79EFD0920FEF79BFD0A2042
:10A9E000FEF798FD0B20FEF795FD0C20FEF792FD7B
:10A9F0000820FEF78FFD0F20FEF78CFD1020FEF7DC
:10AA000089FD1120FEF786FD1220FEF783FD13203D
:10AA1000FEF780FD1420FEF77DFD1520FEF77AFD80
:10AA20001620FEF777FD1920FEF774FD1A20FEF7B9
:10AA300071FD1B20FEF76EFD1C20FEF76BFD1D2037
:10AA4000FEF768FD2020FEF765FD2120FEF762FD80
:10AA50002220FEF75FFD2B689A0600F14D823B68CD
:10AA60001B017FF529AF2320FEF754FD2420FEF7BC
:10AA700051FD21E7FF201EF003F92062F5E600BF3B
:10AA80005CD90308285E002048550020B28C0020C5
:10AA90001F85EB51632D3E05A88E0020000000208D
:10AAA000A48D0020088D0020DEA70020205E00205D
:10AAB000B58C0020008793034450002040550020AF
:10AAC00044550020C0590020B8540020D34D6210D6
:10AAD00096F84D30002B40F0EC8196F84E30DFF8C0
:10AAE00090B3002B3FF4B6ADDBF80820CE4909A89F
:10AAF0000723FEF793FA08F10103404609AACB4960
:10AB00005FFA83F8FDF750FDA4E523F48043F5E6F2
:10AB100043F4C00343F00203E9E6C54D2B6823F07C
:10AB20000103DBE696F85B10B4F914E0002900F0AD
:10AB30003C81C04A4FEAEE7382FB0E02C3EB621205
:10AB4000002AB8BF5242BEF1000FC0F2EE81DFF81A
:10AB5000E4C28CFB0E0CC3EB6C13B7484FF0640CD3
:10AB60000CFB13E380FB03E0DB17C3EBA003002B1C
:10AB7000B8BF5B4200290CBF0F210C21009109A82E
:10AB8000AE49FEF74BFA08F10103404609AAAC4969
:10AB90005FFA83F8FDF708FD61E5B4F90E30A64AC7
:10ABA000A84982FB0302D817C0EBA20202EB820085
:10ABB0004FF0060EA3EB40031BB212B2CDF800E03B
:10ABC00009A8FEF72BFA404609AA9F49FDF7ECFCBD
:10ABD000049BCDF810A0D846DDF80CB0039326E511
:10ABE00009AA1146B4F9120004922AF04BF8049A0B
:10ABF00010462CF027FC954B049A1B88135294495D
:10AC00004046FDF7D1FCD846DDF80CB01BE5BAF89C
:10AC10000030904A8B49A2FB0302D20802EB82006B
:10AC20004FF0060EA3EB40039BB2CDF800E009A85D
:10AC3000FEF7F4F9404609AA8749FDF7B5FC049BE5
:10AC4000D846DDF80CB00393F8E4B6F85E3003F0B4
:10AC50000F02012AC3F3031900F0CF80C0F06B810B
:10AC6000022A40F06481D4F818E07C4B7C4AA3FBB4
:10AC70000E139B0C82FB03121A445211C2EB0211F9
:10AC8000A3EB8103B9F1010F40F02881DFF8E4C1A3
:10AC900068487449ACFB0ECE4FEA5E3EA0FB0EC086
:10ACA00040094FF0640C0CFB10E00DF124090090FA
:10ACB0004846FEF7B3F9B6F85E306B4903F00F0370
:10ACC000404651F823104A46FDF76EFC049BCDF830
:10ACD00010A0D846DDF80CB00393069BDDF814A055
:10ACE0000593079B069376E4B6F85C3003F00F02F9
:10ACF000012AC3F3031900F08380C0F02481022AE3
:10AD000040F01D81A069554B554AA3FB00139B0CD5
:10AD100082FB03121A445211C2EB0218A3EB880300
:10AD2000B9F1010F40F0E180DFF848C1DFF804E13C
:10AD30004C49ACFB00C0400BAEFB00CE4FEA5E1EA0
:10AD40004FF0640C0CFB1E000DF1240900904846E6
:10AD5000FEF764F9B6F85C30434903F00F034A4646
:10AD600051F823100320FDF71FFC0B2307930A2340
:10AD70000693092305930723049306234FF0080A3B
:10AD800003934FF0050B4FF004081FE402EB82031E
:10AD900002EBC3022749D30081FB0321DA17C2EB80
:10ADA00061120F232CE4A069B6E50EEB8E000EEBCA
:10ADB000C00E2E4A1F4B4FEACE004FEAE07E82FBC8
:10ADC00000C2CEEB2232002A83FB00C0B8BF524241
:10ADD000DEEB601E00F1A78083FB0E314FEAEE73BD
:10ADE000C3EB61136420144900FB13E381FB0301EF
:10ADF000DB17C3EBA1030F21C0E6D4F808E034E76A
:10AE0000A06880E723F04003AEE523F0200390E53F
:10AE100043F40043B9E5A06899E5002097E501F007
:10AE20000FFA2B6893E500BF64D80308C8D903085C
:10AE3000205E00201F85EB5167666666D4D9030843
:10AE4000E0D9030830D8030890D90308A8D903082B
:10AE5000ACD90308CDCCCCCC9CD9030883DE1B43F2
:10AE60008988888884D8030800D60308AD8BDB68FE
:10AE7000B85400205917B7D101F0E2F92B684BE51F
:10AE8000A06849E509A9B4F90C0029F0FBFE404689
:10AE900009AA2E49FDF788FB049BCDF810A0D846DF
:10AEA000DDF80CB00393069BDDF814A00593FFF7C3
:10AEB0009CBB09AA1146B4F91000039229F0E2FEE6
:10AEC000039A10462CF0BEFA214B039A1B881352AA
:10AED00020494046FDF768FBD846FEE50DF1240900
:10AEE00048461D49FEF79AF8E5E60DF12409484663
:10AEF0001949FEF793F82DE70E20FEF70BFB0D2006
:10AF0000FEF708FB1820FEF705FB1720FEF702FBF3
:10AF10001F20FEF7FFFA1E20FEF7FCFA9FE5032034
:10AF2000FEF7F8FA46E54FEAEE7352420FE60023C9
:10AF30001A469E46A6E601F083F9864695E6434604
:10AF400042464046ECE601F07BF9DCE674D90308A2
:10AF5000B8D90308BCD9030878D80308F8B5334B2F
:10AF60001B78012B57D0324D324E3348334F0124DA
:10AF700005232946EB742C722C7522F093FB304884
:10AF800030493268304B0C7001685C714FF0000E34
:10AF9000DFF8C4C02D4B85F809E042F0415242F47D
:10AFA000005241F00E010225FC71BD70326001605B
:10AFB0008CF803E04B2503F1EA0E242219244627DE
:10AFC0001E2064214FF4C876DD701A715C711D700B
:10AFD0005A709C709F71DA715875D87583F8371064
:10AFE00083F836105E864E337345EDD1184B6420DE
:10AFF00003F124060021502255254FF4C86418702F
:10B00000587099705A719A71DD7119725C810C33A4
:10B01000B342F4D1F8BD0F4B40F29A204FF4876150
:10B020004FF4FA62188019825A829CE7DC2A0020C9
:10B030001C90002024AA002010DA0308848E00202F
:10B04000E44C0020E85100208C580020B2A80020D9
:10B05000BAA9002098920020045200202DE9F04364
:10B06000314A324E13683060042B89B004D0304C22
:10B07000591C44F8230011602E4B2F4A1B780021E5
:10B0800003F001031160516086F82830012702F0B7
:10B09000BFF8A0230424FDB203E00134E4B21C2C69
:10B0A00013D0FF2BF9DC306802688472C572611E10
:10B0B0000134D2F8188003F10109C9B2DBB22A4683
:10B0C000E4B2C0471C2C4B46EBD10137052FE1D130
:10B0D00068461A4A1A49FDF7A1FF6B460622142159
:10B0E000306802F071F8174B30680822072102F02F
:10B0F0006BF8154B306809220B2102F065F80A2223
:10B100000B21124B306802F05FF8306803685B6A0D
:10B11000984701F095F80E4B00F5741000F510609B
:10B12000186009B0BDE8F0839C970020DC24002063
:10B13000A0970020045C0020205E00201CDA030899
:10B1400024DA030828DA030838DA030844DA0308A3
:10B15000285E00202DE9F84FDFF8B4A0DFF8B490A6
:10B16000DFF8B480274E012308208AF8003029F048
:10B17000D7FAD9F8000001F0E5FE052029F062FABF
:10B18000002029F05FFA062029F05CFA002029F05F
:10B1900059FA98F80040042044F0010429F052FACA
:10B1A000204629F04FFA33888BB1174D174F0024F2
:10B1B00015F804B0072029F045FA584629F042FA5C
:10B1C0002A5D33883A550134A4B2A342F0D807204F
:10B1D00029F038FAFF2029F035FA98F800400420C9
:10B1E00029F030FA204629F02DFAD9F8000001F0B4
:10B1F000AFFE042029F094FA00238AF80030BDE85D
:10B20000F88F00BFEC050020185C0020445E002091
:10B210002D5E0020A8900020355E00202DE9F04131
:10B220004A4E082029F07CFA306801F08BFE484B2A
:10B230001B78012B7BD062D3022B0AD1DFF830813F
:10B24000082388F800300D254FF4C373414F3B802D
:10B2500010E0DFF81C813F4F98F8003003F0400306
:10B26000002B14BF4FF4F0734FF4C3733B8014BF33
:10B2700010250D25002404F11000C0B229F0E2F9D8
:10B280000134012029F0DEF9A3B2AB42F3D398F8E0
:10B290000040314D002029F0D5F9204629F0D2F99F
:10B2A0002E4B1C78022029F0CDF9204629F0CAF94E
:10B2B0002B4B1C78032029F0C5F9204629F0C2F950
:10B2C000284B1C780420044329F0BCF9204629F0BF
:10B2D000B9F9306801F03CFE042029F021FA3A88DF
:10B2E000214800212FF099FA6B7B33B11F4B1B785B
:10B2F00033B300236B73BDE8F081BDE8F081A0207B
:10B3000029F0A0F9002029F09DF900F00603022B96
:10B31000DFF85C8007D000F00500012803D1482346
:10B3200088F8003008E0082388F800308BE7DFF861
:10B330004080482388F8003010254FF4F07385E7EB
:10B34000FFF708FF00236B73BDE8F081A890002091
:10B35000C0900020EC05002000000020C7900020D5
:10B36000C8900020355E0020445E00202D5E002045
:10B37000EE0500200C4B984213D0A3F58063984251
:10B380000FD003F5804398420BD003F580639842B9
:10B3900007D003F58063984203D0044B1868400837
:10B3A0007047024B1868704700040140D491002098
:10B3B000F0B5774B774A87B01968914200AF00F03B
:10B3C000DB800023744A3B607B60136843F4803366
:10B3D000136003E03B68B3F5A04F09D0136803F492
:10B3E00000337B603B6801333B607B68002BF1D00E
:10B3F000694B1B6813F4003318BF01237B607B6823
:10B40000012B7BD0654D644B654AEA606549586FF6
:10B41000654A0860AA605E6B644C654A654826F020
:10B4200080065E635E6F46F080765E67196B0C4344
:10B430001C63596B5963996B9963196C41F05B51AB
:10B4400041F47B1141F41F6141F00F011964596C03
:10B4500007F118040A4348F2FF715A6444F8101DBA
:10B46000002621460123FB733E737E73BE731EF0DC
:10B47000C3FD21464FF6FF734F48BB601EF0BCFD75
:10B480004FF6FF7321464D48BB601EF0B5FD2146C7
:10B490004B481EF0B1FD21464A481EF0ADFD214645
:10B4A00049481EF0A9FD214648481EF0A5FD214649
:10B4B00047481EF0A1FD214646481EF09DFD20464E
:10B4C0001EF0BCFE444B454C1B68BA6844484549D5
:10B4D000A4FB03439B09A0FB0202013B920CB3F1C6
:10B4E000807F0A6007D2404AF0200721536085F828
:10B4F0002300966011601C37BD46F0BD264B3B4CC7
:10B500001A6C3B4942F080521A6420684A690D69FE
:10B51000896940F4404020609868986098681206F5
:10B5200040F40040986042EA8512986842F4800234
:10B53000490842F00802013942EA014240F4A050B1
:10B5400098605A601A6842F080721A601A68920114
:10B55000FCD52849104A40F205700860996821F02E
:10B5600003019960996841F002019960936803F0C2
:10B570000C03082BFAD145E700221A6062B61E4B75
:10B580001B6883F308881D4B1B689847FEE700BFC4
:10B59000FCFF0120EFBEADDE0038024000ED00E010
:10B5A0000005FA05BC87002000000008FF91670035
:10B5B000335F070000000240000402400008024020
:10B5C000000C02400010024000140240001802402B
:10B5D000001C024000200240D4910020D34D621094
:10B5E00083DE1B43C4A1002010E000E00070004097
:10B5F00000000020003C02400000FF1F0400FF1F6D
:10B6000008B5054B1B6803B19847044B044A1A6000
:10B6100072B6FCF7E9FE00BFCC730020FCFF0120EE
:10B62000EFBEADDE2DE9F04FDFF850914E4F8BB0FD
:10B630000326A7EB09071822002104A82FF0EDF834
:10B640004A4BCDF8109005971A69002A04DA484A47
:10B650005A6002F188325A6001228DF82420F322C8
:10B66000DA60444B444C1B88ADF800300222694636
:10B6700004A802F047F8022269464FF6FF70FCF773
:10B68000F7FDDFF8FCA080464FF0000B54453BD39C
:10B690000AAC002524F8245D0222214604A802F009
:10B6A00031F8022221464046FCF7E2FD40BAC04391
:10B6B000ADF80800022202A904A802F023F80798B6
:10B6C00078B106ABC0F10402294618442FF0A5F862
:10B6D000089818B9069904A801F075FF002308908E
:10B6E00007939DF82430089A23B120490B6943F051
:10B6F00000430B61013E2FD0002A9CD1FDF7E1F9F8
:10B7000060B30BB0BDE8F08F65888DF80DB0C5F360
:10B710000B05AB1DADF808302388C3F30B02ADF861
:10B720000A201B0B062202A904A88DF80C3001F098
:10B73000E9FF062202A94046FCF79AFD61688046AF
:10B740002A4604A801F0DEFF616840462A46FCF75D
:10B750008FFD1434804699E7002ACFD0052024F0CD
:10B76000D3FCFFF74DFF00BF00800008003C024003
:10B77000230167459CA903088801000800400008D0
:10B78000D405000808B5034B1B6803B1984772B68F
:10B79000FCF72AFECC73002070B50F4C0F4DC0EBA8
:10B7A000C00004EB8004286B26693043286382B014
:10B7B0009209667BA1600025012101A863618DF8D3
:10B7C00004608DF805208DF806508DF807101EF0E6
:10B7D00091FD02B070BD00BF1C0600200038024081
:10B7E0002DE9F04F6A4C54F8205083B0002D00F042
:10B7F000CA80EE6D002E00F0C8803769D6F804C00C
:10B80000644CA96005F162012C60696105F2622453
:10B810004FF400719B46AC61E9602961C5F854C0E2
:10B82000AA4647B35C4C4FF0000E21464B689F423E
:10B8300001F11C0106D00EF1010EBEF1100FF5D181
:10B840004FF0000ECEEBCE0E04EB8E04DFF85081ED
:10B850002369D8F830104FF00C0941EA030E411C5F
:10B86000C8F830E084F818906176B168A9630CF1EB
:10B8700004042C652F630746F068D946904640B310
:10B88000454C002123465A68904203F11C0365D0C1
:10B8900001311029F7D100210846C1EBC10104EBA9
:10B8A0008104DFF8FCE02369DEF830203B491343D4
:10B8B000CEF830300B227B1C63762276F27F2B464B
:10B8C000FFF76AFF6B6DB168F2686A630433E9637E
:10B8D000EB6495F8610001F0EBF8044695F8600020
:10B8E00001F0E6F88346307F002849D119F0080FAF
:10B8F00036D118F0020F09D044B10B227B1CA27183
:10B90000E3712046727F222101F098F918F0010FAF
:10B9100015D1AB6B7BB996F82020B17F8DF806303E
:10B9200001A8930901228DF805308DF804108DF8D7
:10B9300007201EF0DFFC504603B0BDE8F08FBBF1DE
:10B94000000FE6D001370C238BF807708BF8063018
:10B950005846727F222101F071F9DAE7C8B29CE7FC
:10B960000137FFB214B10B23E771A37119F0100F67
:10B9700020460CBF12210221727F01F05FF9C8E757
:10B9800028F0F6FEB2E7AA46D5E7B246D3E700BFF5
:10B99000B8410020A0A903081C060020D98900088E
:10B9A000003802400348D0F8AC3113B100F5D27032
:10B9B000184770471C0600200348D0F8903113B197
:10B9C00000F5C470184770471C0600200348D0F8E3
:10B9D000743113B100F5B670184770471C0600208B
:10B9E0000348D0F8583113B100F5A87018477047D4
:10B9F0001C0600200348D0F83C3113B100F59A70C2
:10BA0000184770471C0600200348D0F8203113B1B6
:10BA100000F58C70184770471C0600200348D0F8CA
:10BA200004310BB1FC301847704700BF1C060020E2
:10BA30000348D0F8E8300BB1E0301847704700BF3A
:10BA40001C0600200348D0F8CC300BB1C430184796
:10BA5000704700BF1C0600200348D0F8B0300BB17F
:10BA6000A8301847704700BF1C0600200348D0F8D4
:10BA700094300BB18C301847704700BF1C06002073
:10BA80000248836F0BB17030184770471C060020C6
:10BA90000248C36D0BB15430184770471C06002094
:10BAA0000248036C0BB13830184770471C06002061
:10BAB0000248436A0BB11C30184770471C0600202F
:10BAC0000248836803B11847704700BF1C06002076
:10BAD0001549164B16480A6910B48C691549B2FB12
:10BAE000F4F203FB02F30360D1F88820124B134CED
:10BAF00042F47002C1F888201A68002042F0010266
:10BB00001A6098601A6822F0847222F480321A60F7
:10BB10005C601A684FF0006422F480221A60D860DA
:10BB20008C605DF8044B70470000002040420F001D
:10BB3000D491002000ED00E00038024010300024D5
:10BB4000044B4FF4F07002210A22186199615A6186
:10BB5000FFF7BEBF00000020436A8269D154436AE8
:10BB60000169426B01338B4228BF00234362002AE4
:10BB70002FD0EFF31182502383F31288436B19689F
:10BB8000C9072CD470B45E686EB9456A816A8D426B
:10BB900017D084690C44DC600ED9691A596085623B
:10BBA000002180F85810196841F00101D2B21960E3
:10BBB00082F3118870BC70470469611A596086620B
:10BBC000EEE7012380F85830D2B282F3118870BCBE
:10BBD0007047426DD36843F08003D3607047D2B2A0
:10BBE00082F31188704700BF026B10B462B1836C9E
:10BBF000C2684469D11A013B615C5DF8044B08BF1F
:10BC000013468364C8B27047016A4369C4685B5CC9
:10BC10000131A14228BF114601625DF8044BD8B240
:10BC2000704700BF436B13B190F858007047836AA8
:10BC3000406A181AB0FA80F040097047416A836A76
:10BC400099420AD3CB1A416B026961B14968501E0F
:10BC50000B4483420AD2C01A704702691144CB1ABE
:10BC6000416B0029F2D1501EC01A70470020704766
:10BC7000036B43B1826C5B6893422FBF981AC06814
:10BC80009B1AC0187047C269036A9A422FBFD01A24
:10BC9000C0688018C01A70470A4B30B503F114040D
:10BCA00093F900205D78072AC8BF143A811804333D
:10BCB0008D7213F8025C855413F8012C0A75A342A7
:10BCC000EED130BDC8A9030803682DE9F041DF6952
:10BCD0001FB13B46BDE8F0411847002A164611DD6A
:10BCE00004460D460E4400E023689B6820469847B2
:10BCF0000028F9D0236815F8011B1B6820469847D7
:10BD0000AE42F1D1BDE8F08100233C214222017016
:10BD100042708370C370704710B5084B03F10C017B
:10BD200093F900205C78845402449C78D470DC78C9
:10BD3000947104338B42F3D110BD00BFDCA903081A
:10BD400030B4846814B12368A5885D83436840F2E9
:10BD5000E93001E0002833D01D89013815F0020FC9
:10BD600080B2F7D089B2998140F2E93101E000292F
:10BD700050D01889013910F0010F89B2F7D0998994
:10BD800040F2E93101E000292FD01889013910F083
:10BD9000020F89B2F7D092B29A8140F2E93201E003
:10BDA000002A4BD01989013A11F0010F92B2F7D055
:10BDB0009B8914B12368A2881A83012030BC704784
:10BDC0002C498B4208D0A1F578418B424CD001F52B
:10BDD00080618B42D4D10220274901EB00104189B8
:10BDE000013189B241814189CAE7224A934208D090
:10BDF000A2F57842934235D002F580629342D8D1C1
:10BE000002211D4B03EB01114B8901339BB24B8186
:10BE10004B89CEE71748834207D018498B4227D079
:10BE200001F580618B42ABD10221134800EB011177
:10BE30004889013080B248814989A1E70D498B4288
:10BE400007D00E4A934211D002F580629342B0D1DE
:10BE50000222094B03EB0212538901339BB2538137
:10BE60005389A6E70121CCE70120B5E70122F0E7DD
:10BE70000121DAE700300140D4970020003800406B
:10BE800030B50446406D61718389A26823F4005384
:10BE90001B041B0C838185B0A379009213F004026C
:10BEA0002ED04FF4805213F00203ADF804203CD1A1
:10BEB000ADF806304FF480630022ADF8083011F081
:10BEC0000103ADF80C2026D1ADF80A3008238A070B
:10BED000694648BFADF80A301EF044FAA379626D96
:10BEE00013F0080F938A1BD123F008031B041B0CCB
:10BEF000938293899BB243F40053938105B030BD84
:10BF000013F00203ADF8042012D04FF4005513468D
:10BF1000ADF80650D0E70423ADF80A300C23D6E77D
:10BF20009BB243F008039382E3E74FF40053BFE76B
:10BF3000ADF80630C0E700BF10B50446406DA16003
:10BF4000838923F400531B041B0C8381A37984B0E1
:10BF500013F00402009133D04FF4805213F0020327
:10BF6000ADF804203CD1ADF806304FF4806362791F
:10BF7000ADF80830D1074FF00003ADF80A30ADF846
:10BF80000C3045BF0423ADF80A3008230C23694662
:10BF9000920748BFADF80A301EF0E4F9A379626D4C
:10BFA00013F0080F938A16D123F008031B041B0C0F
:10BFB000938293899BB243F40053938104B010BDE4
:10BFC00013F00203ADF804200DD04FF400511346D6
:10BFD000ADF80610CBE79BB243F008039382E8E785
:10BFE0004FF40053BFE7ADF80630C0E72DE9F04F3E
:10BFF000013085B0C3B203930B4602918B4C8C4E3B
:10C00000002B00F099808B4D8B4FDFF8309223F09E
:10C01000E7FE4FF4FA7A4FF0100C4FF47A70D9F82B
:10C020000430C3F30803002B40F0DE80EFF31183EC
:10C03000002B40F0D9802968A26800BF2B68994284
:10C04000F9D1D7F800E000FB0EF39B1AB3FBFEF327
:10C0500000FB01314FF0010E0191D9F80430C3F318
:10C060000803002B40F08780EFF31183002B40F092
:10C0700082802B68A16800BF2A689342F9D1D7F863
:10C0800000B000FB0BF2521AB2FBFBF200FB0323E1
:10C09000019A9B1AB3F57A7FDFD3BAF1010ABED1B8
:10C0A000039B002B40F0BD804FF47A7ADFF88C912F
:10C0B00050464FF0100CD9F80430C3F30803002B9E
:10C0C00075D1EFF31183002B71D12968A26800BFED
:10C0D0002B689942F9D1D7F800E000FB0EF39B1AC8
:10C0E000B3FBFEF300FB01314FF0010E0191D9F8D3
:10C0F0000430C3F3080313BBEFF31183FBB92B68C0
:10C10000A16800BF2A689342F9D1D7F800B000FBBC
:10C110000BF2521AB2FBFBF200FB0323019A9B1AAB
:10C12000B3F57A7FE3D3BAF1010AC4D1029B013B94
:10C130000293002B7FF467AF05B0BDE8F08FEFF3FB
:10C1400011888CF31288A1682368DB0344BFC6F80A
:10C1500000E0A1682B6832685FFA88F888F31188DC
:10C16000D7F800801A4400FB08F35B1AB3FBF8F31E
:10C1700000FB0233D2E7EFF311888CF31288A16839
:10C180002368DB0344BFC6F800E0A1682B6832686F
:10C190005FFA88F888F31188D7F800801A4400FB0A
:10C1A00008F35B1AB3FBF8F300FB023370E7EFF31D
:10C1B00011828CF31288D4F808E02368D90303D5E0
:10C1C00001233360D4F808E02B683168D2B282F3DF
:10C1D00011883A68194400FB02F3A3EB0E03B3FB8A
:10C1E000F2F300FB01317FE7EFF311828CF3128849
:10C1F000D4F808E02368D90303D501233360D4F8C9
:10C2000008E02B683168D2B282F311883A68194489
:10C2100000FB02F3A3EB0E03B3FBF2F300FB0131CF
:10C2200018E7184625F0E2FC3EE700BF10E000E00A
:10C23000BCA10020C0A10020C4A1002000ED00E0AE
:10C24000204B5B68C3F3080330B4BBB9EFF3118331
:10C25000A3B91D4B1D4C1868A16800BF1A68904215
:10C26000F9D11B4B1C684FF47A7202FB04F3591A84
:10C27000B1FBF4F130BC02FB00107047EFF3118208
:10C28000102383F3128811498C680B6813F4803FE4
:10C29000104B02D0012018608C680B49D2B20D6897
:10C2A000186882F311880A4B19684FF47A7228448F
:10C2B00002FB01F31B1B30BCB3FBF1F302FB0030AC
:10C2C000704700BF00ED00E0C0A1002010E000E0DA
:10C2D000C4A10020BCA100202DE9F84F8046FFF743
:10C2E000AFFF254E2549DFF8A0E0254A254D8446BD
:10C2F00010274FF47A740120DEF80430C3F30803EA
:10C30000D3B9EFF31183BBB90B68D2F808A000BF13
:10C31000D1F800904B45F7D1D6F800B004FB0BF9EB
:10C32000A9EB0A09B9FBFBF904FB0393A3EB0C038C
:10C330004345E1D3BDE8F88FEFF3118A87F3128804
:10C34000D2F808B01368DB0344BF2860D2F808B005
:10C350000B68D5F800905FFA8AFA8AF31188D6F84C
:10C3600000A0994404FB0AF3A3EB0B03B3FBFAF31D
:10C3700004FB0933DAE700BFC4A10020C0A10020FC
:10C3800010E000E0BCA1002000ED00E02DE9F04F3E
:10C39000DFF830C1474A4849484E494D804610278A
:10C3A00018F1FF38C0F08480DCF80430C3F30803D0
:10C3B000002B5CD1EFF31183002B58D10B689468EC
:10C3C00000BF08688342F9D1D6F800904FF47A7024
:10C3D00000FB09FEAEEB040EBEFBF9FE00FB03EE14
:10C3E000DCF80430C3F308034FF47A740120FBB97E
:10C3F000EFF31183E3B90B68D2F808A000BFD1F8BE
:10C4000000904B45F7D1D6F800B004FB0BF9A9EB2F
:10C410000A09B9FBFBF904FB0393A3EB0E03B3F585
:10C420007A7FBDD2DCF80430C3F30803002BDFD0E1
:10C43000EFF3118A87F31288D2F808B01368DB0390
:10C4400044BF2860D2F808B00B68D5F800905FFAB6
:10C450008AFA8AF31188D6F800A0994404FB0AF3FB
:10C46000A3EB0B03B3FBFAF304FB0933D5E7EFF3BC
:10C47000118487F31288D2F808901368D80303D583
:10C4800001232B60D2F808900B682868E4B284F38B
:10C490001188D6F800A04FF47A7400EB030E04FB69
:10C4A0000AF3A3EB0903B3FBFAF304FB0E3E97E791
:10C4B000BDE8F08F10E000E0C0A10020C4A1002082
:10C4C000BCA1002000ED00E030B4EFF31183102296
:10C4D00082F312880649074C0A6807480132002592
:10C4E0000A602560DBB2026883F3118830BC7047B4
:10C4F000C0A10020BCA1002010E000E038B5254B11
:10C500001C69236B73B1636D626BCAB1998A1A8817
:10C51000C90592B201D5D20700D438BD4FF6F772E3
:10C520001A8038BD636D99891A88890692B2EBD555
:10C530009206E9D5E26ACAB1988880B29047E2E7EC
:10C5400099891A880D0692B2E0D51006DED5A26A46
:10C55000616A8A4219D0A1692569885C9880013294
:10C56000B2FBF5F105FB1122A262CFE79B88E269DD
:10C570006169DBB28B54E269E068636D0132B2FB42
:10C58000F0F100FB1122E261BEE7DA6822F08002DE
:10C59000DA60BBE7B841002038B5254BDC68236B77
:10C5A00073B1636D626BCAB1998A1A88C90592B278
:10C5B00001D5D20700D438BD4FF6F7721A8038BDC6
:10C5C000636D99891A88890692B2EBD59206E9D5EE
:10C5D000E26ACAB1988880B29047E2E799891A88DE
:10C5E0000D0692B2E0D51006DED5A26A616A8A42D3
:10C5F00019D0A1692569885C98800132B2FBF5F1F8
:10C6000005FB1122A262CFE79B88E2696169DBB278
:10C610008B54E269E068636D0132B2FBF0F100FB1C
:10C620001122E261BEE7DA6822F08002DA60BBE73D
:10C63000B841002038B5254B9C68236B73B1636DFE
:10C64000626BCAB1998A1A88C90592B201D5D2071C
:10C6500000D438BD4FF6F7721A8038BD636D9989E2
:10C660001A88890692B2EBD59206E9D5E26ACAB178
:10C67000988880B29047E2E799891A880D0692B2AD
:10C68000E0D51006DED5A26A616A8A4219D0A16996
:10C690002569885C98800132B2FBF5F105FB112217
:10C6A000A262CFE79B88E2696169DBB28B54E269E1
:10C6B000E068636D0132B2FBF0F100FB1122E26130
:10C6C000BEE7DA6822F08002DA60BBE7B8410020FA
:10C6D00038B5254B5C68236B73B1636D626BCAB16F
:10C6E000998A1A88C90592B201D5D20700D438BDFB
:10C6F0004FF6F7721A8038BD636D99891A888906DA
:10C7000092B2EBD59206E9D5E26ACAB1988880B2B6
:10C710009047E2E799891A880D0692B2E0D5100693
:10C72000DED5A26A616A8A4219D0A1692569885C4E
:10C7300098800132B2FBF5F105FB1122A262CFE72E
:10C740009B88E2696169DBB28B54E269E068636DE2
:10C750000132B2FBF0F100FB1122E261BEE7DA68C0
:10C7600022F08002DA60BBE7B841002038B5254BE3
:10C770001C68236B73B1636D626BCAB1998A1A88A6
:10C78000C90592B201D5D20700D438BD4FF6F77271
:10C790001A8038BD636D99891A88890692B2EBD5E3
:10C7A0009206E9D5E26ACAB1988880B29047E2E77A
:10C7B00099891A880D0692B2E0D51006DED5A26AD4
:10C7C000616A8A4219D0A1692569885C9880013222
:10C7D000B2FBF5F105FB1122A262CFE79B88E2696B
:10C7E0006169DBB28B54E269E068636D0132B2FBD0
:10C7F000F0F100FB1122E261BEE7DA6822F080026C
:10C80000DA60BBE7B841002070B4EFF31186502323
:10C8100083F31288436B1A68D20720D45D686DB920
:10C82000446A826A944217D081691144D9600ED952
:10C83000A21A5A608462002280F858201A6842F0D6
:10C840000102F1B21A6081F3118870BC704701696E
:10C850008A1A5A608562EEE7012380F85830F3B2F5
:10C8600083F3118870BC704703682DE9F041DF69DC
:10C870001FB13B46BDE8F0411847002A164611DDBE
:10C8800004460D460E4400E023689B682046984706
:10C890000028F9D0236815F8011B1B68204698472B
:10C8A000AE42F1D1BDE8F08103689B69184700BF33
:10C8B00003685B69184700BF03681B69184700BF1E
:10C8C0000368DB68184700BF03685B68184700BF50
:10C8D00003681B68184700BF38B50C46097849B192
:10C8E000054601342B6828461B68984714F8011B3D
:10C8F0000029F7D138BD00BF064B53F820302BB1CB
:10C900001A689B8851690B4201D113837047538386
:10C91000704700BFC895002003682DE9F04F03F170
:10C920003F4404F57E04604EA40A0125345D04F002
:10C930001F066409032C05FA06F500F0AF80042CED
:10C9400000F0A780022C54D08588B5FA85F0C0F19C
:10C950001F0080B2C40803EB840400F00700266ABD
:10C9600080000F27874026EA07062662276A01F023
:10C97000030602FA00F0721E3843012AC1F3810C4B
:10C98000C1F300182062C1F3411137D900242246B7
:10C9900001274FF0030E03E0102A04F1020426D011
:10C9A00007FA02F0A84302F10102F5D1D3F800C062
:10C9B0000EFA04F0C04300EA0C0CC3F800C0D3F830
:10C9C000008006FA04FC4CEA080CC3F800C0D3F857
:10C9D0000CC000EA0C00D860D3F80CC001FA04F0D7
:10C9E00040EA0C00102AD86004F10204D8D1BDE856
:10C9F000F08F2E4C666C35436564A5E70020024637
:10CA00004FF0010E4FF0030904E00132102A00F14B
:10CA100002003CD00EFA02F737EA0504F5D1D3F84C
:10CA200000A009FA00F4E4430AEA040AC3F800A0EB
:10CA3000D3F800B006FA00FA4AEA0B0AC3F800A0DD
:10CA4000D3F808A004EA0A0AC3F808A0D3F808B08B
:10CA50000CFA00FA4AEA0B0AC3F808A0D3F804A0BB
:10CA60002AEA07075F60D3F804A008FA02F747EA4A
:10CA70000A075F60DF683C40DC60DF6801FA00F4B1
:10CA800001323C43102ADC6000F10200C2D1BDE853
:10CA9000F08F064C266B3543256355E7034C266C17
:10CAA0003543256450E700BFFCD30308003802403B
:10CAB00010B50409013C032C17D80D4B33F8142092
:10CAC00000F00F0042FA00F313F001030DD0012330
:10CAD00003FA00F0013810402BF07EF9054A064BAE
:10CAE000125D104403EBC00010BD002010BD00BF5C
:10CAF0004CD7030848D70308EC9F00202DE9F04FDE
:10CB00004A484B494B4B4C4C4FF0010A4FF002093D
:10CB10004FF004084FF0080C4FF0100E202740266D
:10CB2000802530F8022B12F0010F03D01960A3F812
:10CB300004A0083312F0020F03D01960A3F8049088
:10CB4000083312F0040F03D01960A3F804800833EF
:10CB500012F0080F03D01960A3F804C0083312F0D4
:10CB6000100F03D01960A3F804E0083312F0200F6F
:10CB700002D019609F80083312F0400F02D0196074
:10CB80009E80083312F0800F02D019609D80083318
:10CB900012F4807F05D04FF4807B1960A3F804B0B5
:10CBA000083312F4007F05D04FF4007B1960A3F81E
:10CBB00004B0083312F4806F05D04FF4806B196015
:10CBC000A3F804B0083312F4006F05D04FF4006BE3
:10CBD0001960A3F804B0083312F4805F05D04FF455
:10CBE000805B1960A3F804B0083312F4005F05D02D
:10CBF0004FF4005B1960A3F804B0083312F4804FBF
:10CC000005D04FF4804B1960A3F804B00833D20B61
:10CC100004D04FF4004219609A80083301F5806116
:10CC2000A1427FF47EAFBDE8F08F00BF4CD7030870
:10CC300000000240EC9F00200010024000286AD053
:10CC400003682DE9F04F03F13F4404F57E045F4E85
:10CC5000A40A0125345D04F01F066409032C05FABB
:10CC600006F559D0042C00F0AC80022C59D08588F0
:10CC7000B5FA85F0C0F11F0080B2C40803EB84044C
:10CC800000F00700266A80000F27874026EA070683
:10CC90002662276A01F003068240701E3A4301288B
:10CCA000C1F3810CC1F300182262C1F341113DD9D7
:10CCB0000024224601274FF0030E03E0102A04F15E
:10CCC000020426D007FA02F0A84302F10102F5D1CE
:10CCD000D3F800C00EFA04F0C04300EA0C0CC3F80D
:10CCE00000C0D3F8008006FA04FC4CEA080CC3F834
:10CCF00000C0D3F80CC000EA0C00D860D3F80CC018
:10CD000001FA04F040EA0C00102AD86004F1020491
:10CD1000D8D1BDE8F08F70472D4C266C3543256483
:10CD2000A5E72B4C666C35436564A0E700200246FE
:10CD30004FF0010E4FF0030904E00132102A00F118
:10CD400002003CD00EFA02F737EA0504F5D1D3F819
:10CD500000A009FA00F4E4430AEA040AC3F800A0B8
:10CD6000D3F800B006FA00FA4AEA0B0AC3F800A0AA
:10CD7000D3F808A004EA0A0AC3F808A0D3F808B058
:10CD80000CFA00FA4AEA0B0AC3F808A0D3F804A088
:10CD90002AEA07075F60D3F804A008FA02F747EA17
:10CDA0000A075F60DF683C40DC60DF6801FA00F47E
:10CDB00001323C43102ADC6000F10200C2D1BDE820
:10CDC000F08F034C266B3543256350E7FCD30308F3
:10CDD00000380240002855D0026802F13F4303F5B5
:10CDE0007E032DE9F04F9B0A544DEB5C03F01F05C9
:10CDF0005B090124032B04FA05F444D0042B00F052
:10CE00009780022B44D001F00306731E012BC1F35F
:10CE1000810CC1F300188588C1F341113DD900246C
:10CE2000234601274FF0030E03E0102B04F1020408
:10CE300026D007FA03F0A84303F10103F5D1D2F895
:10CE400000C00EFA04F0C04300EA0C0CC2F800C0A7
:10CE5000D2F8008006FA04FC4CEA080CC2F800C0C4
:10CE6000D2F80CC000EA0C00D060D2F80CC001FA75
:10CE700004F040EA0C00102BD06004F10204D8D179
:10CE8000BDE8F08F70472E4B1D6C2C431C64BAE735
:10CE90002B4B5D6C2C435C64B5E7002003464FF0E0
:10CEA000010E4FF0030904E00133102B00F10200E2
:10CEB0003CD00EFA03F737EA0504F5D1D2F800A00A
:10CEC00009FA00F4E4430AEA040AC2F800A0D2F81E
:10CED00000B006FA00FA4AEA0B0AC2F800A0D2F83B
:10CEE00008A004EA0A0AC2F808A0D2F808B00CFAAE
:10CEF00000FA4AEA0B0AC2F808A0D2F804A02AEA0B
:10CF000007075760D2F804A008FA03F747EA0A07B0
:10CF10005760D7683C40D460D76801FA00F4013309
:10CF20003C43102BD46000F10200C2D1BDE8F08F69
:10CF3000034B1D6B2C431C6365E700BFFCD3030848
:10CF40000038024010B1036882885A83704700BFDE
:10CF500010B1036882881A83704700BF18B1036854
:10CF6000828809B95A8370471A8370470E4B1B8811
:10CF700001463BB90D4B0E4A1B7810680BB981F086
:10CF80000101EBE70B4B5A691AB118B91A68106026
:10CF900058747047084A18681188084A92FBF1F2E1
:10CFA0000121026059747047D4950020D695002065
:10CFB000D8950020DC950020F495002020A10700E2
:10CFC00010B40A4B0A4A1C7801238340234052F8CC
:10CFD000200029B9B3FA83F149095DF8044BBDE794
:10CFE000191C18BF01215DF8044BB7E7C595002057
:10CFF000C89500202DE9F0410B4E346873691C4040
:10D000000FD0DFF828800127B4FA84F3C3F11F039F
:10D0100007FA03F558F8230003689847AC43756195
:10D02000F2D1BDE8F08100BF003C014074A10020B6
:10D030002DE9F0410B4E346873691C400FD0DFF8C6
:10D0400028800127B4FA84F3C3F11F0307FA03F51C
:10D0500058F8230003689847AC437561F2D1BDE8E6
:10D06000F08100BF003C014074A100202DE9F04197
:10D070000B4E346873691C400FD0DFF828800127FD
:10D08000B4FA84F3C3F11F0307FA03F558F8230039
:10D0900003689847AC437561F2D1BDE8F08100BFE9
:10D0A000003C014074A100202DE9F0410B4E346892
:10D0B00073691C400FD0DFF828800127B4FA84F38D
:10D0C000C3F11F0307FA03F558F8230003689847D4
:10D0D000AC437561F2D1BDE8F08100BF003C014076
:10D0E00074A100202DE9F0410B4E346873691C4097
:10D0F0000FD0DFF828800127B4FA84F3C3F11F03AF
:10D1000007FA03F558F8230003689847AC437561A4
:10D11000F2D1BDE8F08100BF003C014074A10020C5
:10D120002DE9F0410B4E346873691C400FD0DFF8D5
:10D1300028800127B4FA84F3C3F11F0307FA03F52B
:10D1400058F8230003689847AC437561F2D1BDE8F5
:10D15000F08100BF003C014074A100202DE9F041A6
:10D160000B4E346873691C400FD0DFF8288001270C
:10D17000B4FA84F3C3F11F0307FA03F558F8230048
:10D1800003689847AC437561F2D1BDE8F08100BFF8
:10D19000003C014074A10020084A094808B5536CBE
:10D1A00043F480435364002140222DF036FB054BAD
:10D1B0004FF0FF321A60C3F8032008BD0038024068
:10D1C00074A10020B4A100202DE9F04104461846C6
:10D1D0000D46164698462AF035F92768E672284427
:10D1E000A07229467D69434632462046AC46BDE8DA
:10D1F000F0416047036810B504461B6898472368F0
:10D2000020469B689847A37B0133A37310BD00BFE2
:10D2100010B5036804469B689847FF230122637397
:10D22000227310BD144B984224D003F580639842BA
:10D2300020D0028822F040021204120C02800288E0
:10D2400022F038031B041B0C59B141F480710029F2
:10D2500091FAA1F2B2FA82F108BF4FF0FF31013921
:10D26000C9000B439BB2038003889BB243F0400389
:10D27000038070474908DCE700380040F0B4848937
:10D280004FF6FF764FF47A7463B300293CD00F78E1
:10D29000013101E0B4421AD00589013C15F00205C4
:10D2A000A4B2F7D0BCB284814FF47A7402E0BCB26D
:10D2B000B4420CD0058915F0010504F1FF37F6D012
:10D2C0008589ADB20AB115700132013BDCE7104B24
:10D2D00098420BD0A3F57843984217D003F58063AA
:10D2E000984202D00120F0BC70470225094B03EBA5
:10D2F00005156B8901339BB26B81688980B2003060
:10D3000018BF0120F0BC7047FF27C5E70125EDE7F6
:10D3100000300140D497002070B50546806810B1F8
:10D3200004688088608341F08001686840F2E934D5
:10D3300000E0E4B10689013C16F0020FA4B2F8D077
:10D3400089B2818140F2E93100E029B304890139D1
:10D3500014F0010F89B2F8D081890021FFF78EFF08
:10D36000AB6813B11A689B881383012070BD1649FE
:10D37000884208D0A1F57841884221D001F580612A
:10D380008842EAD10224114901EB04146189013178
:10D3900089B261816189E0E70B4CA04207D00C495A
:10D3A00088420FD001F580618842D6D10221074C16
:10D3B00004EB01114C890134A4B24C814989CCE7BA
:10D3C0000124E0E70121F2E700300140D49700207A
:10D3D00000380040F8B5624C0601A7190546387AB6
:10D3E00027F0C6F93B7A03F01F015B090122032BEA
:10D3F00002FA01F26DD0042B66D0022B5CD0A31987
:10D4000001351879FFF754FBEDB2074610B112232E
:10D41000C5718371A3195879FFF74AFB10B1132323
:10D42000C5718371A3199879FFF742FB10B11423DA
:10D43000C5718371A5190A21EA793846FFF7FEFB09
:10D440006879FFF735FBEA790A21FFF7F7FBA8793E
:10D45000FFF72EFBEA790A21FFF7F0FBA359414AB7
:10D46000934246D0404A93424ED0404A934256D0CF
:10D470003F4A93425ED03F4A934266D03E4A93422F
:10D480002CD03444227BE2B901220220198801F415
:10D49000415141F445710A4302431A809A8B22F4A8
:10D4A00000621204120C07219A8319821A8892B220
:10D4B00042F040021A80F8BD304B596A0A435A6262
:10D4C0009DE700221046E1E72C4B19690A431A61D7
:10D4D00095E72A4B196A0A431A6290E702F56442FB
:10D4E000516A41F400115162516A21F400115162F4
:10D4F000C7E702F58432516A41F480515162516AA2
:10D5000021F480515162BCE702F50032116A41F406
:10D5100080411162116A21F480411162B1E702F584
:10D52000FE32116A41F400411162116A21F4004196
:10D530001162A6E702F58232516A41F4005151624C
:10D54000516A21F4005151629BE702F56842516A29
:10D5500041F480115162516A21F48011516290E7C7
:10D56000D49700200030014000380040003C0040CB
:10D570000034014000500140005401400038024096
:10D58000427A02B9704710B504460368406804F156
:10D590000A0198470023637210BD00BF437A5A1CEA
:10D5A0000344D2B242729972037A934200D802B90C
:10D5B000704710B504460368406804F10A019847B3
:10D5C0000023637210BDF8B50468C4F30D0405466A
:10D5D0000E4604B32F681CF079FE092840F08980BC
:10D5E000454C236923F440732361236943F400739A
:10D5F0002361236943F0010323613E601CF066FE52
:10D600002369092823F00103236172D12B680433B5
:10D610002B600020F8BD394B394A93422CD902F5D2
:10D620008042934227D902F5804293422BD902F5DA
:10D630008042934229D902F58032934227D902F5DC
:10D640000032934225D902F50032934223D902F5E4
:10D650000032934221D902F5003293421FD902F5DC
:10D66000802293421DD9B3F1016F1CD3052022F013
:10D670004BFDFDF7C5FF08241CF028FE092814D037
:10D680004FF0FF30F8BD1024F6E71824F4E720240B
:10D69000F2E72824F0E73024EEE73824ECE74024D2
:10D6A000EAE74824E8E75824E6E7134F3B6923F408
:10D6B00040733B613B6943F400733B613B6923F07A
:10D6C000F8033B613B6943F002031C433C613B6947
:10D6D00043F480333B611CF0F9FD3B6923F0020306
:10D6E0003B613B69092823F0F8033B613FF472AFCB
:10D6F000C6E76FF00100F8BD003C024000400008A2
:10D70000FF3F0008F8B504460D468E180027B542C5
:10D7100001D12069F8BDE368591CE160234415F884
:10D72000012B1A720429F2D1206918B9A168204688
:10D73000FFF749FF2061E760E9E770B544880646D6
:10D740000D46C4F30B042246002128462DF065F84F
:10D7500033690A4A934209D3094A934206D22246C0
:10D7600028461946BDE870402AF040BD23B1214645
:10D770002846BDE87040184770BD00BFD4050008BA
:10D78000D4060008064B07498B4202D300231846F3
:10D7900070471A88C2F30B029042F8D01433F3E7B3
:10D7A00088010008D4050008024A136823EA000033
:10D7B0001060704724AA00202DE9F04F2DED028B58
:10D7C00093B083461AF0E6F8914B1D7825B113B05B
:10D7D000BDEC028BBDE8F08F8E4B1B685905F6D56A
:10D7E0008D4B8E4E1B6863B18D4A31681368CB1A1E
:10D7F0007C2B06D98B48116003780133037019F034
:10D8000085FD894B1B78002B72D0884C884AD4F850
:10D810001031ABEB0303934201F2548394F8189157
:10D82000B9F1000F35D1DFF83C82D8F80000FFF7DE
:10D830004BF8C0B201280FD902287E4F42F0668013
:10D840003B78002B42F0B181D4F81C31ABEB0303E1
:10D85000B3F57A6F82F0EF82D4F82031002B47D0F5
:10D8600094F81831C3B9744B1B689B7801211E3B97
:10D8700000228B4284F8181184F82C2142F29682FF
:10D88000D8F800000221043019F0F8FC94F8243193
:10D8900011E0D4F820315BB3D4F8283140F6B73228
:10D8A000ABEB0303934223D994F82431002B01F00E
:10D8B000F986DFF8B081013BDBB284F82431002B1C
:10D8C00001F02684D4F8207194F82C2117F8011B5C
:10D8D00094F82D31D8F80000C4F820710A440133BF
:10D8E00084F82C2184F82D31FEF7F2FFC4F828B11A
:10D8F000524B37681B7853B1DFF86C81D8F80000C1
:10D9000028B14F4B1B78013B012B41F211844D4B49
:10D910001B7873B1DFF85481D8F800304BB133680D
:10D92000424C02931A46D4F84431D31A632B01F2C5
:10D93000B281DFF83C8198F80030022B01F08A8632
:10D940003C4F97F87430032B01F0CC833E4B1B788F
:10D9500073B13E4D2B685BB1344CFEF771FCD4F8CB
:10D960005031029044F61F62C31A934200F2308194
:10D97000374B1B78002B7DD1364B1B7843B12B4C9A
:10D98000D4F8A03203F5C333A0339B4581F03E8227
:10D99000314B1B78002B3FF41AAF244E2F4C304DE7
:10D9A00006F2C1272068FEF78FFF00283FF40FAF73
:10D9B0002068FEF785FF2B7880465A1E33B1206819
:10D9C0002A70FEF781FF0028F2D100E703223946D2
:10D9D000781E2CF008FF96F8C03296F8C12286F81F
:10D9E000C38283F47F4383F0FF039B1A1FFA88F8F6
:10D9F0009BB2B8EB132FD5D196F8C222DBB29A4274
:10DA0000D0D1781E1BF0BAF92B7818442870C9E7DA
:10DA10002C5E0020A88E0020B0540020C0A1002061
:10DA2000205500201C550020F25500200C25002018
:10DA30003F0D03002C000020D0540020F45500209E
:10DA4000FC550020045600200C56002010560020E3
:10DA50007C5600208D560020165600201C560020B3
:10DA600020560020CC540020C4540020945B002099
:10DA7000DE430020484C2278A2B1484B9B7A53B138
:10DA8000FEF7DEFB464B1B68C31AA3F57A73B3F5AA
:10DA9000FA6F07D82278434B43491868FEF7E4FE33
:10DAA00000232370414CD4F8983203F5C333A033DC
:10DAB0009B45FFF461AF3E4DC4F898B22B78002B24
:10DAC00041F035873B4D2B78002B41F08D8694F843
:10DAD0009C2239498D5CEA0701F1E787AF0701F124
:10DAE000A787680702F12B802A0748D5334B344FAC
:10DAF0000B9312AA1146A3F13D0241F8202D0020FC
:10DB0000A3F140020D4603F8400C039102231121BA
:10DB10005170937028463968FBF76AF9284679688E
:10DB2000FBF766F9FB89274903EBC3039B00053329
:10DB300081FB0321DB17C3EBA101284689B2FBF768
:10DB40006FF93B8A03EB8303590089B22846FBF740
:10DB500067F91D4B039D1B789B0743BF398901F56E
:10DB60007A7189B24FF47A712846FBF759F90A9B0A
:10DB70003A7D591C0A9128461A7019F09BFE134AE7
:10DB800094F89C321178013393FBF1F201FB1233CC
:10DB900084F89C32F0E600BFE45500201C90002081
:10DBA0008073002080560020A45500200C25002002
:10DBB000845600208556002088560020A455002059
:10DBC0004855002067666666445500208C56002044
:10DBD00094F85631002B41F08A85DB4B1A6802F02D
:10DBE0000803002B4AF60B4048F603414BF60F435F
:10DBF00049F6074704BF03460F4612F0040F4FF0E3
:10DC0000190118BF1F46900684F8561103D547F432
:10DC1000804747F02007CD4B5A79C7F30909002AFE
:10DC200042F031819B79002B42F03D82984664207E
:10DC30004FF0FF3A4FF0000C0A970B97ADF834C045
:10DC4000CDF83AC0CDF83EC0CDF842C0CDF8309006
:10DC5000ADF83680ADF838A08DF846000AAF0FCF8A
:10DC6000DFF800E384F805C0AEE80F0097E80F0086
:10DC7000AEE807002EF8023B71464FF0010C1B0C7A
:10DC8000FE271F20C82201F81E39A770A27184F850
:10DC900007C0E07094F86601207180F0F10383EA18
:10DCA0000313DAB2130983F0E70343EA022383EA9A
:10DCB000C2031BB283EA0312D2B2C3F3072383EA7F
:10DCC000121343EA022383EAC2031BB283F0C802A1
:10DCD00082EA0212D2B2C3F3072383EA121343EAA1
:10DCE000022383EAC2031BB283EA0C0787EA071701
:10DCF000FFB2C3F3072282EA171242EA072200EBBF
:10DD00000C0382EAC7070EEB0C0084F8663127800B
:10DD100011F8013B7B4083EA0313DBB21A0982EA64
:10DD2000172242EA032282EAC3031BB29FB2814256
:10DD30002780EDD183F07C0383EA0313DBB24FEA43
:10DD4000131E8EEA172E8EEA032E8EEAC30E0FFAEA
:10DD50008EFE1FFA8EF9DFF810C2A4F800905FFA69
:10DD60008EFE4FEA192984F8289084F827E00CF5F4
:10DD7000C77804F1220ADCF80000DCF80410DCF8B3
:10DD80000820DCF80C3047460FC70CF1100CD445C6
:10DD9000B846F0D1DCF8000038606D4F9CF80430D4
:10DDA00088F8043007F1270884F8B5E184F8B691C3
:10DDB00017F8011F2868FEF78BFDB845F8D194F8D5
:10DDC0005731002B41F08E846249326809780A206D
:10DDD00084F85701002901F021865F4F0129388816
:10DDE000069042F257810229B7F802E002F06580FE
:10DDF000B8880590032902F05D81F8880490042911
:10DE000002F06E810529388902F065810629B7F88C
:10DE10000A9002F05C810729B7F80C8002F0548167
:10DE2000FB89039394F866110A920B4683F0300243
:10DE300082EA0212D2B217094849079387F07A079B
:10DE400047EA02270988237187EAC202444FC1EBDF
:10DE5000012187FB013A069B4FF0000C63F30F0C86
:10DE6000059B6EF31F4C4FF0000E63F30F0E049BE7
:10DE7000CDF82CC012B28A440027C91763F31F4E95
:10DE8000C1EB6A2A039BCDF830E082EA021160F30D
:10DE90000F070020C9B268F30F00C2F3072269F32D
:10DEA0001F4782EA111263F31F404FF000090D97DC
:10DEB0008DF83DA00E908DF83C9042EA01220DF1C4
:10DEC000280C82EAC107BCE80F003FB287F0C808FF
:10DED00088EA0818DFF88CE084F805905FFA88F883
:10DEE000C7F30727AEE80F0087EA181747EA0823A9
:10DEF0009CE8030083EAC8031BB283F023024EF8B8
:10DF0000040B82EA0212D2B2C3F30723079F83EA0B
:10DF10001213704643EA022383EAC20207F1010C9E
:10DF200020F814194FF023081621FE27C82384F87F
:10DF300066C1228084F807800EF1020EA770E1709E
:10DF4000A371114612E000BF405500202C5500205F
:10DF50009B26002020730020088D0020B28C00201A
:10DF600003082080142500200E25002010F8013B16
:10DF70004B4083EA0313DBB21A0982EA112242EA18
:10DF8000032282EAC3031BB299B270452180EDD10E
:10DF900083F0F40383EA0313DBB24FEA131E8EEA25
:10DFA000112E8EEA032E8EEAC30E0FFA8EFE1FFA92
:10DFB0008EF8CA4FA4F800804FEA182C5FFA8EFE44
:10DFC00084F81EE084F81FC07968BA683868FB6876
:10DFD00007F5C778A8E80F0038697969BA6904F2CB
:10DFE0008F17A8E8070004F2AD1884F8ADC184F8D3
:10DFF000ACE117F8011F2868FEF76AFCB845F8D1B4
:10E0000094F85A31002B41F07783B54B1B681922E5
:10E01000990684F85A2140F1FC82B24BB24F1B782A
:10E020009A0741F128873B7D042B8CBF4FF00308F2
:10E030004FF00208FEF704F93B8A3A890A9003EB95
:10E0400083035B00ADF842304FF47A703B680C9369
:10E05000F98997F814E07B688DF8448000FB02F2A0
:10E060004FF0000C0AA84FF0FF398DF845E0CDF8CD
:10E070002CC0CDF83C900E920D93ADF84010804628
:10E080000390B8E80F00DFF870E2AEE80F0098E800
:10E090000F00AEE807007246182122F81C39E17122
:10E0A00094F8661184F805C081F0780383EA0313BD
:10E0B000D8B2030983F0F60343EA002383EAC003DE
:10E0C0001BB283EA0310C0B2C3F3072383EA101321
:10E0D00043EA002383EAC0031BB283F0C80080EA4E
:10E0E000001C5FFA8CFCC3F3072080EA1C1040EA96
:10E0F0000C2080EACC0000B280F0180383EA0313FE
:10E10000DBB2C0F3072080EA131040EA032080EA64
:10E11000C30301F101081E204FF0FE0C4FF0C809A7
:10E12000E0700EF1020E217184F86681238084F87C
:10E1300002C084F80690184612F8011B414081EA9B
:10E140000111C9B20B0983EA102343EA012383EAD0
:10E15000C10109B288B272452080EDD181F0180169
:10E1600081EA0111C9B20A0982EA102383EA012374
:10E1700083EAC1031BB29AB2DFF860A12280DBB24E
:10E18000120A0592049384F8272084F82630D64694
:10E190000AF5C77904F12208DEF80000DEF8041061
:10E1A000DEF80820DEF80C30CC46ACE80F000EF1AB
:10E1B000100EC645E146EFD1DEF80000CCF80000B5
:10E1C0009DF81030DFF8348184F8B4319DF81430B4
:10E1D00084F8B531C14619F8011F2868FEF778FBAD
:10E1E000424B4B45F7D1FEF72BF8414B414AB3F96F
:10E1F0000410B7F808E03B680B930A907B680C9317
:10E2000082FB01274FF47A70C9174FF0000C00FB16
:10E210000EF0C1EBA701DDF80CE0ADF83CC0ADF8A5
:10E220003EC0ADF840C0ADF842100D900E90BEE873
:10E230000F00314F84F805C00FC79EE807004FF06C
:10E24000210C87E807001C23C8224FF0FE0EE37064
:10E2500084F807C084F802E0A27194F86611217175
:10E2600081F06A0383EA0313DAB2130983F0D5035A
:10E2700043EA022383EAC2031BB283EA0312D2B247
:10E28000C3F3072383EA121343EA022383EAC20398
:10E290001BB283F0C80282EA0212D2B2C3F3072390
:10E2A00083EA121343EA022383EAC2031BB283EA1E
:10E2B0000C0282EA0210C0B2C3F3072282EA1012F3
:10E2C00042EA0022013182EAC0020C3784F866116A
:10E2D0002280A7F11C01104612E000BF0E2500208D
:10E2E000405500204455002048550020C1260020FC
:10E2F0002455002067666666142500209B260020B2
:10E3000011F8013B434083EA0313DBB21A0982EAA6
:10E31000102242EA032282EAC3031BB298B2B94236
:10E320002080EDD183F0680383EA0313DBB219097F
:10E3300081EA102282EA032282EAC3031BB29AB264
:10E34000DB4F2280DBB24FEA122C049384F8243096
:10E3500004F1220384F825C007F5C7790593FB680B
:10E3600038687968BA68CE46AEE80F00059B10376A
:10E370009F42F146F3D13B88AEF800309DF8103053
:10E38000CC4F84F8B231C14684F8B3C119F8011FEB
:10E390002868FEF79DFA4F45F8D194F866C1C64A41
:10E3A000C64F84F804C08CF0EB0383EA0313D9B2A0
:10E3B0000B0983F0C50343EA012383EAC1031BB2BF
:10E3C00083EA0310C0B2C3F3072181EA101141EAC6
:10E3D000002181EAC0010CCA09B281F0C80E8EEAA0
:10E3E0000E1E5FFA8EFE4FF000090A92C1F307215C
:10E3F000039A0B93CDF8309081EA1E1343EA0E2363
:10E4000007CA83EACE031BB283F0310E87E8070008
:10E410008EEA0E1E5FFA8EFEC3F3072383EA1E13F5
:10E4200043EA0E2383EACE0394F808E0607AA17AE7
:10E43000E27A277B84F805901BB28EEA030E8EEAFF
:10E440000E1E5FFA8EFEC3F3072383EA1E1343EA10
:10E450000E2383EACE031BB2584080EA0010C0B2FC
:10E46000C3F3072383EA101343EA002383EAC003BC
:10E470001BB2594081EA0110C0B2C3F3072181EAFF
:10E48000101141EA002181EAC00109B24A4082EA42
:10E490000212D2B2C1F3072383EA121343EA022322
:10E4A00083EAC2031BB25F4087EA0717FFB2C3F3D8
:10E4B000072383EA171343EA0723607BA17BE27BF0
:10E4C00094F810E094F8119083EAC7031BB2584007
:10E4D00080EA0010C0B2C3F3072383EA101343EAB3
:10E4E000002383EAC0031BB2594081EA0111C9B27B
:10E4F000C3F3072383EA111343EA012383EAC10329
:10E500001BB25A4082EA0212D2B2C3F3072383EA53
:10E51000121343EA022383EAC2031BB28EEA030EFC
:10E520008EEA0E1E5FFA8EFEC3F3072383EA1E13E4
:10E5300043EA0E2383EACE031BB289EA030989EA80
:10E5400009195FFA89F9C3F3072383EA191343EA28
:10E55000092383EAC903A17CE27C594F1BB25940CD
:10E5600081EA0111C9B2C3F3072383EA111343EA15
:10E57000012383EAC1031BB25A4082EA0212D2B2DB
:10E58000C3F3072383EA121343EA022383EAC20395
:10E590001BB283F0270989EA0912D2B2C3F3072913
:10E5A00089EA121949EA022989EAC2090FFA89F9A6
:10E5B0001FFA89F20CF101034FEA122E5FFA89F972
:10E5C00031204FF0FE0C0C2184F86631C8232280E4
:10E5D000E07184F802C0E170A37184F8149084F8AB
:10E5E00015E0DAF80410DAF80820DAF80C30DAF876
:10E5F0000000BAF810C00FC727F803CB84F8A3E1D6
:10E6000084F8A29118F8011F2868FEF761F94745C0
:10E61000F8D194F85EC1BCF1000F41F07880294B2D
:10E6200094F866E1B3F90010B3F90220B3F90430AD
:10E630009FED256A214F84F805C007EE103A336834
:10E640000A938EF06A0383EA031306EE901AD9B296
:10E650000B0983F0D50343EA012383EAC1031BB20C
:10E6600083EA03115242C9B207EE902AC3F307238B
:10E6700083EA111343EA0123F8EEE77AF8EEE66A3B
:10E68000B8EEC77A83EAC1031BB267EE867A66EEFC
:10E69000866A27EE067A002083F0C808CDED0C7A52
:10E6A000CDED0B6A8DED0D7A0E900F900EE000BF50
:10E6B0000E250020BF2600209C8D00201425002060
:10E6C0009C2600202455002088C3E43A109088EA54
:10E6D00008160DF12809F6B2C3F30728B9E80F00B0
:10E6E00088EA161848EA062888EAC6080FFA88F861
:10E6F0000FC788F01E0699E8070086EA0616F6B2EC
:10E70000C8F3072383EA161343EA062387E80700C2
:10E7100083EAC606C8214FF005084FF01E0CFE2301
:10E720001C200EF10102A17184F85E8184F807C0FB
:10E73000A370E070A7F1100184F804E00C37268084
:10E7400084F8662111F8013B734083EA0313DBB2BE
:10E750001A0982EA162242EA032282EAC3031BB2A2
:10E760009EB2B9422680EDD183F0270383EA0313DA
:10E77000DBB24FEA131E8EEA162E8EEA032E8EEAC5
:10E78000C30E0FFA8EFE1FFA8EFCD94FA4F800C0FC
:10E790005FFA8EFE4FEA1C2C84F825C084F824E032
:10E7A00007F5C77804F1220938687968BA68FB6808
:10E7B00046460FC610374F45B046F5D1CD4E3B8883
:10E7C000A8F8003006F1240784F8B2E184F8B3C158
:10E7D00016F8011F2868FEF77BF8B742F8D194F8C5
:10E7E0005F81B8F1000F40F08C87C34B1B68052296
:10E7F0009B0684F85F2141F10B81C04BDFEDC06ABD
:10E80000DA891B8907EE902A07EE103AF8EEE77ACC
:10E81000B8EE477A67EEA67A94F866C1B94BBA4A61
:10E82000B3F90410B2F90620B84EB948CDED0B7A11
:10E830008CF0220383EA0313DFB23B0983F0590310
:10E8400043EA072383EAC703B2F5FA6F1BB2A8BFF6
:10E850004FF4FA6283EA0317FFB2B2F57A7FC3F38B
:10E86000072383EA1713B8BF4FF47A724FF0640E90
:10E8700043EA0723A2F57A720EFB02F283EAC70786
:10E8800086FB02E680FB01E03FB2C917D217C2EB5C
:10E89000A612C1EBA0034FF000090AA987F0C80631
:10E8A0008DED0C7AADF83A20ADF83830CDF82890DF
:10E8B000CDF834908E4686EA0616F6B20391C7F379
:10E8C0000727BEE80F0087EA161747EA062787EAF8
:10E8D000C606904FDEF800E084F804C00FC736B2D9
:10E8E00086F04A0383EA0313DBB2C6F3072181EA09
:10E8F00013113A4641EA03210CF1010C81EAC303EA
:10E90000142042F810E9FE264FF04A0E002184F848
:10E9100066C14FF0C80CE0702380043784F807E02C
:10E92000A670617184F806C0184612F8011B4140B8
:10E9300081EA0111C9B20B0983EA102343EA0123DA
:10E9400083EAC10109B288B2BA422080EDD181F0D8
:10E95000140181EA0111C9B24FEA111E8EEA102E8C
:10E960008EEA012E8EEAC10E0FFA8EFE1FFA8EF687
:10E97000DFF87CA126804FEA162C5FFA8EFE84F821
:10E980001CE084F81DC0DAF80410DAF80000DAF8A8
:10E990000820DAF80C30BAF818900AF5C7770FC7D4
:10E9A000DAF81000DAF8141003C704F28F16A7F88B
:10E9B0000090374684F8ABC184F8AAE104F2AB19A1
:10E9C00017F8011F2868FDF783FFB945F8D1524BAE
:10E9D000524A1B781278013B12F00100DBB214BFDF
:10E9E000C0214021172B03D84D4A134493F830809F
:10E9F0004C4B1A8897071ABF002341F010010123DE
:10EA000012F4027F18BF022312F0100F18BF062362
:10EA100012F0200F18BF1023002841F002824FF09F
:10EA2000030C94F866E10A938EF0460383EA03131D
:10EA3000DAB2130983F0920343EA022383EAC203A2
:10EA40001BB283EA0310C0B2C3F3072282EA10129A
:10EA500042EA002282EAC00212B282F0C80787EAC4
:10EA60000717FFB2C2F3072282EA171200238DF8BC
:10EA70002FC0032042EA072C039A8DF82C808DF8D2
:10EA80002D308DF82E108DF8300007CA8CEAC70C97
:10EA90000FFA8CFC1F4FE3718CEA0C1803C75FFA66
:10EAA00088F8CCF3072C8CEA181C4CEA082181EA80
:10EAB000C80894F808C03A700FFA88F88CEA080C75
:10EAC0008CEA0C1C5FFA8CFCC8F3072282EA1C1249
:10EAD00042EA0C22607AA17A94F80B80637182EA90
:10EAE000CC0212B2504080EA001C5FFA8CFC1BE0A2
:10EAF0000E2500209B260020405500204855002070
:10EB00000AD7233C24550020088D0020D34D6210E5
:10EB100067666666142500201C520020045C0020F5
:10EB2000E8A90308308D0020C2F3072080EA1C10FA
:10EB300040EA0C2080EACC0000B2414081EA011199
:10EB4000C9B2C0F3072282EA111242EA012282EA24
:10EB5000C10212B288EA020888EA08185FFA88F847
:10EB6000C2F3072282EA181242EA082294F80CC083
:10EB7000607BA17B84F804E082EAC80212B28CEACE
:10EB8000020C8CEA0C1C5FFA8CFCC2F3072282EAAE
:10EB90001C1242EA0C2282EACC0212B2504080EAF5
:10EBA0000010C0B2C2F3072282EA101242EA002229
:10EBB00082EAC00212B2514081EA0111C9B2C2F325
:10EBC000072282EA111242EA012282EAC102E17BB3
:10EBD00094F8108013B281EA030282EA0212D2B2E0
:10EBE000C3F3072383EA121343EA022383EAC2032F
:10EBF0001BB288EA030282EA0212D2B2C3F30723ED
:10EC000083EA121343EA022383EAC2031BB283F0AE
:10EC1000320282EA0212D2B2C3F3072383EA12134A
:10EC200043EA022383EAC2031BB29AB24FF0FE0CFE
:10EC30000920C8210EF1010EDBB284F802C04FEAB0
:10EC4000122CE070A17184F866E1228084F812C071
:10EC50006374DAF80000DAF80410DAF80820BAF879
:10EC60000C9007F5C07EAEE8070007F5C8778EF870
:10EC70000280AEF8009084F8A0C184F89F3116F8A5
:10EC8000011F2868FDF724FEB742F8D1029BC4F8A3
:10EC90005031FEF76DBEDFF824A27C4FDFF82092E2
:10ECA00041201AF0E9FABAF9023087FB0320DB179A
:10ECB000C3EBA00080B21AF0C3FABAF9003087FBA8
:10ECC0000320DB17C3EBA00080B21AF0B9FABAF93F
:10ECD000043087FB0320DB17C3EBA00080B21AF0DF
:10ECE000AFFA99F80010D8F80000FDF7F1FD94F89C
:10ECF00048A11AF0010700F01085654B1B689A06C1
:10ED000072D5644B644F1B789B0741F14B803B7D70
:10ED1000042B8CBF4FF0030A4FF0020A47201AF071
:10ED2000ABFA38681AF058FA78681AF055FAFB8985
:10ED30005A4AD8F80000A2FB0323C3F3471319462D
:10ED40000393FDF7C5FD3A8999F80010039B6420F1
:10ED50004B4000FB02F089F800301AF03DFA3F7D8D
:10ED6000D8F800004AEA8707FFB23946FDF7B0FD40
:10ED700099F80030D8F800005F40394689F80070F3
:10ED8000FDF7A6FD94F848A1BAF1000F2CD1444F2D
:10ED90004F201AF071FA38681AF01EFA78681AF0E3
:10EDA0001BFA50461AF018FA0121D8F80000FDF7B6
:10EDB0008FFD384A99F800301778D8F8000007F02E
:10EDC0000107394683F0010389F80030FDF780FD23
:10EDD00099F80030D8F800005F40394689F8007093
:10EDE000FDF776FD94F848A1029B2E4AC4F8443101
:10EDF0000AF10103DBB2A2FB0312D20802EB82028A
:10EE0000A3EB420384F84831FEF793BD94F8A43293
:10EE1000254AC4F8A0B202EB8302926C42B312AD51
:10EE200004F2AB23214E45F8203D002104F2BD231E
:10EE300031800B9380211523A52784F8AA32284618
:10EE400084F8A91284F8A872904728463188FAF706
:10EE50000DF80A9D164804F52A716D1A152DA8BFE4
:10EE600015252A4629F0C2F9124A94F8A4321570E1
:10EE7000114A013382FB0312A2EBE37202EB42025E
:10EE80009B1A84F8A432FEF783BD00BF67666666EE
:10EE90004055002044550020485500201F85EB5167
:10EEA0009C8D0020CDCCCCCCE8A90308B454002024
:10EEB000087200201D72002056555555245500201B
:10EEC000985B0020C24AC34BD4F8141130681B88E9
:10EED00092F80BE0C04A401A4FF47A71DFB201FB9E
:10EEE0000EF11B0A9777177588424FF00007D3770A
:10EEF00053759770177180F0F784B849DFF808C32D
:10EF00000B688968B648B74F007897F814A08CFB57
:10EF100003E8DB178CFB01EC4FEAE17EC3EBA801B1
:10EF200011770912CEEBAC0E5177F4214FEA2E2C5B
:10EF300082F820E091764FF0010E302182F81BE03C
:10EF400082F82210A84B82F821C04FF0750E78216C
:10EF500082F823E082F82410820783F81AA040F197
:10EF6000BF84D7F800C0A14AD7F804E0A04882FBCC
:10EF70000C194FEAEC7182FB0E82C1EBA9514FEAEA
:10EF8000EE79C9EBA25200FB01C9029200FB02E03C
:10EF900009EB4909974A4FEA490982FB0982049221
:10EFA00000EB4000934A4000039082FB0008049A63
:10EFB0009014029A0490F8893F8902EB820200EBD8
:10EFC000C00002EB820207F5FA770692BAF1050F4C
:10EFD0004FEA80021FFA87FA0398049F029201EB1E
:10EFE00081014FEAE97201EB810105914FEAE0717D
:10EFF000A7EB0200804F83F815A0024607FB129290
:10F00000059F4FEAA84840B200EB8709A8EB010032
:10F01000794F0399804607FB1010069F77494FFAF6
:10F0200088F84FEADC7C4FEADE7E83F809C083F87B
:10F030000EE0DFF8D8C108EB870E029F81FB078145
:10F040004FEAE778BCF800700397C8EBA1116C4F4A
:10F05000029187FB021887FB00170299DFF8B0C105
:10F060001FFA89F91FFA8EFE4FEAE2724FEAE0704A
:10F07000C2EB681883F80A90C0EB671283F80FE0C0
:10F080004FEA19274FEA1E29C1F3072E0399BCF84E
:10F090000000DF7283F810904FEA222783F80C807B
:10F0A0005A749DF80820DA714FEA282C4FEA1A2A80
:10F0B0004FEA112934BF4FF032084FF033089DF862
:10F0C0000C2083F80DC09F7483F816A083F808E025
:10F0D000DA7483F8149083F81B801877C4F810B1A1
:10F0E000FEF79CBBDFF82C91D9F80000FDF7E0FBA0
:10F0F00000283EF42BACD9F800000121FDF7D4FB29
:10F100000222002387F8742088F80030FEF71EBC26
:10F1100094F82C1194F82D31D8F800004A1C0133D2
:10F1200084F82C2184F82D31FDF7D2FBFEF7DEBBED
:10F13000344CDFF8E4904FF0000A0BE01B2B00F09A
:10F140009F820D2B00F079814FF0010389F8013087
:10F15000D8F80000FDF7B8FB00285FD0D8F8000011
:10F16000FDF7AEFB83B27E2B32682AD099F80110EE
:10F170000029EDD194F82E21002ADFD07D2B00F05C
:10F18000648294F83CE1BEF1000F04D080F02003CB
:10F19000DBB284F83C11511CC9B22244092984F81D
:10F1A0002E1182F8303100F044820829D0D8B4F80A
:10F1B0003A21134403EB132303F0FF03A4F83A317D
:10F1C000C6E784F82EA184F82FA189F801A0BFE733
:10F1D000C8590020C059002024560020B8540020EF
:10F1E0004455002048550020505600206BCA5F6BE4
:10F1F000806967FF83DE1B4340420F00D34D6210DE
:10F200001F85EB510C25002067666666A48D0020E3
:10F21000A68D0020384400202C00002094F83D31B9
:10F2200033B194F8313184F83D01302B00F0D785AB
:10F2300094F82F21BA4BBB49DFF818A3DFF81893D5
:10F2400002954FF0010E90464246002A00F05B8383
:10F250003268D21B012A00F21F8294F83E21002A54
:10F2600040F0348294F83FC133F81C00F0B984F8C0
:10F270003FE10A689506E7D59AF800209007E3D5A4
:10F28000A94FAA49FA89029D4FF4F36303FB02F3E5
:10F2900081FB0321DB17C3EB61114FF403601AF00C
:10F2A00005F8002384F82F31FEF731BB0CF1010C77
:10F2B0005FFA8CFCB0F5E06F84F83FC100F09A80F3
:10F2C0001BD8B0F5047F00F0498136D8B0F5887FAF
:10F2D00000F0D380B0F5007F00F0B880B0F5807FFB
:10F2E000B2D10A685207AFD50021029D19F0DEFFA6
:10F2F000002384F82F31FEF70ABBB0F5026F00F04F
:10F300005E816CD8B0F5E46F00F08480B0F5006FDA
:10F3100000F0DD80B0F5E26F96D1854B029DDA6B8F
:10F32000998A642303FB02F393FBF1F119F0BEFF0A
:10F33000002384F82F31FEF7EABAB0F5826F00F0AF
:10F340005581B0F5C06F00F02981B0F5806F7FF472
:10F350007BAF94F84031029D0133DBB2032B00F206
:10F36000AF8142F2107184F8403101FB03F1714B1F
:10F370001B88002B40F0A28101316F4B1B78DB070B
:10F380006E4B1B8848BF0431DF0748BF0A3198071E
:10F3900048BF14311A0648BF2831DF0548BF28315D
:10F3A000580748BF64311A0748BFC8319F0548BF96
:10F3B00001F5C871980648BF01F57A71DA0648BFB1
:10F3C00001F5FA615F0648BF01F57A614FF480608C
:10F3D00019F06CFF002384F82F31FEF798BAB0F5CE
:10F3E000046F1CD0B0F5116F56D0B0F5036F7FF4E9
:10F3F0002BAF3EE74E4B029D90469A6B998A642351
:10F4000003FB02F393FBF1F119F050FF84F82F8115
:10F41000FEF77DBA464B029D90461A6CEEE7484BCC
:10F42000029DB3F9041001EB81019046490019F0E7
:10F430003DFF84F82F81FEF76ABA4FF0010184F88E
:10F440002E1184F83031A4F83A2181E699F806208B
:10F45000002A3FF4F9AE3B4B3B491B68029D81FB00
:10F460000321DB17C3EBA1014FF4007019F01EFF5D
:10F47000002384F82F31FEF74ABA0A6852077FF555
:10F48000E3AE00214FF48870029D19F00FFF0023B6
:10F4900084F82F31FEF73BBA99F80520002A3FF493
:10F4A000D3AE2A4A107800283FF4CEAE284B029DF6
:10F4B0001B8803EB8303590091FBF0F14FF41160BB
:10F4C00019F0F4FE002384F82F31FEF720BA0A6801
:10F4D00095067FF5B9AE9AF8002090077FF5B4AE97
:10F4E0001CF0010F029D104F104900F068847A68EB
:10F4F00082EAE273A3EBE27303EB5303A1FB033154
:10F50000C908002AACBF41F0004141F040414FF42E
:10F51000006019F0CBFE002384F82F31FEF7F7B915
:10F52000E8A9030840550020485500201F85EB51ED
:10F53000D4540020DC8C0020045C0020308D00209E
:10F5400024550020B854002067666666D65900200E
:10F55000C0590020445500202C55002099F8052062
:10F56000002A3FF471AEC64A107800283FF46CAE12
:10F57000C44B029D5B7B002B00F08184C24B1B8837
:10F5800093FBF0F000EB800041004FF4047019F0A1
:10F590008DFE002384F82F31FEF7B9B999F80620C3
:10F5A000002A3FF451AEB94B029D99684FF4C060F8
:10F5B00019F07CFE002384F82F31FEF7A8B90D68FE
:10F5C000AD067FF541AE9AF800C01CF0020F3FF483
:10F5D0003BAEAF4F029D3B896421904601FB03F196
:10F5E00019F064FE84F82F81FEF791B90A6890063D
:10F5F00040F10181A74BA64F1878397D029D00F09C
:10F600000203002B0CBF00234FF47A7340F6B8328C
:10F6100008BF4FF4FA6210F0010F18BF13461944E7
:10F620004FF4826019F042FE002384F82F31FEF778
:10F630006EB9B4F83A21C2F1FF0293427FF484AD6F
:10F640004FF0010384F83D317EE54FF0010384F86B
:10F650003C317DE5FCF7F4FD8F4B1B68C01A40F68A
:10F66000B833984200F25881DFF858A29AF8043073
:10F670003A2B00F0C782002388F80030FEF766B905
:10F68000D8F80000FDF720F900287FF45DAD4FF0B9
:10F69000010384F82F315BE50023029D84F82F31AC
:10F6A000FEF735B9C4F8203184F81831DFF8188234
:10F6B00017F014FE94F82431FEF7FDB802315CE631
:10F6C000012384F8403142F2107150E67349029DE3
:10F6D000062019F0DDFB002384F83E0184F82F3169
:10F6E000FEF715B9013B84F85731FEF789BC013BA1
:10F6F00084F85631FEF763BB013B84F85A31FEF7BC
:10F7000088BF08F1FF3884F85F81FFF7BFBA0CF1BA
:10F71000FF3C84F85EC1FFF762B8614B1B88D805D7
:10F7200013D4D90600F17B839A0600F1DA835806D8
:10F7300000F1DC83190700F1DB83DA0700F1EC83C9
:10F7400013F0020F0CBF04270C27564B564A1B78A8
:10F75000D27803F001030AB143F00203532003936C
:10F7600019F08AFD484A128802EB820202EB8202FB
:10F77000900080B219F064FD002019F061FD4B4A41
:10F780004B491288D8F80000C2EBC212520081FB2C
:10F79000023111444FEAE27ACAEB612A5FFA8AFA2F
:10F7A0005146FDF795F899F80020039BD8F8000022
:10F7B0001F438AEA020A002189F800A0FDF788F8B1
:10F7C0003946D8F80000FDF783F899F80030D8F8EA
:10F7D00000007B40DBB2194689F80030FDF778F86D
:10F7E00094F848A1FFF7D0BA32493A2019F050FBFB
:10F7F0002870FEF7C1B8304A1268120600F1F7828D
:10F80000204A127B002A3FF41FAD94F84111029D5B
:10F81000032900F28383DFE801F059281902274BFE
:10F820001B6859799A79DB7901F1407101EB02216A
:10F8300001EB0341002384F841314FF4826019F059
:10F8400035FD002384F82F31FEF761B81C4B1A6890
:10F85000137A507992781B0403EB002313444A1C5B
:10F8600084F8412103EB0161E7E7154B1A68D3796E
:10F87000107952781B0403EB00231344EFE700BF19
:10F88000D6590020C8590020C0590020B854002083
:10F890004855002044550020E44300200585020817
:10F8A000308D0020045C0020B88C0020B28C002039
:10F8B0000308208015790208A88E0020C0AB002024
:10F8C000A4A80020CC430020CC540020BA4B1A68D6
:10F8D0009379D07812781B0403EB00231344BEE71E
:10F8E0002D22DA76FFF7FABBB44B31681B78C4F8E7
:10F8F0001411013B012B3FF600AB10210223917044
:10F900001371FFF7FABA029DFEF701B817F0D8FCA1
:10F9100001233B70FDF7A0BFA94AB2F84A3100218C
:10F920000133A2F84A3188F80010FEF70FB8A54E4F
:10F93000A54B00930024A6F13F01A44BA44A0891D3
:10F9400006F8404CA34909960AA8F9F767FB089EF8
:10F95000731C08933470089B2922591C08911A7053
:10F96000089BEA22591C08911A70089BC822591C4E
:10F9700008910AA81A7027F065FD471C0AA93A46A3
:10F98000089828F033FC089AD31901330893D4550A
:10F99000089B5A1C08921C70089B5A1C08921C70E9
:10F9A000089B5A1C08921C70089B5A1C08921C70D9
:10F9B000089B5A1C08921C70089B5A1C08921C70C9
:10F9C000089B5A1C08921C70089B5A1C08921C70B9
:10F9D000089B5A1C08921C70089B5A1C08921C70A9
:10F9E000089B5A1C08921C70089BFF22591C089106
:10F9F0001A70089B0122991812A808911A7050F8E1
:10FA0000283D9B1B337017F055FF2C70FDF7B4BFDA
:10FA1000DFED717AB0EE677AFEF7FEBE8846894662
:10FA20000846049105918E4606910391FEF7FAB9B6
:10FA3000644A6A4B0B9212AEA2F13D0046F8200DCB
:10FA40001988674FA2F1400300204FF00A0E02F818
:10FA5000400C082283F801E030469A70F9F7E0F98B
:10FA60003B686049DA1781FB0313C2EBA30399B229
:10FA70003046F9F7D5F90CF05DFABF680A9B3A0CED
:10FA8000591C0A911A700A9B3A0A591C0A911A7059
:10FA90000A9B5A1C0A921F700A9B5A1C0A921870E1
:10FAA000304617F007FFFEF71CB84F4F9FED4F8A07
:10FAB000B7F9022043480B9007EE902AF8EEE77A58
:10FAC00012AE67EE887AA0F13D01FDEEE77A46F8C6
:10FAD000201D00F8403C0823CDED027A00F83F3CA1
:10FAE0001E23BDF8081000F83E3C3046F9F798F99F
:10FAF000B7F9003007EE903AF8EEE77A304667EE55
:10FB0000887AFDEEE77ACDED027ABDF80810F9F7B4
:10FB100087F9B7F9043007EE903AF8EEE77A304605
:10FB200067EE887AFDEEE77ACDED027ABDF808102F
:10FB3000F9F776F9304617F0BDFEFDF7CFBF2C4A36
:10FB4000204B12680B93A3F14007002103F8401CDF
:10FB50002123D100BB7040F1B88126490326264BF2
:10FB60001B885A0500F1A681D80700F1BC8103F07B
:10FB70000203224A002B1CBF03261146DFF88080B7
:10FB80003246404628F032FB06EB080312A8013348
:10FB9000A8F1020140F8203D00225B1A06F8082077
:10FBA0007B7017F087FEFDF79FBFC4F81CB187F884
:10FBB0000090FDF751BE00BFA4A80020B58C002026
:10FBC0000C250020A4550020BA9000201CDA030860
:10FBD00054DA030860DA030800000000C05900206E
:10FBE000B8540020676666662455002058A08B41F3
:10FBF0004450002008D80308308D002024D8030882
:10FC0000675500209AF80240C4B1013CE4B20134C7
:10FC100054445146002211F8013B534083EA031338
:10FC2000DBB2120ADF0042EA03228C4287EA131396
:10FC300082EA0302EFD1002A7FF41DADBC4ABD4F1A
:10FC4000BD4B1288BD4CFA61DFF824931A68FA6242
:10FC50009B68B4F84A21F8660021FB64D9F80000DB
:10FC6000F963FA65FCF704F8029000287DF469AEA8
:10FC70000221D9F80000FCF717FE94F84C319AF8ED
:10FC800003200392642B4FF0040287F8742040F0A5
:10FC9000738194F84D31072B04BF9DF8083084F828
:10FCA0004D3194F84D31069307EB031ADAF804103E
:10FCB0000291084627F0C6FBDAF8081005915FFAB2
:10FCC00080FA084627F0BEFBC0B204900AEB00029F
:10FCD000069B9B48029902900832C27123F00F02E2
:10FCE00086468272049803F00F0300EBCA008EF878
:10FCF0000D3052468EF80E000EF10F0028F076FA05
:10FD0000904B049A05990AF10900184428F06EFAFC
:10FD10000298C37903F1010ACBB1013B5FFA83FC7E
:10FD20000CF1080CDFF84CE284440023073010F893
:10FD3000011B59408B00CA0883EA410302F01802F4
:10FD40004B404EFA02F253408445DBB2EFD17D4A7C
:10FD500003980AF8023028F0D3F994F84D310022C4
:10FD6000013384F84D3184F84C21029BDDF808A062
:10FD70009B785BB11AF80510D9F80000FCF7A8FDD4
:10FD800001359AF80230EDB2AB42F3D894F84C3119
:10FD90000322013384F84C3187F8742088F800205E
:10FDA000FFF7A2B94FF0010AFEF7B8BF0221D8F859
:10FDB0000000FCF779FD94F82431FDF77CBD3A682A
:10FDC00082EAE273A3EBE27303EB5303A1FB03317B
:10FDD000C908002AB8BF41F08041FFF798BB5A49D3
:10FDE000881F19F0F9F884F83E01FFF721BA1023B3
:10FDF0000027042218460AA9029D8DF828308DF8A4
:10FE000029208DF82A708DF82B708DF82C708DF8C4
:10FE10002D7017F017FA84F82F71FDF778BD34278D
:10FE200093E44A4AD278002A0CBF4FF0040C4FF0FA
:10FE3000050CFEF7F6BD0123D8F800003B70FCF777
:10FE40003FFD0746D8F80000FCF73AFD7B067DF43D
:10FE500003AD8A284ED08E287DF4FEAC94F818317C
:10FE6000002B7DF416AD3A4BC4F820312D2384F8D5
:10FE70002431FDF7F8BC4FF00108FEF7DBB82C4B3E
:10FE80001888FFF77FBB2A499A790B8803EB830315
:10FE900003EB83034FEA83081FFA88F8002A00F077
:10FEA0001081254B1B680FFA83FA0CF043F840B21F
:10FEB000FDF7C0BE0326274960E6984699461846D6
:10FEC000049305930393FDF7ADBF234B234A1B68AF
:10FED000234903F48003002B16BF11460426032692
:10FEE0003DE6242731E41F49042647E610272CE489
:10FEF00020272AE41C4B1B689F067DF5ADAC94F8C7
:10FF00001831002B7DF4C5AC184BC4F820312D23DB
:10FF100084F82431FDF7A7BC082716E44B1CDBB29C
:10FF2000042B84F841314FEA01613FF483AC84E44F
:10FF3000C05900202C000020B85400200C250020BF
:10FF4000E8870020EE87002044260020B88C00209F
:10FF50002456002050DA0308A88E002008D8030891
:10FF60000CD803081CD80308405500205056002028
:10FF7000384400200007090E97F875A05B490495E6
:10FF80001AF00F0F04BF0AF1010A5FFA8AFABAF1F8
:10FF9000070F28BF4FF0010A4FEA0A1C07EB0C03BA
:10FFA000187C534B02930A18002392F82410504AED
:10FFB00093725FFA8CF31A464E4B964607EB0C028F
:10FFC0004EEA000001291870D26803F101000CD933
:10FFD0000239C9B28D1C1D44034603F8012BAB4204
:10FFE0004FEA1222F9D101310844BC4422F06003E7
:10FFF0000AF1010A9CF811205FFA8AFA1343BAF158
:020000040801F1
:10000000080F037000F1010340D04FEA0A1C07EB10
:100010000C01384A087C354901449A1A91F8241099
:1000200055180EF1100E132D5FFA8EFEC6DD049DDD
:100030000298DFF8CCE0D2B2931DDBB243F040016E
:10004000C17103F1010CCBB10532D3B20833C3182F
:1000500004930EF10100002310F8011B59408B009E
:1000600083EA4103CA084B40234902F0180241FACF
:1000700002F25340049A8242DBB2EDD103980CF8AD
:100080000E3087F875A028F03BF86EE6194A049DFB
:100090009A1ACDE7984699461846049305939E46CA
:1000A0000393FDF7BFBE154B9046B3F900A0642043
:1000B000FDF7C0BD98469946184604930393FDF793
:1000C000B1BE4FF0FF33EEE60393FDF7ABBE9846AB
:1000D0000393FDF7A7BE984699460393FDF7A2BE8A
:1000E0009846994618460393FDF79CBEE8A9030875
:1000F000E8870020F58700200007090EB85400208B
:10010000EE87002038B50B4C23688BB15A68821AF1
:10011000002A054604DA0CE05A68AA1A002A07DB0E
:100120009A68226018461A6890472368002BF3D11A
:1001300038BD38BD487300200D4B042100228907CB
:1001400010B4027203F1600402D5197981540132AE
:100150009C4203F1180308D0072A06DC9979890725
:10016000F3D49C4203F11803F6D15DF8044B7047B9
:10017000D0D6030810B4104C0423214613F0010319
:100180004FF0000201F1180108D10132052A0ED00A
:100190008B7913F0010301F11801F6D002EB420252
:1001A00004EBC2025DF8044B1379037070470370CF
:1001B0005DF8044B704700BFD0D6030808B511F0B6
:1001C000A1FFFBF7DFFA00BF038A2DE9F04785891D
:1001D000ADB21D4029D00F4606464FF000484FF003
:1001E0000009B5FA85F328FA03F2D24391B21B3B1A
:1001F00015403182042B16D8DFE803F0312921198C
:1002000003007B6A002B32D003F1FF3A1FFA8AFA0F
:10021000C7F824903C6A34B1236820465146984779
:100220006468002CF8D1002DDBD1BDE8F087386878
:10023000716B036889B29847002DD2D1F5E77868D1
:10024000B16B036889B29847002DCAD1EDE7B86851
:10025000F16B036889B29847002DC2D1E5E7F868D1
:10026000316C036889B29847002DBAD1DDE7F36A93
:100270001FFA83FACEE700BF2DE9F04F2DED028B78
:10028000A0F10A0389B00C46E72B00F21187DFE8E2
:1002900013F01C010F070F070F070F070F070F07BA
:1002A0000F070F070F070F070F070F070F070F079E
:1002B0000F070F070F070F070F070F070F070F078E
:1002C0000F0780010F070F070F0771010F070F07B7
:1002D0000F0764010F076F020F072C020F0721029F
:1002E0000F0719020F07F4010F07E0010F070F07AF
:1002F0000F07DA01D3010F0776030F070F076F030C
:100300000F0747030F070F070F073C030F070F07E0
:100310000F070F07E4020F07FC000F072603030374
:100320000F070F070F070F070F070F070F07DB0454
:100330000F07AD040F0779040F0725040F071104F9
:100340000F070F070F070F07BE0384037D03B302D8
:10035000E800F405DF051906D4050F079C057F05A5
:100360000F070F070F070F0760050F070F073E0561
:100370000F070F070F07A1068906740631060F073E
:100380000F070F07C906B106D9061D050F070F078E
:100390000F070F070F070F070F070F070F070F07AD
:1003A0000F070F070F070F070F07BE030F070F07F2
:1003B0000F070F070F070F070F070F070F070F078D
:1003C0000F070F070F072D010F070F070F070F0765
:1003D0000F070F070F070F070F070F070F070F076D
:1003E0000F070F070F070F070F070F070F070F075D
:1003F0000F070F070F070F070F070F070F070F074D
:100400000F070F070F070F070F070F070F070F073C
:100410000F070F070F070F070F070F070F070F072C
:100420000F070F070F070F070F070F070F070F071C
:100430000F070F070F070F070F070F070F070F070C
:100440000F070F070F070F070F070F070F070F07FC
:100450000F070F070F070F070F070F070F079E0163
:10046000A901AE4E337853B1AD4F002537F8021FC6
:100470002046F8F7FBFC33780135AB42F6DC01206F
:1004800009B0BDEC028BBDE8F08FA44E3378002B91
:10049000F5D0A44F0025B846236817F81520591C3D
:1004A00021601A7098F8011001EB810101EB8101C4
:1004B00001F2EE2189B22046F8F7D8FC33780135F5
:1004C000AB4208F10208E7DCD9E7974D284626F051
:1004D000B9FF0028D3DD2B460544226813F8011B21
:1004E000501C9D4220601170F7D1C8E70B68DFF8FF
:1004F0007CC2591C9CF8002021601A709CF80030C6
:10050000002BBCD0894E8A4D8A488B490023226833
:1005100016F8017F02F1010EC4F800E0177022689E
:1005200015F8017F02F1010EC4F800E0177022688F
:1005300010F8017F02F1010EC4F800E01770226884
:1005400011F8017F02F1010EC4F800E017709CF869
:10055000002001339A42DADC91E70B68774A581C95
:1005600011782060197023685278591C216001208D
:100570001A7085E7724D08462988F8F777FCA98834
:100580002046F8F773FC20462989F8F76FFC012014
:1005900076E76C4D05F15006287823F0E3F92368DF
:1005A000027A591C21601A7023686A78591C2160EC
:1005B0001A702368AA78591C21601A702368EA7897
:1005C0000435591CAE4221601A70E5D157E75E4DE3
:1005D0000846E989F8F74AFC2046A989F8F746FC5D
:1005E00001204DE7594B03F1700522681978501C22
:1005F0002060117022685978501C206011702268A8
:100600009978501C206011702268D978501C2060A5
:10061000117022681979501C206011702268597974
:10062000501C20601170226899790733501C9D423C
:1006300020601170D9D122E70B680122991821603E
:1006400010461A701CE708460021F8F7F7FB012056
:1006500016E73F4D3F4E05F1300795F902103E4B2E
:1006600093F906208A4203F1080300F024859E4294
:10067000F6D10835BD42F0D101E7384B03F15A05F8
:1006800022685979501C2060117022681978501C1A
:100690002060117022685978501C20601170226807
:1006A0009978501C206011702268D978501C206005
:1006B0001170226819790633501C9D422060117018
:1006C000DED1DCE60B68264A591C527D21600120F0
:1006D0001A70D5E6234D05F1800655F8041F204613
:1006E000F8F7ACFBAE42F8D1C9E61F4D05F1400664
:1006F000B5F880102046F8F7B9FB236895F88220FA
:10070000591C21601A70236895F883200435591C00
:10071000B54221601A70EBD1B1E600BF2073002012
:10072000068D0020404C0020D05100209762002010
:10073000A7620020C7620020B76200201C52002080
:10074000E041002020520020F451002058460020B3
:10075000D090002018900020E88F0020F04C00205E
:100760001C90002090560020945600209562002096
:10077000B84D0B682A7A591C21601A70A98B204643
:10078000F8F774FB298B2046F8F770FB698B20463D
:10079000F8F76CFB2368EA7C591C21601A70A98C5D
:1007A0002046F8F763FBE98C2046F8F75FFB2368E7
:1007B000AA7F591C21601A70236895F82020591CC3
:1007C00021601A70698C2046F8F750FB2368EA7A9A
:1007D000591C21601A70E9682046F8F72FFB23683E
:1007E0002A7C591C21601A70236895F82120591C15
:1007F000216001201A7043E6974D984E9FED988A2C
:10080000DFF8A482DFED978A05F120070EE0FCEE09
:10081000E77ACDED017ABDF8041020460435F8F7EB
:1008200025FBAF4206F118063FF429AE717C002982
:10083000F3D08D4BD5ED007A1B78012BE7D18B4B94
:100840001B68DB0440F1F384F5EE407AF1EE10FA18
:1008500040F01F8540F2DC51DFE70B68844D591CE6
:100860002A7921601A7023686A79591C21601A70EC
:1008700029882046F8F7FAFA2368AA79591C2160DA
:100880001A7069882046F8F7F1FA2368EA79591C4A
:10089000216001201A70F3E50B68764E01255A1C81
:1008A0000A601D700B68B278591921601A7012F035
:1008B000C9FA2368704A71495F1927601870B1F945
:1008C0000010B2F90000F8F74BFC23685A192260B7
:1008D000187031882046F8F7C9FA2846D0E50B6829
:1008E00000255A1C0A601D700B685A1C0A601D7096
:1008F0000B685A1C0A6029461D702046F8F79EFABC
:1009000029462046F8F79AFAB9E50B6800255A1CE3
:100910000A60204629461D70F8F790FA2946ECE750
:100920000B68574A574D1178574A581C2060197068
:1009300011682046F8F782FA2368464A591C127A51
:1009400021601A7029882046F8F790FAA988204675
:10095000F8F78CFA29892046F8F788FA0021204612
:10096000F8F784FA20460021F8F780FA012087E59D
:10097000084608223749F8F731FA012080E50B686C
:10098000424A581C917820601970ECE50846102204
:100990003F49F8F723FA012072E53E4B9B8AB3F5F5
:1009A000006F00F25984B3F5806F00F26F84B3F5E5
:1009B000007F34BF01270227374D05F10C0655F89B
:1009C000041B91FBF7F1204689B2F8F74FFAB542C4
:1009D000F5D1324D324F05F10C06B5EC010AD7EDD9
:1009E000087A80EE270A27F00BFE81B22046F8F73E
:1009F0003DFAB542F1D12B4D05F10C0655F8041B1B
:100A0000204689B2F8F732FAAE42F7D137E5002531
:100A10008146DFF89880DFF898B005950495069533
:100A2000079501214FF6FF7A05E001350B2D00F007
:100A3000608318F9011F4F1C4AFA05F3F5D0DE0751
:100A4000F3D5BBF800302B41D807EED506A8F8F750
:100A500043FDEAE71C900020FC4F0020D8910020C5
:100A60000000404200E08244BC920020A88E00209A
:100A7000504F0020F2A900205A5000205C50002066
:100A80001C520020E041002024AA00201052002027
:100A9000EC4F0020D45400200C5500209C8E0020E8
:100AA00004980020DC4F0020DB9B91416CAA0308D6
:100AB000308D00200B68AD4AAD49D078AD4A5D1C41
:100AC0002560187023684979581C206019702368C4
:100AD000D278591C216001201A70D1E400212046EF
:100AE000F8F7C4F900212046F8F7C0F900212046A4
:100AF000F8F7BCF92368A04D00265A1C22601E702E
:100B000023682A68591C92F82C2021601A702368E7
:100B10002A68591C92F8362021601A7023682A68C6
:100B2000591C92F8372021601A7023685A1C2260E1
:100B30001E7023685A1C22601E7023685A1C226093
:100B40001E702B682046598FF8F790F92B682046C5
:100B5000198FF8F78BF923682A68591C92F82E2010
:100B600021601A7023685A1C22601E702B68204670
:100B7000598EF8F77BF92B682046998EF8F776F9AD
:100B800001207DE47D4E0B6872797B4D591C2160FC
:100B90001A702B682046198CF8F768F92B682046E4
:100BA000D98BF8F763F971892046F8F75FF9B189B5
:100BB0002046F8F75BF92B682046598CF8F756F970
:100BC0002B682046998CF8F751F9F1892046F8F7FF
:100BD0004DF9318A2046F8F749F92A68236892F8D6
:100BE0002620591C216001201A7049E4634EF378D5
:100BF000002B00F025830B680822591C21601A7015
:100C000023680122991821601A7023685C4D591CD1
:100C10002A7921601A702368AA78591C21601A70F9
:100C200029882046F8F722F9E9892046F8F71EF9C5
:100C30002368F279591C21601A702368EA78591CDC
:100C4000216001201A701BE41AF0D8FDFF28064627
:100C500000F0058308A9002501F8125D0DF10D00D3
:100C60008DF80D501AF0AAFD08A800F8115D1AF0D1
:100C700099FD08A800F8105D1AF088FD08A820F872
:100C8000085D1AF077FD23685A1C22601E702368E5
:100C90009DF80D20591C21601A7023689DF80E20C4
:100CA000591C21601A7023689DF80F20591C21607F
:100CB0001A7023689DF81020591C21601A70204674
:100CC000BDF81810F8F7D2F8FFF7D9BB0B682D4F15
:100CD000591C3A7821601A703B78002B3FF4CFAB57
:100CE0000025EEB2304617F0CBFF23684278591C3E
:100CF000216030461A7017F0C3FF01892046F8F7CB
:100D0000B5F83B780135AB42EBDCFFF7B8BB1E4DC5
:100D100005F16006A9882046F8F7A8F8E98820467A
:100D2000F8F7A4F829892046F8F7A0F82368AA7AEA
:100D3000591C21601A702368EA7A591C21601A70C4
:100D400055F80C1B2046F8F779F8AE42E2D1FFF7D0
:100D500096BB0E4952232268501C2060137011F874
:100D6000013F002BF7D1FFF78ABB00BFF4510020F1
:100D70008C58002004520020A4A80020848E00205B
:100D800098920020F48A0020644500203CAA0308C1
:100D9000B44800232268056803EB4301561C6D5CD0
:100DA00026601570026825680A446E1C5278266019
:100DB0002A70026825680A4401339278691C0A2B5C
:100DC00021602A70E6D1FFF75ABBA74D0B682A684D
:100DD000591C127821601A702B6822689978531C6C
:100DE0002360002311702A6821681A440133527964
:100DF000481C032B20600A70F5D123682A68591C0F
:100E0000127A21601A7023682A68591CD2782160EE
:100E10001A7023682A68591C127921601A702B688D
:100E200020465989F8F722F82A682368527A591C13
:100E300021601A702A68FFF796BB00212046F7F759
:100E4000FDFF20460021F8F711F80120FFF718BB3D
:100E5000864B08461988F8F709F8854B204619880B
:100E6000F8F704F8834B22681B78511C03F0010348
:100E7000216001201370FFF703BB7F4B0A681B78CA
:100E80007E4D511C03F002032160137023682A7DFC
:100E9000591C21601A7029682046F7F7CFFF69684E
:100EA0002046F7F7CBFF29892046F7F7DFFFE989CE
:100EB0002046F7F7DBFF2046298AF7F7D7FF012006
:100EC000FFF7DEBA6E4D08462988F7F7CFFF69882D
:100ED0002046F7F7CBFFB5F904306A4AD91782FBF1
:100EE0000323C1EBA301204689B2F7F7BFFF01201E
:100EF000FFF7C6BADFF8B4E10027FEB2714600235F
:100F00002268501C206016702268501C20601370EC
:100F1000226811F8010F0133551C062B2560107053
:100F2000EED10137062F0EF1060EE6D15649002309
:100F30002268501C206017702268501C20601370BB
:100F4000226811F8010F0133551C0B2B256010701E
:100F5000EED123684D4A581C072120601970236880
:100F60000021581C20601970236892F8F020591C49
:100F7000216001201A70FFF783BA0B68444A454983
:100F80001078454A5D1C2560187023688978581CC4
:100F90002060197023689278591C216001201A7012
:100FA000FFF76EBA0A683D4B3D491878551C25601D
:100FB000107022685878551C2560107022689B7844
:100FC000501C206013702046C988F7F74FFF01209E
:100FD000FFF756BA324D08462988F7F747FF698868
:100FE0002046F7F743FF2046A988F7F73FFF012087
:100FF000FFF746BA0A682B4B501C19782060117015
:1010000022685978501C2060117022689978501C11
:10101000206011702268DB78511C21600120137060
:10102000FFF72EBA204D0846298AF7F71FFF698A75
:101030002046F7F71BFF2046A98AF7F717FF012084
:10104000FFF71EBA144B0F49B3F9003081FB03219F
:10105000DB17C3EBA101204689B2F7F707FF012098
:10106000FFF70EBAA4A80020C0AB0020A48D00207A
:10107000A68D0020588D00204455002048550020A2
:101080002455002067666666775700209456002036
:10109000848E0020F451002004520020EC510020E6
:1010A000384F00207C620020989200205357002087
:1010B0000020FFF7E5B923685A1C226019702988BF
:1010C0002046F7F7D3FE2368EA78591C21601A708E
:1010D00023682A79591C21601A702368AA79591C3F
:1010E00021601A7023686A79591C21601A70FFF711
:1010F000C0BADFF83CA200254FF008080135C5F161
:10110000200208FA02F2A5F120032AFA05F6164396
:1011100028FA03F31E43252D06F001024FF00003C9
:101120000BD01343EAD0E8B225F01EFC0028E5D02E
:10113000294606A8F8F7D0F9E0E7754B1B78DA07DF
:1011400000F194800025734E2F4602E00135252DD5
:101150000DD029463046F8F7CFF90028F6D02946B9
:1011600006A8F8F7C9F900285CD10137EEE76A4B09
:101170006A4DB3F850102046F7F778FE002120465C
:10118000F7F774FE664B19684B0103F02002C1F3B8
:1011900040031343C1F3800243EA4203C1F3C00298
:1011A00043EA8203C1F3401243EAC20301F0100193
:1011B00019432046F7F75AFE04A904222046F7F700
:1011C0000DFE23682978574A581C20601970118831
:1011D0006429A8BF64212046F7F748FEB9F1960FAD
:1011E00049D000212046F7F741FE2168B7F11903E5
:1011F00048BFA7F11203A3F3C4034A1C2260204690
:101200001A460B7005A9F7F7E9FD2368464A581CF2
:1012100010212060197020461188F7F70FFE012079
:10122000FFF72EB9394604A8F8F756F99DE7F4EE12
:10123000C87AF1EE10FA49DA4FF47A71FFF7EDBA95
:101240000B68B178394A581C2060197023681278ED
:10125000591C21601A70D8E40827FFF7ADBB23683A
:101260005A1C226001201E70FFF70AB9069B43F04A
:101270000103069366E723680322591C21601A7054
:1012800023686A78591C21601A70AEE70427FFF7BB
:1012900093BBF4EEC87AF1EE10FA3FF5DBAAF4EE58
:1012A000E87AFDEEE77AF1EE10FA17EE901A20D800
:1012B0006FF4F973303903FB01F140F2E73391FB2E
:1012C000F3F101F2DB5189B2FFF7A7BAFDEEE77A3D
:1012D00040F2E73217EE903A303B02FB03F388FB13
:1012E0000312D917C1EB622101F2E93189B2FFF78C
:1012F00094BA40F2F313A1F5836103FB01F140F2CC
:10130000E73391FBF3F101F2DD5189B2FFF785BAC2
:10131000045C00203C97002068010020B49000206D
:1013200040550020A2530020DC8C0020E851002012
:1013300090E33FF408B501210220FBF741FE094B81
:101340001B7803F00503052B08D000210120FBF7D3
:1013500037FE00210846FBF733FEFEE710F064FF7E
:10136000F3E700BFB4410020022828BF022010B4D8
:10137000084C094B207000EB8002C0EBC202074909
:101380005DF8044B013003EB4203C0B20B600CF07C
:101390003BBA00BFB4900020B2A80020A4A800204F
:1013A00008B51CF0B5F9FAF73DF9BDE808401CF0A6
:1013B00097B900BF38B5484B5A899989914224BFE3
:1013C00000225A81198ADA89914224BF0022DA81E7
:1013D000DA78CAB1072A41496AD091F85700404DDE
:1013E000012400210A282C709C70D9715DD00C2832
:1013F00007D0002A6CD0DFED3B7A072A0ED00A28EE
:1014000062D0DFED397A09E0344A92F857000A28B1
:1014100056D00C285BD1D979DFED347A344C9FED6E
:10142000350AA278002918BFF0EE407A062A04D8BF
:10143000314901EB820191ED0F0A217979B1013A2D
:10144000032A0BD8F7EE007A87EE800A27F0D8F847
:101450002388984228BF1846208038BD38BD9B7825
:101460001F4A07EE103A1178B8EEC77A67EE277A6E
:1014700007EE101AB8EEC77A27EE277AB4EEC70A3D
:10148000F1EE10FAEADD80EE277AFDEEC77A17EE6C
:10149000903A102BA8BF1023012BB8BF0123DBB259
:1014A0008B4238BF0B46137038BDDFED147AA4E7CA
:1014B00091F857000A2803D00C28ACD0D9799AE7C4
:1014C000D979DFED0E7AA9E7DFED0D7AA6E7D979B4
:1014D000DFED047AA2E700BF848E0020049800208C
:1014E000E85100206F1203396F12833A0AD7A339EB
:1014F000989200206F1203383CAA03085304E9387D
:101500000F506E3A2DE9F047AF4FB04E1CF000F986
:10151000BE421ED2DFF84083DFF840934446258860
:1015200062197DB14A450DD2052D0BD933886188EA
:10153000C3F30B03994200F0F58014462588621925
:10154000002DEFD1716830461436FCF7F6F8BE4234
:10155000E4D39F4A1378A3F1170102290FD99D49BB
:1015600011F83300002840F02281D8000144497866
:1015700029B1994911F833300BB918231370974CDE
:101580006378022B84BF002363702378022B84BF0F
:1015900000232370924B9A78042A00F0FF8032B91E
:1015A0001A88B2F5F07F84BF4FF4F0721A808D4D27
:1015B0008D4A2B681A40002A00F00281D80700F1FA
:1015C000E880590400F1E0801A0700F1D8809B04FC
:1015D00000F1CE80854D2B685A8C998C914224BFA6
:1015E00000225A84FFF7E6FE1FF00CFA002800F0F4
:1015F000BB804020FCF7D8F84FF40070FCF7D4F81B
:101600004FF40030FCF7D0F84FF40010FCF7CCF8A2
:101610004FF00070FCF7C8F84FF08060FCF7C4F89A
:101620006378022B06D8724A724903EB430302EB3C
:1016300083030B602378022B07D803EB83016E4AE8
:10164000C3EBC10302EB43032B6025F0DFF900215C
:1016500030226A4829F0E1F8286810F025FA684B32
:101660002D6803F1500102E0043399427AD01A78D0
:10167000002AF9D19C78D8788442F5D26149624B2E
:101680000A7028461D601AF00DF8604B604A1E79FA
:1016900060496148614B1160C825642212FB065203
:1016A0005F4C406B31F8061C5A60002221809A6022
:1016B000DA601A615A619A61DA6183F8202083F84E
:1016C000212008B11BF064FE564B9FED575A1B8832
:1016D000564A9FED576A5579564C57495748086006
:1016E00006EE903AF8EEE66A1388C5EE265A07EE43
:1016F000103A53881279C4ED005A07EE903AB8EECA
:10170000C77A4F4BF8EEE77A1D725A7227EE067AC7
:1017100067EE867ABDE8F04783ED017AC3ED007A83
:101720001BF0DEBF63799B077FF407AF716894F805
:1017300004A03046FCF701F83388BAEB133F04D01D
:101740001436BE42FFF4EAAE03E773887068AA1F3E
:10175000C3F30B039A4204F10601A8BF1A4626F010
:1017600045FDEDE7012289E736480AF045FC40E7F0
:101770003548FCF719F84020FCF716F82AE73348FB
:10178000FCF712F82B6822E73148FCF70DF82B68BC
:101790001AE73048FCF708F82B6812E79A8AB2F586
:1017A0007A7FBFF404AF4FF47A729A82FFE6D800D2
:1017B0000C186468002C7FF4D9AE17241470D5E699
:1017C00043F400532B60F9E6D405000888010008B3
:1017D0001C520020C0CC030898AF0308B49000202E
:1017E0009892002024AA002009600002A4A80020EA
:1017F000BAA90020C0AB0020B2A80020982A00207F
:101800002052002004230020CC2A0020504F00202A
:1018100014970020FA510020D4540020B88C0020E6
:1018200024770020F4280020C0C9FB48D0270020DE
:1018300017B7D138F8280020BC4C00203661023D93
:10184000984C0020D0900020094000020160000266
:101850000920000208600002024000080080000821
:1018600008B51BF055FFF9F7DDFE1BF039FFFFF758
:1018700049FE0120BDE808400BF0C6BF38B50D4C4D
:101880000D4DAC4206D2616820461434FBF755FF7B
:10189000AC42F8D3F9F762FB084A094B094C1460D3
:1018A000002209491A705A7008480860BDE838409B
:1018B0001DF012BD88010008D4050008A4A800206E
:1018C000B4900020B2A80020C0AB0020BAA900202C
:1018D00008B5FFF7D3FF1BF01BFFF9F7A3FEBDE828
:1018E00008401BF0FDBE00BFF0B50C2934D8DFE87E
:1018F00001F0893333335E3333333433333307000A
:10190000048C9689B2F802E01788734D24F4805451
:101910002404240C0484038C8488818B23F40053D6
:1019200021F4E6411B0409041B0C46EA0E06090CCF
:1019300043EA063341EA0721A8429BB2A4B289B226
:1019400000F09E8005F58065A84200F099809268BD
:101950008480818302640384F0BD048C9589B2F88D
:1019600002C0B2F800E05C4F24F480742404240C1C
:101970000484038C8688818B23F400731B0421F07C
:1019800073011B0C45EA0C04090443EA0423090C07
:10199000B8429BB2B6B241EA0E015CD04F4CA042B5
:1019A00059D0926886808183C2630384F0BD048C21
:1019B0009589B2F802C0B2F800E0474E24F0100456
:1019C0002404240C0484038C8788018B23F02003D7
:1019D00021F4E6411B0409041B0C45EA0C04090C24
:1019E00043EA041341EA0E21B0429BB2BFB289B26E
:1019F0005DD03A4CA0425AD09268878001838263BE
:101A00000384F0BD048C9789B2F802E01688324D49
:101A100024F001042404240C0484038C8488018BA6
:101A200023F002031B0421F073011B0C47EA0E078D
:101A300009043B43090CA8429BB2A4B241EA060147
:101A400025D005F58065A84221D092688480018365
:101A500042630384F0BDD589148A578A23F4006356
:101A600043EA05254FF6FF332B40958826F4405670
:101A70003C4343EA052346EA04169BB2B6B290E71C
:101A8000158A24F4804444EA8514A4B25FE7D68919
:101A9000158A578A23F00803334324F44074968848
:101AA0003D4323F004032C433343A4B2CDE7D48950
:101AB000158A568A23F0800343EA04134FF6BF7455
:101AC0001C40938827F44067354344EA031347EAF0
:101AD00085079BB2BFB28FE70000014000040140C0
:101AE0002DE9F04F7822002183B0C248C24CDFF8C4
:101AF0002493C24DC24EC34FDFF81C8328F08DFEE5
:101B0000C148C249DFF814E3DFF814C30022A35828
:101B1000834200F0D381B3F1804F00F0D181AB421A
:101B200000F0D081B34200F0CF81BB4200F0CE8103
:101B3000734500F0CD81634500F0CC81434500F052
:101B4000CB81DFF8E0A2534500F0C8810AF5806A36
:101B5000534500F0C5810AF5806A534500F0C28103
:101B6000AAF5983A534500F0BF810AF5806A5345BB
:101B700000F083810AF5806A534508BF0D2300F009
:101B80007D811832782AC2D13920FAF791FF0028D6
:101B900040D001689E4C01F13F4303F57E039A0A51
:101BA0000123A25C02F01F045209032A03FA04F382
:101BB00000F09C81042A00F0B781022A03D1934AE5
:101BC000546C2343536483880093B3FA83F3C3F1C3
:101BD0001F039BB2DA0801EB820203F00703106ACD
:101BE0009B000F249C4020EA04001062146A03202A
:101BF00000FA03F3234313620846002302226946D6
:101C00008DF804208DF805308DF806308DF80730FA
:101C100018F0F2F93820FAF74BFF00283FD001689E
:101C20007B4C01F13F4303F57E039A0A0123A25C3A
:101C300002F01F045209032A03FA04F300F06A8138
:101C4000042A00F07B81022A03D1704A546C23439A
:101C5000536483880093B3FA83F3C3F11F039BB2E9
:101C6000DA0801EB820203F00703106A9B000F24DD
:101C70009C4020EA04001062106A022404FA03F374
:101C8000034313620846002369468DF804408DF82B
:101C900005308DF806308DF8073018F0ADF9372093
:101CA000FAF706FF00283FD00168594C01F13F4385
:101CB00003F57E039A0A0123A25C02F01F04520975
:101CC000032A03FA04F300F02081042A00F03B8188
:101CD000022A03D14D4A546C2343536483880093F2
:101CE000B3FA83F3C3F11F039BB2DA0801EB82025C
:101CF00003F00703106A9B000F249C4020EA0400B5
:101D00001062106A022404FA03F3034313620846C4
:101D1000002369468DF804408DF805308DF80630B3
:101D20008DF8073018F068F93620FAF7C1FE002860
:101D300040D00168364C01F13F4303F57E039A0A17
:101D40000123A25C02F01F045209032A03FA04F3E0
:101D500000F0D680042A00F0EC80022A03D12B4A3E
:101D6000546C2343536483880093B3FA83F3C3F121
:101D70001F039BB2DA0801EB820203F00703106A2B
:101D80009B000F249C4020EA04001062146A032088
:101D900000FA03F323431362084600230222694634
:101DA0008DF804208DF805308DF806308DF8073059
:101DB00018F022F91020FAF77BFE00285AD00168AB
:101DC000134C01F13F4303F57E039A0A0123A25C01
:101DD00002F01F045209032A03FA04F300F08B8077
:101DE000042A00F09C80022A1ED1084A546C234326
:101DF000536419E010530020D0D6030800040040BB
:101E000000080040000C0040000001400038024083
:101E1000FCD3030858D3030800040140001000401D
:101E2000001400400040014083880093B3FA83F31C
:101E3000C3F11F039BB2DA0801EB820203F0070330
:101E4000106A9B000F249C4020EA04001062106A74
:101E5000022404FA03F3034313620846002369468D
:101E60008DF804408DF805308DF806308DF8073078
:101E700018F0C2F803B0BDE8F08F0C2309EBC303E0
:101E80004FF0010A1B7903F01F0B5B09032B0AFAC1
:101E90000BFA0ED0042B07D0022B7FF472AE4B6CE2
:101EA0004AEA03034B646CE60B6B4AEA03030B63D9
:101EB00067E60B6C4AEA03030B6462E60023DDE786
:101EC0000123DBE70223D9E70323D7E70423D5E780
:101ED0000523D3E70623D1E70723CFE70823CDE780
:101EE0000923CBE70A23C9E70B23C7E7184A146C79
:101EF0002343136467E6164A146C2343136493E781
:101F0000134A146C234313642DE7114A146C2343C2
:101F10001364E3E60E4A146C2343136499E60C4AF7
:101F2000146B234313637FE7094A146B2343136342
:101F300049E6074A146B2343136314E7044A146BFE
:101F40002343136385E6024A146B23431363C5E6F8
:101F50000038024001490248FEF736B960530020BC
:101F60000004014001490248FEF72EB960530020E9
:101F70000004014001490248FEF726B93853002009
:101F8000000C004001490248FEF71EB91053002022
:101F900000040040F0B504683F4DA30AAB425CD09A
:101FA0003E35AB4255D0403DAB4200D0F0BD4FF086
:101FB000200E00264779B0004FEA970C002956D032
:101FC00063460227A5899F4083190CEB43032F43E7
:101FD00003F1040C314DBFB245F8231045F82C2015
:101FE000A781EFF31181502282F31288821905EB49
:101FF000C202136953B313620433821905EBC202A0
:10200000576917B11F6053690433821905EBC20287
:10201000976917B11F6093690433821905EBC202F7
:10202000D76917B11F60D36904330027CAB21F6094
:1020300082F31188304405EBC000036A8BB9A38991
:1020400023F001031B041B0CA381F0BD05EB0E0361
:10205000D3E74FF0700E0226ACE74FF0480E012692
:10206000A8E7A3899BB243F00103A381F0BD02233B
:10207000BF0803FA07F7A389084D9BB223EA0703B9
:1020800087190CEB470CA3810CF1040345F82C10C5
:1020900045F82320A5E700BF0300100010530020DF
:1020A0002B4B98423CD0B0F1804F3BD0A3F57C4302
:1020B000984239D003F58063984237D003F58063A6
:1020C000984235D003F58063984233D003F580639E
:1020D000984231D003F5704398422FD003F57053E6
:1020E00098422DD003F5806398422BD003F580638E
:1020F000984229D0A3F59833984227D003F58063FE
:10210000984207D003F58063984208BF0D2202D0A1
:10211000002070470C220F4B03EBC2031879704765
:102120000022F8E70122F6E70222F4E70322F2E7B1
:102130000422F0E70522EEE70622ECE70722EAE7B1
:102140000822E8E70922E6E70A22E4E70B22E2E7B1
:102150000000014058D303082DE9F047B0F90850BA
:102160000D81EDB2442D92B00C4600F0B3820646CC
:1021700042D9812D00F0EF8100F29580542D00F0BE
:10218000C88040F2D5816E2D00F07282802D40F023
:102190001181B54B93F8009009F1020919F0FF097C
:1021A00000F09480B14BB24FB24EDFF804A39944D3
:1021B00003F101080A2516E0322D00F0BA82A5F1DC
:1021C0003C00C0B2132840F2BC8200232268511C9C
:1021D000216015702268C84502F101012160137069
:1021E00074D018F8015B0A2DE6D1BAF80030FF2B45
:1021F000A8BFFF23DBB2E9E7052D00F059821ED806
:10220000022D7ED040F28181032D00F02782042D23
:1022100040F0D0802A4698492046F6F7DFFD00219D
:102220002046F6F723FE22680221531C0125236075
:1022300028462B461170638112B0BDE8F087242D2B
:102240005DD040F2F380282D00F0CD81382D40F094
:10225000B1800A68894B0125511C216015702268E4
:10226000052150192060117022680A215019206040
:1022700011702268002150192060117022681978AD
:10228000501920601170226859785019206011701F
:1022900022689978531923602B4611702846638170
:1022A00012B0BDE8F087A02D17D040F20381B82D01
:1022B00000F0D281FE2D7DD1714D05F1080635F873
:1022C000021B2046F6F7D2FDB542F8D101252B4678
:1022D0002846638112B0BDE8F0876A4B084619684A
:1022E000F6F7ACFD684B20461968F6F7A7FD674B7B
:1022F000196820460125F6F7A1FD2B46E8E7644B57
:10230000F6E70422634920460125F6F767FD2B46D0
:10231000C4E70B68604A614F581C11212060197096
:1023200023681278591C21601A70236897F85B2083
:10233000591C21601A70236897F85A20591C216093
:102340001A70B7F856102046F6F790FD0021204687
:10235000F6F78CFDB7F858102046F6F787FDBD1E3E
:1023600007F1480635F8021F2046F6F77FFDAE421A
:10237000F8D122684A4B0C21501C20605D18117066
:10238000226813F8011F501CAB4220601170F7D176
:1023900023680222591C21601A70B7F85C1020468D
:1023A000F6F764FD0125B7F85E102046F6F75EFDEE
:1023B0002B4673E721462846FDF75EFF002885D1AE
:1023C000742D00F0BB80772D0CD1336872689A426F
:1023D0001BBF5A1C326001461978324A204621F050
:1023E0006DFA73E7762D00F07D81392D376800F0A6
:1023F0006A8200F20182212D01F07C82292D40F0B9
:10240000A3827B1C33603B780A2B01F09882502B0F
:1024100041F04A803046F6F7CFFC234F38803046F3
:10242000F6F7CAFC012578802B4637E7202DC1D16D
:102430000B681E4D591C6A7821601A7023682A782F
:10244000591C21601A702368AA78591C21601A70DF
:1024500029892046F6F70AFD23686A79591C21600C
:102460001A702268A979E0E6F48A002094AA030889
:1024700067666666302B0020BA90002099A800207D
:10248000FC580020107AFF1F147AFF1F187AFF1FD4
:1024900024AA0020C4DA0308C4900020DEA700208C
:1024A00027A80020BD2B0308182B00202C55002046
:1024B000582B0020822D7FF47DAF0B68B94ABA4DAE
:1024C0001178BA4A581C2060197011892046F6F715
:1024D000CDFCB74B22681B88FF2B02F10101A8BF7E
:1024E000FF2321601370A96881F3100189B220468F
:1024F000F6F7BCFC296801F30F0189B22046F6F714
:10250000B5FCAC4B226819788FE6012D7FF452AFF1
:102510000B680022591C21601A7023685A1C226023
:102520001D7022682421531C23602B461170B5E6D0
:10253000522D7FF43FAF2268002176E6336872683F
:102540009A421BBF5A1C3260014619789A4A2046AB
:1025500021F0B4F9BAE6994B1E78033616F0FF065F
:102560003FF4B4AE964B974F1E4403F101094FF070
:102570000A0820E0B8F1500F00F0E180B8F1320F06
:1025800000F0F480A8F13C00C0B2132840F2F180C2
:102590000025294623685A1C2260204683F80080C3
:1025A000F6F764FC29462046F6F760FCB1453FF497
:1025B0008DAE19F8018BB8F10A0FDBD1824B9D6803
:1025C000196805EB85054FF6FF736D009D42A8BFA6
:1025D0001D469942A8BF194625EAE57521EAE17131
:1025E000ADB289B2D6E70B68DFF80882774E591C86
:1025F000022221601A70236806275A1C22601F706D
:1026000023680A22591C21601A70236801255A196F
:1026100022601D70B8F800102046F6F727FCB8F8C5
:1026200002102046F6F722FC23685A1922601F7018
:1026300023685022591921601A7023680022591901
:1026400021601A7031882046F6F710FC7188204608
:10265000F6F70CFC2B4621E65D4B49E60B685A1C4D
:102660000A601D700B680222591C21601A7062E713
:102670004F4B0A681B884C4DFF2BA8BFFF23511CF2
:1026800021601370A96881F3100189B22046F6F722
:10269000EDFB504B20461988F6F7E8FB296801F35B
:1026A0000F0189B220460125F6F7E0FB2B46F5E540
:1026B0000B2249492046F6F791FB0822474920465C
:1026C000F6F78CFB0125072245492046F6F786FBE5
:1026D0002B46E3E5002A3FF4F9AD424B1360012598
:1026E0002B46DBE533685A1C32601B78002B01F067
:1026F0002181102B07BF3C4A92E82200054629465B
:102700002268501C206013702046F6F797FB29467C
:102710002046F6F793FB354B20461968F6F78EFBFB
:1027200020460021F6F7A2FB00212046F6F79EFB8B
:1027300001E73388FF2BA8BFFF23DBB246E52C4B14
:102740003DE716F09DFA00283FF43FAD03780A2BD1
:1027500025D8B0F9023087FB0312DB17C3EBA203C5
:102760009BB2FF2BA8BFFF23DBB22FE597E8220027
:1027700027E716F085FA00283FF40AAF03780A2B02
:102780003FF606AFB0F90430B0F9061003EB83034F
:1027900083F3500521EAE171ADB289B2FAE6002374
:1027A000E2E700BFD6590020B85400202C55002085
:1027B000C0590020B58C002065370308F48A00203A
:1027C000A4AA0308282B0020E42A0020182B0020AC
:1027D000E44C0020B28C0020CCDA0308D8DA0308DD
:1027E000E4DA0308BD010108D02A0020E027002018
:1027F0001C2B0020E4510020552D76D0572D40F0A1
:10280000A3807B1C336017F8378B0DF1070201336F
:10281000336013F8011C02F8011F9F42F7D1DFF863
:10282000209199F80050002DFDD1DFF818A1012664
:10283000082089F8006021F073FFDAF80000FAF749
:1028400081FB3D4B28461E7021F0FCFE284621F0FE
:10285000F9FE092021F0F6FE404621F0F3FE02AF1A
:102860003D460DF13E08EE1BF6B20A2021F0EAFECD
:10287000304621F0E7FE15F8016B0B2021F0E2FE57
:10288000304621F0DFFE0020FAF736F8A845EAD1FD
:10289000082021F0D7FEA02021F0D4FEA02021F0B6
:1028A000D1FE002021F0CEFE10F02006F6D1DAF89D
:1028B0000000FAF74DFB0125042021F031FF89F8D3
:1028C00000602B46EAE47B1C33603B780A2B01F066
:1028D0003C803046F6F77CFA3046F6F779FA012567
:1028E0003046F6F775FA2B46D8E47B1C336097F830
:1028F0000080B8F1FF0F01F09D80B8F1FE0F01F0EC
:1029000033803046F6F758FA96E80C009B1A002BF5
:1029100007DD531C336013781BB9B8F10B0F41F27C
:102920007E80B8F1240F00F28182044B012523F848
:1029300018002B46B2E400BF365E0020DEA7002060
:102940002D5E0020A890002072680B3DD31BEF2D58
:1029500000F26C8201A151F825F000BFE9330108B3
:102960002D2E01082D2E01082D2E01082D2E0108D7
:102970002D2E01082D2E01082D2E01082D2E0108C7
:102980002D2E01082D2E01082D2E01082D2E0108B7
:102990002D2E01082D2E01082D2E01082D2E0108A7
:1029A0002D2E01082D2E01082D2E01082D2E010897
:1029B0002D2E01082D2E01082D2E01089933010816
:1029C0002D2E01083F3301082D2E01081D3301086B
:1029D0002D2E01082D2E01082D2E0108F53201089B
:1029E0002D2E01089B3201082D2E010869320108A5
:1029F0002D2E0108CF3801082D2E01089538010829
:102A00002D2E01083B3501082D2E0108EF34010859
:102A10002D2E01082D2E01082D2E01082D2E010826
:102A2000CD2201082D2E0108D33401082D2E0108D6
:102A30002D2E0108B93401082D2E01085F3401083C
:102A40002D2E01082D2E01082D2E01082D2E0108F6
:102A50002D2E01082D2E01082D2E01082D2E0108E6
:102A60001F3401082D2E01084D3701082D2E0108B5
:102A70002D2E01080D3701082D2E01082D2E0108DD
:102A80002D2E01082D2E01082D2E01082D2E0108B6
:102A90002D2E0108413601082D2E01088F35010821
:102AA0002D2E01082B3801082D2E01089B37010817
:102AB0002D2E0108A73801084B3201082D2E0108E0
:102AC0002D2E01082D2E01082D2E01082D2E010876
:102AD0002D2E01082D2E01082D2E01082D2E010866
:102AE0002D2E01082D2E01082D2E01082D2E010856
:102AF0002D2E01082D2E01082D2E01082D2E010846
:102B00002D2E01082D2E01082D2E01082D2E010835
:102B10002D2E01082D2E01082D2E01082D2E010825
:102B20002D2E01082D2E01082D2E01082D2E010815
:102B30002D2E01082D2E01082D2E01082D2E010805
:102B40002D2E01082D2E01082D2E01082D2E0108F5
:102B50002D2E01082D2E01082D2E01082D2E0108E5
:102B60002D2E01082D2E01082D2E01082D2E0108D5
:102B70002D2E01082D2E01082D2E01082D2E0108C5
:102B80002D2E01082D2E01082D2E01082D2E0108B5
:102B90002D2E01082D2E01082D2E01082D2E0108A5
:102BA0002D2E01082D2E01082D2E01082D2E010895
:102BB0002D2E01082D2E01082D2E01082D2E010885
:102BC0002D2E01082D2E01082D2E01082D2E010875
:102BD0002D2E01082D2E01082D2E01082D2E010865
:102BE0002D2E01082D2E01082D2E01082D2E010855
:102BF0002D2E01082D2E01082D2E01082D2E010845
:102C00002D2E01082D2E01082D2E0108213201083C
:102C10002D2E01080B3201082D2E01082D2E010842
:102C20002D2E01082D2E01082D2E01082D2E010814
:102C30002D2E01082D2E01082D2E01082D2E010804
:102C40002D2E01082D2E01082D2E01082D2E0108F4
:102C5000B13101085F310108273101082D2E01082B
:102C60008B30010871300108053001082D2E010854
:102C7000EB2F0108852F01085D2F01084B2F01085C
:102C8000F12E01082D2E0108C32E01082D2E01085A
:102C90002D2E0108A12E0108732E01085F2E0108B8
:102CA000372E01080F2E0108ED2D0108C12D010856
:102CB000A92D01082D2E01082D2E01082D2E010809
:102CC0002D2E01082D2E01082D2E01082D2E010874
:102CD0002D2E01082D2E01082D2E01082D2E010864
:102CE0002D2E01082D2E01082D2E01088F2D0108F3
:102CF0002D2E01082D2E0108372D01082D2E01083B
:102D00002D2E01082D2E01082D2E01082D2E010833
:102D10002D2E01082D2E01081D2D0108C04B1B78FA
:102D2000DB0700F183800125FEF73AFBFEF7EAFBA3
:102D30002B46FFF7B3BA7B1C33603B780F2B75D85B
:102D4000BA1C3260C3EBC303B64A7978D154F91C7C
:102D500031601344BA785A703A1D3260FA789A702A
:102D60007A1D32603A79DA70BA1D32607A791A7156
:102D7000FA1D3260BA795A7107F108023260FA79A5
:102D80009A7101250DF0FEFB2B46FFF787BA3046FE
:102D9000F6F712F8A44FF8813046F6F70DF8012542
:102DA000B8812B46FFF77ABA3046F6F705F89F4A06
:102DB00000EB80004300012513802B46FFF76EBA1D
:102DC0003A467B1C33609A4B12F8021B1970326032
:102DD0007A785A70FA1C3260BA789A703A1D32606A
:102DE000FA78DA7001252B46FFF758BA3046F5F726
:102DF000E3FF904F38823046F5F7DEFF78823046A9
:102E0000F5F7DAFF0125B8822B46FFF747BA3B46B4
:102E10007A1C326013F8020B3360FB1C7978336044
:102E2000BA7815F0F9F800287FF450AA4FF0FF3572
:102E30002B46FFF733BA3B467A1C32607E4A13F8C2
:102E4000021B11703360784A7B789370FB1C3360EF
:102E5000764BBA789A7001252B46FFF71FBA774B4D
:102E6000774918684E22012525F0C0F92B46FFF757
:102E700015BA3A467B1C3360724B12F8021B19706C
:102E800032607A785A70FA1C3260BA789A7030469A
:102E9000F5F792FF6C4B0125D8802B46FFF7FEB962
:102EA0003046F5F789FF684F38803046F5F784FFE4
:102EB00078803046F5F780FF0125B8802B46FFF774
:102EC000EDB9DFF8A48198F80030002B3FF4FEA99B
:102ED0005E4F00253046F5F76FFF0FF091F898F838
:102EE0000030A7EC010A01359D42F3DBFFF7EEB994
:102EF0000D2B9BD17B1C33603D78072D96D8DFF8D6
:102F00006C8130460C27F5F757FF07FB05F708EBF8
:102F10000705A8803046F5F74FFFE8803046F5F703
:102F20004BFF336828811A46591C316012F8021B86
:102F3000A97232605B78EB72304624F0E4FF012521
:102F400048F807002B46FFF7A9B93046F5F734FFDC
:102F50003F4B012518802B46FFF7A0B97B1C33603F
:102F60003878060600F10E862D4B1B78DD073FF5FD
:102F7000ADA9032828BF00200125FEF7F5F92B464F
:102F8000FFF78CB97B1C3360304697F8009024F033
:102F9000BAFF8046304624F0B6FF0546304624F09E
:102FA000B2FF07463046F5F707FF3046F5F704FF56
:102FB0003046F5F70DFFB9F1000F00F0CE85B9F1FD
:102FC000100F7FF483A9234BC3F800805D600FB11D
:102FD000214B1F602149224B0222081F01251A7034
:102FE00018F0FEFA2B46FFF759B90D4B1B78D8079E
:102FF0003FF56CA90125FEF76BFCFEF783FA2B4623
:10300000FFF74CB9064B1B78DA073FF55FA9154A65
:103010001378012543F0040313702B46FFF73EB9E4
:10302000045C002058460020F45100200452002087
:103030007C62002098920020848E0020A4A80020AA
:1030400034B10308EC510020384F0020904E00208E
:10305000708E0020D02A0020E0270020D42A0020F3
:103060005A8D002044550020F48A00206445002039
:10307000B94B1B78D9073FF529A9B84B4FF4C87253
:1030800001251A802B46FFF709B9092B7FF7CEAE31
:10309000DFF800833B467A1CD8F80050326013F802
:1030A000022B2A7033607B78AB70FB1C3360BB78DB
:1030B000642BA8BF64233A1D6B713260FB78642BCC
:1030C000A8BF64237A1DAB7132603B79EB71BB1DE5
:1030D00033607B79642BA8BF6423FA1D2B723260A6
:1030E000BB79EB7007F108033360FB792B71304635
:1030F000F5F762FE726833686881D11A00290CDD29
:10310000591CD8F800003160521A002A197841720F
:1031100003DD9A1C32605B784370012523F076FC56
:103120002B46FFF7BBB88E4B1868FB1C02462137B5
:10313000991E316013F8031C1170591E316013F889
:10314000021C5170336013F8011C917003339F42CD
:1031500002F10302ECD10EF01FFEFFF7B7B87B1CA3
:1031600033603B787F4A002B00F08684137843F06D
:103170000203B91C13707C4D31607B782B7530468F
:1031800024F0C1FE2860304624F0BDFE6860304661
:10319000F5F712FE28813046F5F70EFE734AE881F6
:1031A0001378012543F0020313702B46FFF776B81E
:1031B000C3F34705122D3FF639AEB5B112AB0DF191
:1031C000060903EB4507C846423F3046F5F7F4FDD4
:1031D00028F8020F4745F8D1654B39F8022F23F83C
:1031E000022FC845F9D1112D09D8624A6B00023B64
:1031F00013440021223223F8021F9A42FBD15E4A77
:1032000001231D461370FFF749B85C4F0023304679
:103210003B6024F078FE012538602B46FFF73EB86E
:103220003B467A1C326013F8025B3360FB1C7878F3
:103230003360B978002D00F03B84012D7FF446A85F
:1032400008F008FA2B46FFF729B8434B1B7813F018
:1032500001017FF4EBAD7B1C33603878012524F04D
:1032600081FE2B46FFF71AB8454D05F14007304661
:10327000F5F7A2FD3368A5F88000591C1A463160A5
:1032800012F8021B85F8821032605B7885F8833073
:103290000435BD42EBD1FFF719B87B1C394D3360C3
:1032A0003B782B723046F5F787FDA8833046F5F75B
:1032B00083FD28833046F5F77FFD32686883531C11
:1032C00033601278EA747268D31A032B00F37684A1
:1032D0003368D11A052900F36084D21A002A7EF7D8
:1032E000F5AF5A1C32601B7885F8213001252B463A
:1032F000FEF7D4BF7B1C3360234938780870D21A9C
:10330000002A7EF7E3AFBB1C33607B78003318BF25
:10331000012301254B702B46FEF7C0BF3046F5F761
:103320004BFD1A4F38603046F5F746FD7860304661
:10333000F5F742FD0125B8602B46FEF7AFBF144FED
:1033400000233B60304624F0DEFD3B68012503434B
:103350003B602B46FEF7A2BF045C0020DEAB0020E2
:10336000A4A800204455002048550020588D002076
:10337000EA420020EC42002010430020E44C0020F0
:10338000945600201C9000201C520020E041002098
:1033900024AA0020C0AB00207B1C33603D78132D95
:1033A0003FF644ADBB1C3360787820F0C1FA0028AA
:1033B0003FF43CAD934B027803F82520FA1C3260B1
:1033C00003EB8503BA785A703A1D3260FA789A7026
:1033D0007A1D32608C493A79DA700868012524F048
:1033E000C5FE2B46FEF75ABF884A102B4FF000014E
:1033F00028BF1023116051609160D1601174002BBF
:103400003EF464AF3168013A0B440131316011F888
:10341000010C02F8010F8B42F7D1FEF757BF3B4674
:103420007A1C7B4D326013F8022B2A7133607B7853
:103430006B713046F5F7C0FC336828805A1C326047
:103440001B78AB713046F5F7B7FC336868805A1CBF
:1034500032601B78EB7101252B46FEF71FBF7B1CEA
:1034600033606C4B3A78DFF8D0811A700023C8F8CB
:103470000030304624F047FD3268D8F80030664905
:10348000664D0343501CC8F80030306013780B724F
:103490003046F5F791FC28603046F5F78DFC686002
:1034A0003046F5F789FCA8603046F5F785FC3046D4
:1034B000F5F782FCFEF70ABF594B07F10802013706
:1034C000376017F8011C03F8011F9742F7D1FEF788
:1034D000FDBE3B467A1C3260524A13F8021B9170C3
:1034E00033607B78537001252B46FEF7D7BE072249
:1034F000B3FBF2F2C2EBC2055B1B7FF497ACD2B216
:1035000002F1FF385FFA88F8002A3EF4DFAEDFF8F8
:10351000189108F101081D467B1C3360424B97F956
:103520000010002793F902208A4203F1080300F0FB
:1035300051820137062FF5D178E47B1C33603B784C
:103540000E2B3FF673ACBA1C3260787803283FF636
:103550006DAC3649062202FB03F28B18FD1C587134
:103560003560B87888543A1D3260FA785A707A1DFE
:1035700032603A799A70BA1D32607A79DA70FA1D3F
:103580003260BA791A7101252B46FEF787BE3B4699
:103590007A1C3260DFF8A48013F8022B88F802202E
:1035A0003360234A7B781370FB1C3360214DBB785A
:1035B0002B713B1D3360FB78092BA8BF09233046D4
:1035C000AB70F5F7F9FB336872682880D11A0129CE
:1035D00005DD3046F5F7F0FB33687268E8819A4202
:1035E00040F0B282FDF7E6FE336872689A423EF41C
:1035F0006DAE5A1C32601B78EB7001252B46FEF72E
:103600004DBE00BF20520020A4A80020D0510020B1
:10361000504F00201C5200201C900020E041002050
:103620001B90002010520020D0900020F04C002071
:10363000E85100209892002024AA0020848E0020C7
:103640003046F5F7B9FB054618F0D8F8FF283EF4E8
:103650003DAE3F2D00F261820DF14808002308F8CD
:10366000403DEF0841460DF107008DF80730013766
:1036700018F0A4F89DF80730FFB205F00705BB422B
:1036800005F1010503D19DF80830AB4203D029466E
:10369000384618F09FF833687268D21A012A7EF70C
:1036A00015AE5A1C12A8326000221D7800F8412D78
:1036B00018F078F89DF80730AB420AD0B44B1B687D
:1036C0003BB19A79AA4204D31B681B690BB1284607
:1036D000984733685A1C3260404600221D788DF8A6
:1036E000082018F053F89DF80830AB423EF4EEADD8
:1036F000A74B1B68002B3EF4E9AD1B685B69002BF0
:103700003EF4E4AD28469847FEF7E0BDA14B1B7898
:10371000012B3EF6DBAD39467B1C3360DFF8AC8213
:1037200011F8023B88F802303160FB1C7878336076
:10373000D31A012BB97840F3A4813046F5F73CFB4E
:103740000125A8F800002B46FEF7A8BD7B1C3360BE
:1037500097F80080B8F1110F3FF668ABBB1C3360DF
:103760008D4D7B7805F818303046F5F725FB40F68F
:10377000CA039842A8BF184640F2EE23984205EBD0
:103780004801B8BF18460125A0F2EE222B461920A9
:1037900092FBF0F24A70FEF781BD3046F5F70CFB64
:1037A0003046F5F709FB3046F5F706FB3046F5F7EE
:1037B0000FFB3368794D1946581C2A68306011F8A0
:1037C000020B82F82C003160597882F83610D91C2F
:1037D00031609B7882F837303046F5F7F9FA304699
:1037E000F5F7F6FA3046F5F7F3FA30462F68F5F7B5
:1037F000E3FA788730462F68F5F7DEFA33687268A7
:103800003887D11A01290ADD591C2A6831601B78D2
:1038100082F82E303046F5F7DBFA33687268D31A37
:10382000032B00F33A81286895E47B1C33605B4DE1
:10383000DFF89C813B7888F8053030462F68F5F733
:10384000BBFA388430462F68F5F7B6FA72683368E9
:10385000F883D11A072900F34981D11A032900F30B
:103860003881D21A002A05DD591C2A6831601B787C
:1038700082F82630FDF79EFD1CF06EFD484B1B685C
:10388000002B00F01B81286801250CF00DFF2B4652
:10389000FEF704BD7B1C3360424B3A785A75012514
:1038A0002B46FEF7FBBC3B467A1C32603E4A13F8BF
:1038B000021BD17033603D4A7B785371FB1C33602F
:1038C0003B4BBA78DA7001252B46FEF7E7BC7A1C31
:1038D00032603D781F2D3FF6A9AA052B7FF4A6AADA
:1038E000304624F010FB334B43F825001BF0F4FC6A
:1038F000FEF7ECBC3B467A1C32602F4D13F8022BCE
:103900006A7033607B782B70FB1C3360BB78AB70C4
:103910003046F5F751FA33682881591C1A46316050
:1039200012F8021B697132605B78AB7101252B467E
:10393000FEF7B4BC214A92E82200FEF7E1BE304611
:10394000F5F73AFA1E4FFEF769BDBB1C33601D4BFD
:103950007A781A70FA1C3260BA785A703A1D32605E
:10396000FA789A70FEF7B2BCBB1C33607D78022DEA
:103970003FF65CAA3046F5F71FFA134B03EB4503FD
:103980004FF0FF35A3F85C002B46FEF787BC00BF65
:1039900068640020EFA90020404C0020A4A800206B
:1039A000185200201C900020F45100208C58002058
:1039B00004520020945600202C5500209C8D00209D
:1039C000E451002099A80020DEA70020F2A90020E1
:1039D000848E002009EBC70A30468AF80210F5F7FA
:1039E000EBF9336829F837001A46591C316012F890
:1039F000021B8AF8031032605A788AF80420DA1C15
:103A000032609A788AF806201F1D37600135DB780E
:103A10008AF80530A8457FF47FADFEF757BC774B99
:103A20000030984418BF0120012588F84A002B4631
:103A3000FEF734BCBB1C3360714B7A781A70FB1CE8
:103A40003360DFF8B881BB7888F85B303B1D3360AA
:103A5000FB7888F85A303046F5F7AEF9A8F85600EA
:103A60003046F5F7A9F93046F5F7A6F90125A8F88B
:103A700058002B46FEF712BC137803F0FD03FFF746
:103A800078BB604B1A88012512FB00F22B4692FB93
:103A9000F1F2A8F80020FEF701BC30462F68F5F7D8
:103AA0008BF9788630462E68F5F786F9B086BAE647
:103AB00001250CF0B3FF2B46FEF7F0BB52485349EB
:103AC000534A544B036001250B6013602B46FEF7ED
:103AD000E5BB3046F5F770F9A8F80E003046F5F76B
:103AE0006BF933687268A8F81000BAE63046F5F74B
:103AF00063F9A8F80A003046F5F75EF9A8F80C005B
:103B000030462F68F5F758F9788430462F68F5F776
:103B100053F933687268B8849FE60DF1080840468F
:103B200017F028FEBDF80830AB423FF4B4AD3A4B75
:103B30001B68002B3FF4AFAD1B689B69002B3FF463
:103B4000AAAD28469847A6E55A1C32601B78003378
:103B500018BF012388F8073044E5304B1020C3F824
:103B600000805D6009F068FE2D4A137843F0010380
:103B70001370002F3EF4AAAB2A4B01251F602B4681
:103B8000FEF78CBB00F07F00032828BF0020012532
:103B900007F07CFD2B46FEF781BB5A1C32601B7878
:103BA000EB72304624F0AFF93368E8605A1C32609B
:103BB0001B782B7433687268FFF78FBB3046F5F7BC
:103BC000FBF8A8843046F5F7F7F833687268E884A4
:103BD000D11A03297FF77DAB1A46591C316012F8C0
:103BE000021BA97732605B7885F820303046F5F704
:103BF000E3F8336872686884FFF76BBBDEA70020C8
:103C0000C49000205A500020D046002024470020B5
:103C1000244B00206D820008686400209C8D0020E9
:103C200044550020E02700202DE9F04F2DED0A8BB0
:103C30003C4B1B7895B0012B089001F08B863A4CD9
:103C400094F80021002A41F0CB80072B374D01F07A
:103C50007C864FF0000B6B6834489847002800F0D2
:103C60006881B5F8B470002285F85520002F40F027
:103C70004387B5F93E00AA6AB5F93C60696AB5F9AF
:103C80004030DFF8B4A0821AE86A6A63711A1B1A1E
:103C90002963274895F85610AB6319F0FBFADAF858
:103CA0000030990040F1F080D5ED0D5AD5ED0C7A39
:103CB000204A94ED676AD4ED686A94ED697AD4F885
:103CC000A8311268B8EEE58AD5ED0E5AF8EEE77A1B
:103CD000F8EEE58A013377EE867A38EE268A78EEBA
:103CE000878A9342C4ED677A84ED688AC4ED698A55
:103CF000C4F8A83101F0E4830A4B1F78142F02F0B6
:103D0000A0870023D4F8B0610493062E00F2AF80A0
:103D1000DFE816F0D2162F16F41443161400C0155F
:103D2000581500BFF8580020E42700200498002010
:103D300034980020D0730020A88E0020D94B1A7828
:103D4000D4F8B4E1DFF8D0C39FEDD77A4FEACE00C4
:103D50000CEB000383ED007A002A7DD0D349B0EE4E
:103D6000476AF0EE476A0023F1EC017A013367EE0F
:103D7000A77A05EE903AB4EEE77AF1EE10FAF8EE93
:103D8000E55AB8BFB0EE677A934276EEA76AA7EE1F
:103D9000A56AE9D1F5EEC06A0CEB0003F1EE10FA6A
:103DA00083ED007A58DDC6EE265AC14BC14A12880F
:103DB000F7EE007A75EEE75AD3ED007A65EEA77A52
:103DC000FDEEE77A17EE903A812B43F33986934262
:103DD000A8BF134607EE903AF8EEE77AB64B00EB31
:103DE0000E0103EB810393ED057AD3ED003A93EDD9
:103DF000066A93ED014AD3ED046AD3ED034A93EDCD
:103E0000025AA3EEA77AA4EE276A66EEC76AA7EE67
:103E1000646ABDEEC77AE5EE276A17EE101A8129AB
:103E200083ED056AC3ED066A43F307868A42A8BF9D
:103E30000A4607EE902AF8EEE77AFCEEE77ACDED37
:103E4000057ABDF814300CEB00029380BEF1000F30
:103E500002D1132F04F08D82152F42F0A484604408
:103E6000DFF86882838828F81E30D4F8B061934B5D
:103E7000013683FB06239A19F317C3EBA203C3EBA6
:103E8000C303F61AC4F8B0618D4B1B78002B01F008
:103E9000B4808C4EDFF8849206F2DC6800278A4BEF
:103EA000D5ED087A1B78172B01F09E8396ED007AEA
:103EB000B8EEC78A082B28EE278A08D1B0EE480A48
:103EC000049324F09DFB814B23F81700049BDAF840
:103ED000002092000BD5002F04F07785B0EE480A41
:103EE000D5F8783708F170009847B0EE408AB0EE08
:103EF000480AD5F89836A8F170009847D5F80837E1
:103F000040469847704B1B78032BB0EE408A01F077
:103F10007983D6F85C06D5F8B830B0EE480A9847F1
:103F20000137032F08F12408A9EC010A06F1040661
:103F3000B5D1654B93F80090B9F1070F00F0998661
:103F400094F8C031002B40F0A186614B5B79002BC7
:103F500040F0CC8501235C4A84F8C0311278072AEE
:103F600002F0A18000230B935A4B94ED729A93EDCB
:103F7000007A594BDFF8A881D3F800A0574B05937E
:103F8000F7EE007A37EEC9BA554B07932BEE07BA16
:103F9000544B0993544B0693B4EEE7BA08F1680307
:103FA0000025F1EE10FA0A93D4ED71BA4F4BDFF809
:103FB00074B1DFED4F8A9FED4FAADFED3BAADFED35
:103FC0004E9ADFF864914D4F049388BFB0EE67BA04
:103FD0002E464B4B98ED008A2B44D3ED007AF5EE3C
:103FE000407AF1EE10FA17D0464B2B44D3ED006A1D
:103FF00038EE667AB0EEC76AF4EEC67AF1EE10FAE1
:1040000008D5B5EEC07AF1EE10FACCBF37EEA68A2D
:1040100036EEE78A83ED008A059B1A88930700F045
:104020008780022E00F08480374B9AF82E1033F9E7
:10403000163007EE103A0A9B07EE901A2B44F8EE62
:10404000E76AB8EEC77AD3ED007A4B42A6EEA77ABC
:10405000700007EE903AF8EEE77AB4EEE77AF1EE08
:1040600010FA0AD407EE901AF8EE677AF4EEC77ADF
:10407000F1EE10FA88BFF0EE477A244B244903444E
:10408000085EB3F90C30C01A07EE100AB8EEC77A12
:10409000D007E7EE687A40F101861E4B93ED008A67
:1040A00044E000BFD673002000000000E427002099
:1040B000D8730020D47300200C76002093244992FA
:1040C000C973002034980020F8580020FC580020C4
:1040D000848E00205C4E0020A4A80020308D00209B
:1040E000A4000020045C0020988E0020B84F00201F
:1040F000CDCCCC3DAE47813F0000C842C44F00202C
:10410000504E0020B029002074290020F4510020D6
:1041100024550020384E0020F47500209C8E00208D
:10412000E8280020CC460020D04F002027EE888AC7
:10413000069B94F8D8212B44D3ED01CA38EE6CCA03
:10414000002A3DD0D24BD4F8DC2108991B688A1A8A
:104150009A4235DD9AF84830022B02F01A80022E7E
:1041600004F0B783CB4B1B68990740F12D87CA4BEE
:10417000CA49DFF890E331F916C09EED008ADFF8F6
:1041800088E3C7ED00AA03EB460028EE288AB0F9C1
:104190000C00A0EB0C0007EE900AF8EEE77ADEF8D0
:1041A000000027EE888A904238EE6CCAC1F23A814C
:1041B000F7EE007AB4EEE79AF1EE10FA01F1098118
:1041C000B74B2B4493ED000A049B2BEE800A022E82
:1041D00020EE0C0AA3EC010A049304F0A283079BCF
:1041E0009BED007AD3ED007AAE4BD7ED006A93EDEC
:1041F000006AAD4B67EE277A2B4427EE8B7AD3ED1E
:10420000007A67EE277AF0EE665AE7EE8C5AB1EE46
:10421000467AF4EEC75AF1EE10FA08D4F4EEC65A14
:10422000F1EE10FA8CBFB0EE467AB0EE657A94EDFE
:10423000726AF7EE007AB4EEE76AF1EE10FAACBFFC
:104240000123002343B1F0EEE66AF0EEC77AF4EE04
:10425000E67AF1EE10FA01D587ED007A022E04F02D
:104260001983924A924B52F826001B68B0EE6C0AF2
:104270009847904A904B52F826001B6898479AF846
:10428000373023B1059B1B88002B00F07185B0EE01
:104290006A8A8A4B9BED007A38EE400A2B4493EDF4
:1042A000008A83ED000A9AF8483030EE480AC0EEE2
:1042B000077A2BB3099B1B78DB0721D5B7EE007A71
:1042C000B4EEC79AF1EE10FA04DB94F8D831002B63
:1042D00000F06787D4F8DC31089AD31A6C4A126868
:1042E0009A420DDD764B93ED007AB0EECCCAB4EE77
:1042F000C7CAF1EE10FA41F1B180002384F8D83139
:10430000704B94F8E8212B4493ED007A2BEE877ADA
:1043100067EE277AC9ED007A32B9049BC7ED00AA8F
:1043200043ED01AAC9ED00AA0136032E08F10408E5
:1043300009F1040907F1040705F104057FF449AE0A
:10434000614B1B78072B01F04F83012B01F09886FE
:10435000002794F8F031002B40F000865B4A5C4B5C
:1043600010681B6810F4805A93F82C3040F06E8669
:10437000584A594992ED006A498B584A84ED806A3F
:1043800092ED007A564A84ED817A07EE901AF8EEA3
:10439000E76AD2ED037A534A84ED7E6A37EE467AB5
:1043A00077EEE67AD2ED006A84ED7D7A012284F818
:1043B0000822C7EEA65A4C494C4A91ED005A4C4986
:1043C0009FED4C6A91ED004A4B49DFED4C6AD1ED0F
:1043D000004A92ED007A35EE045AF7EE007AF4EED8
:1043E000E75A35EE245AF1EE10FA88BFF0EE675A1C
:1043F00025EE065AF4EEE65AB1EE476AF1EE10FAEF
:10440000B4EEC65AB8BFF0EE665AF1EE10FAC4ED3B
:10441000835A01F1E280B4EEC75AF1EE10FA88BF78
:10442000B0EE475A304ADFED336AD2ED017A304AB6
:1044300092ED014A304A77EE847AD2ED014A77EE66
:10444000A47A67EEA67AB4EEE76AF1EE10FA08DC19
:10445000B4EEE77AF1EE10FA8CBFB0EE676AB0EE18
:10446000476A214ADFED236AD2ED027A204AD2ED73
:10447000024A234A77EEA47A92ED007A67EEA67A92
:10448000B1EE473AF4EEC37AF1EE10FA47D43DE0CC
:10449000644E002040550020F45100202455002097
:1044A0000C4E0020804E0020184E0020D4460020E4
:1044B000D04600202847002024470020C42900209F
:1044C000704E0020244E0020F8580020A88E0020B6
:1044D000A4A80020605000201C900020C45100209F
:1044E000D8590020404F0020B84F0020844E0020B3
:1044F000C44F00206F12833AD04F0020000000000C
:10450000884E0020384E0020604E0020F4EEC77A1E
:10451000F1EE10FA8CBFB0EE473AB0EE673AF04ACF
:1045200052780AB9B1EE433A002B41F08583F7EE99
:10453000003AEC4D2A78002A02F0FE86EA4BDFEDC5
:10454000EB7AD3ED024AD3ED016A93ED037A66EE7E
:10455000244AE5EE264AE3EE074A63EEA44AF4EE67
:10456000E74AF1EE10FAB4BFB0EE674AB0EE644A23
:1045700098BFF0EE647A012ACDED0C4A02F0018773
:1045800093ED067AD3ED052AD3ED076A26EE077A76
:10459000A5EE227AA3EE267A23EE877AB4EEE77AA6
:1045A000F1EE10FAB4EEC47A8CBFF0EE676AF0EE6A
:1045B000476AF1EE10FA88BFF0EE676AB4BFF0EE1A
:1045C000447AF0EE477A022A8DED0D7A00F0DE8013
:1045D00093ED0A7AD3ED092A93ED0B4A26EE077A7A
:1045E000A5EE227AA3EE047A23EE877AB4EEE67A79
:1045F000F1EE10FAB4EEE77A8CBFB0EE664AB0EE98
:10460000474AF1EE10FA98BFF0EE446AA8BFF0EE08
:10461000477A032A8DED0E7A00F0B88093ED0E7A7A
:10462000D3ED0D2A93ED0F4A26EE077AA5EE227AF6
:10463000A3EE047A23EE877AB4EEE67AF1EE10FA6E
:10464000B4EEE77A8CBFB0EE664AB0EE474AF1EEC0
:1046500010FA98BFF0EE446AA8BFF0EE477A042A39
:104660008DED0F7A00F0928093ED124AD3ED112A6E
:1046700093ED137A26EE044AA5EE224AA3EE074AEA
:1046800023EE844AB4EEE64AF1EE10FAB4EEE74ABD
:104690008CBFB0EE667AB0EE447AF1EE10FA98BFB5
:1046A000F0EE476AA8BFF0EE447A052A8DED104A75
:1046B0006CD093ED164AD3ED152A93ED177A26EEBA
:1046C000044AA5EE224AA3EE074A23EE844AB4EE3A
:1046D000E64AF1EE10FAB4EEE74A8CBFB0EE667A25
:1046E000B0EE447AF1EE10FA98BFF0EE476AA8BF38
:1046F000F0EE447A062A8DED114A47D093ED1A4A1E
:10470000D3ED192A93ED1B7A26EE044AA5EE224A30
:10471000A3EE074A23EE844AB4EEE64AF1EE10FA1D
:10472000B4EEE74A8CBFB0EE667AB0EE447AF1EEB2
:1047300010FA98BFF0EE476AA8BFF0EE447A072A55
:104740008DED124A22D093ED1E7AD3ED1D2A93ED02
:104750001F4A26EE077AA5EE227AA4EE037A27EE08
:10476000237AB4EEE67AF1EE10FAB4EEE77A8CBF73
:10477000B0EE666AB0EE476AF1EE10FA8DED137A8C
:1047800098BFF0EE466AA8BFF0EE477A77EEE67A79
:10479000F7EE006AF4EEE67AF1EE10FAC4ED727A02
:1047A00043F3CC8586EEA77A022ADDED0D7A67EE1B
:1047B000244A67EE877ACDED0C4ACDED0D7A2DD0E7
:1047C000DDED0E7A67EE877A032ACDED0E7A25D0DD
:1047D000DDED0F7A67EE877A042ACDED0F7A1DD0D2
:1047E000DDED107A67EE877A052ACDED107A15D0C7
:1047F000DDED117A67EE877A062ACDED117A0DD0BC
:10480000DDED127A67EE877A072ACDED127A05D0B0
:10481000DDED137A27EE877A8DED137A344B1E681F
:1048200016F0805601F0AF80F6EE005AC4ED835AC0
:10483000002A02F076852F4BD4ED814A93F803804D
:1048400094F908320999D4ED806A91F800E0DFF814
:10485000B0C02949DFF8AC90B1F906109CED007AA0
:10486000049106EE103AFDEEE44A244B99F80090CC
:10487000B3F81AB094ED7D5AD4ED7E7A14EE903AE6
:10488000FDEEE64A00F0100C00F480000EF0010E80
:10489000B8EEC66A14EE901A0590B8F1000F41F018
:1048A0000D82DFF84480BCF1000F41F0B98098ED33
:1048B000007ADDED0C6ADFF850C025EE877AA6EEAF
:1048C000267AF0EE676AE5EE076ABDEEE67A17EE45
:1048D000106A17EE100A9E42A8BF184616E000BFE5
:1048E0001C520020F48A0020B04E0020000000007E
:1048F00044500020B88C0020088D00201C9000201F
:104900008C4E0020BC920020FC4F0020B142C8BF5A
:10491000084607EE100AB8EEC77A012A8CED007A35
:1049200000F0DC8098ED047ADDED0D6A25EE877AE3
:10493000A6EE267AF0EE676AE5EE076ABDEEE67A45
:1049400017EE106A17EE100A9E42A8BF1846B14231
:10495000C8BF084607EE100AB8EEC77A022A8CEDE7
:10496000017A00F0BB8098ED087ADDED0E6A25EE45
:10497000877AA6EE267AF0EE676AE5EE076ABDEE64
:10498000E67A17EE106A17EE100A9E42A8BF184684
:10499000B142C8BF084607EE100AB8EEC77A032A2C
:1049A0008CED027A00F09A8098ED0C7ADDED0F6ABA
:1049B00025EE877AA6EE867AF0EE676AE7EE056A5C
:1049C000BDEEE67A17EE106A17EE100A9E42A8BFF7
:1049D0001846B142C8BF084607EE100AB8EEC77ABB
:1049E000042A8CED037A79D098ED107ADDED106A07
:1049F00025EE877AA6EE867AF0EE676AE7EE056A1C
:104A0000BDEEE67A17EE106A17EE100A9E42A8BFB6
:104A10001846B142C8BF084607EE100AB8EEC77A7A
:104A2000052A8CED047A59D098ED147ADDED116ADF
:104A300025EE877AA6EE867AF0EE676AE7EE056ADB
:104A4000BDEEE67A17EE106A17EE100A9E42A8BF76
:104A50001846B142C8BF084607EE100AB8EEC77A3A
:104A6000062A8CED057A39D098ED187ADDED126AB8
:104A700025EE877AA6EE867AF0EE676AE7EE056A9B
:104A8000BDEEE67A17EE106A17EE100A9E42A8BF36
:104A90001846B142C8BF084607EE100AB8EEC77AFA
:104AA000072A8CED067A19D098ED1C7ADDED136A91
:104AB00065EE875AE6EE265AE5EE257AFDEEE77AB0
:104AC00017EE900A8342A8BF03468142C8BF0B4637
:104AD00007EE903AF8EEE77ACCED077ABEF1000FD8
:104AE00040F04982002A40F0418244E2AE4B1B78FC
:104AF000013BDBB2FFF72FBAAC4B06934FF47A764B
:104B00001B68B6FBF3F3C3EB4316A949DFF8CC826D
:104B100091F801A0A749B8F9060091F8009003EBBD
:104B20008603DE00B6B2B74202F06E81D5F8881077
:104B3000B5F93CE0EB6E4A1C07EE90EA7344012A9B
:104B4000C5F88820EB66F8EEE77A02F06881D5EDCB
:104B50001E5AD5ED206A07EE102A37EEE56AB8EE48
:104B6000C75A012F86EE057A37EE257A77EEC77A97
:104B700085ED1F7AE7EE866A85ED1E7AF0EE667A9D
:104B8000C5ED216AC5ED206A02F03A85D5F89C1082
:104B9000B5F93EE02B6F4A1C07EE90EA7344012AF8
:104BA000C5F89C202B67F8EEE77A02F05181D5ED2D
:104BB000235AD5ED256A07EE102A37EEE56AB8EEDE
:104BC000C75A012F86EE057A37EE257A77EEC77A37
:104BD00085ED247AE7EE866A85ED237AF0EE667A33
:104BE000C5ED266AC5ED256A02F03385D5F8B0100B
:104BF000B5F940E06B6F4A1C07EE90EA7344012A56
:104C0000C5F8B0206B67F8EEE77A02F03A81D5ED8F
:104C1000285AD5ED2A6A07EE102A37EEE56AB8EE73
:104C2000C75A012F86EE057A37EE257A77EEC77AD6
:104C300085ED297AE6EE276A85ED287AF0EE667A28
:104C4000C5ED2B6AC5ED2A6A02F02C85A8F806008E
:104C5000B5F8B430574A013B92F80090A5F8B4304B
:104C600006990023B9F1070F4B608B60CB607FF48E
:104C700067A9F7F7E5FADFF8648194F8C031A0EB93
:104C80000B00A8F80000002B3FF45FA9013B84F85B
:104C9000C03115B0BDEC0A8BBDE8F08F94ED5E7AA3
:104CA000B1F90000D4ED5F6AB1F902E0424AF4EED6
:104CB000C76A80EAE0738EEAEE71A3EBE073F1EE6F
:104CC00010FAA1EBEE71B4BFB0EE476AB0EE666ABF
:104CD0008B42B8BF0B4607EE103A1378B8EEC77A8E
:104CE00027EE287A002B40F02D82344BD3ED005A6A
:104CF000F4EECA5AF1EE10FA41F1FC80B7EE005A18
:104D000075EE654ADFED2E6A9FED2E5A2E4B36EE7C
:104D1000C77A24EE855AD3ED006AE7EE055A65EEB0
:104D2000A65AF5EEC05AF1EE10FA40F22886C9EE06
:104D3000A56AB7EE007AF0EE475AE6EE665AF0EE54
:104D4000656AF4EEC76AF1EE10FA88BFF0EE476AC2
:104D5000F5EEC06AF1EE10FAB8BFF0EE6A6A1B4BCE
:104D600093ED007A67EE877AA7EEA68AFFF7E0B99F
:104D7000174B184A2B4493ED007AD2ED007A164B6C
:104D800067EE277AF7EE006AF4EEE67AF1EE10FAB3
:104D900093ED007A88BFF0EE667A67EE877A27EEA9
:104DA000888AFFF776BA00BFE8510020988E00206D
:104DB000848E0020F8580020444E00204C4E0020E5
:104DC00000003443610BB63B404E00203C4E0020B7
:104DD0005C290020344E0020304E0020FC5800207A
:104DE000072B02F0C9824FF00009DFF84CA3B94D40
:104DF000DAF800305A0501F18280B74B19680B07C9
:104E000001F1E380B54B1B78002B40F0F581DFF812
:104E100010B394F8126126B1B14B1B889F0742F082
:104E20003F8294F81831002B41F073809BF81E608C
:104E3000002E00F0F783022E02F08B80032E01F08B
:104E40002D83A84A52889BF81F700237FFB2002BAF
:104E500002F07380002A02F07080A3490E68B2FB52
:104E6000F6F216B2A4F84861002F03F06F8207EE45
:104E7000906AF8EEE77AF7EE006A86EEA77A9B4A28
:104E8000012FD4ED576AD2ED007A77EEE67A67EE1D
:104E9000877AC4ED537A21D0D2ED017AD4ED586AE5
:104EA00077EEE67A022F67EE877AC4ED547A15D052
:104EB000D2ED027AD4ED596A77EEE67A032F67EEE7
:104EC000877AC4ED557A09D0D2ED037AD4ED5A6AC7
:104ED00077EEE67A67EE877AC4ED567A84490978E8
:104EE000092903F0E882002E40F3A28397B394EDE2
:104EF000577AD4ED537A77EE877A012FC4ED577A3B
:104F0000C2ED007A21D094ED587AD4ED547A77EE40
:104F1000877A022FC4ED587AC2ED017A15D094ED4C
:104F2000597AD4ED557A77EE877A032FC4ED597A02
:104F3000C2ED027A09D0D4ED5A7A94ED567A77EE22
:104F4000877AC4ED5A7AC2ED037A013F022FB8BFC7
:104F50000227FFB2002B18BF02276AE3099B654DA9
:104F60001B78DE0700F166812A7822B1920062493F
:104F7000624823F03BF9624B1B68002B40F0318301
:104F8000604B1B789BB1287870B1DFF87081DFF837
:104F9000AC910026F0B2D9F80030B8EC010A98477D
:104FA000287801368642F5DB574B1B689847504BF3
:104FB0001B78072B00F02D85012384F8003115B0F4
:104FC000BDEC0A8BBDE8F08F504BC7ED00AA1B6803
:104FD0009342BFF6EDA84E4B1A88002384F8D831CF
:104FE000002A41F0E9864B4A4B4B1178186881F052
:104FF0000101F7F7B3FFFFF7E3B8484FDFF840913F
:1050000007F24C7607F5F768F7EC017A95ED080A98
:10501000D5F87837F8EEE77A304627EE800A9847D9
:10502000A6F1E000D5F898369847A6F17000D5F8BB
:1050300008379847D7F85806D5F8B8309847243637
:10504000B045A9EC010ADFD1FEF773BF099A1278C7
:10505000D50703D4324A128BA4F8FC21314A2349E4
:10506000128891ED037A07EE902AF8EEE77AB4EE13
:10507000E77AF1EE10FA41F229812B49098807EE0F
:10508000901AF8EEE77AB4EEE77AF1EE10FAC1F290
:1050900055802649264AD1ED006A92ED006A2549DD
:1050A000C4ED806ABCEEC75A76EE665A15EE102A39
:1050B000C4ED7E6AC4ED7D5A84ED816AA4F8FC21BA
:1050C0000122D1ED006A84F8082277EE677AFFF7B3
:1050D00070B900BF04980020405500200423002030
:1050E000308D00202073002018520020D859002055
:1050F000F8580020F48A0020904E0020FC4F002039
:10510000C8460020C4950020B8920020604E0020C0
:10511000D4950020D6950020D89500203498002002
:105120001C900020444F0020464F0020304F0020AC
:10513000C45100204C4F0020A88E0020B0920020C7
:105140009C8E0020CD4B93ED005AB5EEC05AF1EE87
:1051500010FA40F31484CA4BD3ED006AF5EEC06A2E
:10516000F1EE10FA40F30B8436EEC77A66EE695A18
:1051700087EE266AC5EE856AB7EE007AB4EEC76A96
:10518000F1EE10FA88BFB0EE476AB5EEC06AF1EEF4
:1051900010FA76EE876AB8BFB0EE6A6A66EE266AE3
:1051A000CFE5B84A92ED007AF0EEE76AF4EEC76A0E
:1051B000F1EE10FA7FF78EA8B34A92ED007AF0EE86
:1051C000CC6AF4EEC76AF1EE10FA7FF783A8AF4A13
:1051D00098ED007AD2ED006AB0EEC77AB4EEE67AC6
:1051E000F1EE10FA7FF576A801220899C4F8DC11D7
:1051F00084F8D821FFF772B8A54BDFF8B8B2B3F93D
:105200000620BBF81A309A423FF703AEA14B1B7839
:10521000012B01F07D86192B01F07A860E2B3FF4CD
:10522000F8AD082B3FF4F5AD9B4A00239360C4F81A
:105230000C31EEE52B78002B3FF49DAED4ED5F3AB8
:1052400094ED5E6AD4ED7E7A944A94ED7D7AD2ED47
:10525000005A94ED5C4AD4ED5B4ADFF85C82DFF8DB
:105260005CC2F4EEC63AF3EE046AF1EE10FA37EEE1
:10527000A65A01F1648098ED026A26EE446AF0EEC7
:10528000674AE6EE074AF4EEC54A34EEE66AF1EE06
:1052900010FA48BFB0EE656A012B8CED006A3FF44E
:1052A0006AAE98ED066A26EE446AF0EE674AE6EECC
:1052B000074AB4EEE45A34EEE66AF1EE10FA88BF1B
:1052C000B0EE656A022B8CED016A3FF454AE98EDA6
:1052D0000A6A26EE446AF0EE674AE6EE074AF4EE02
:1052E000C54A34EEE66AF1EE10FA48BFB0EE656AE0
:1052F000032B8CED026A3FF43EAE98ED0E6A26EE6B
:10530000446AF0EE674AE6EE074AB4EEE45A34EE39
:10531000E66AF1EE10FAC8BFB0EE656A042B8CEDB8
:10532000036A3FF428AE98ED126A26EE446AF0EE66
:10533000674AE6EE074AB4EEE45A34EEE66AF1EE66
:1053400010FAC8BFB0EE656A052B8CED046A3FF415
:1053500012AE98ED166A26EE446AF0EE674AE6EE63
:10536000074AF4EEC54A74EEE66AF1EE10FAB8BFE9
:10537000F0EE656A062BCCED056A3FF4FCADD8ED86
:105380001A6A66EEC46AF0EE674AE6EE874AB3EE42
:10539000046AB4EEE45A74EEC66AF1EE10FAC8BFBD
:1053A000F0EE656A072BCCED066A3FF4E4ADD8ED6C
:1053B0001E6A26EEC44AE4EE077AF4EEC57A77EE6A
:1053C000C67AF1EE10FA48BFF0EE657ACCED077AB6
:1053D000D1E50699324BD1ED017A93ED007AF0EEEA
:1053E000E77AF4EEC77AF1EE10FA7EF5E9AED1ED88
:1053F000027AF0EEE77AB4EEE77AF1EE10FA7EF791
:10540000DFAED1ED037AF0EEE77AB4EEE77AF1EEB3
:1054100010FA7EF7D5AE234B1B689A077FF5DBADFC
:105420002149224BB3F90C20B1F900E02048AEEB42
:10543000020E00688EEAEE72A2EBEE728242BEF6B7
:10544000BFAEB3F90E30B1F90220D21A82EAE2738C
:10545000A3EBE27398427EF7B3AEBCE50B4B98ED3D
:10546000007AD3ED006AB0EEC77AB4EEE67AF1EED8
:1054700010FA7EF745AFFEF740BF00BF404E002058
:10548000484E0020744E0020704E0020784E0020C0
:10549000088D00201C520020D85900208C4E00207E
:1054A0006C4E00204055002024550020F45100206F
:1054B000684E00201C900020B04E0020FC4F0020C1
:1054C00007EE103A534BDFF858811B78C4F8A871E7
:1054D000B8EEC77AF7EE006A132B86EE879AB8F912
:1054E0000400B4F8AC6195ED080A01F0F0834A4B72
:1054F0004A4A93ED001AD3ED053A93ED122A93ED43
:10550000173AD3ED091AD3ED0E4A93ED016A93EDE4
:10551000064A93ED0A7AD3ED0F5AD3ED132AD3ED51
:10552000186A93ED045AD3ED030A67EE897A69EE9F
:10553000288A29EE088AE1EE273A02EB8607002145
:10554000A2EE283AC4F89C11C4F8A011E1EE884AF2
:10555000A6EE274AE7EE085A93ED167A93ED0D6A08
:1055600093ED021AD3ED0C1AC7ED003AE2EEA86AE9
:1055700025EE635A27EE437A93ED0B2AD3ED152AD5
:10558000C7ED204AA0EEE34A26EE646AD3ED143A52
:1055900083ED054AA1EE275AF0EE477AE1EEE45A90
:1055A000A2EE086AE2EEC36AE3EEA87A83ED065A39
:1055B000C3ED0E5A83ED0F6A87ED403AC3ED176ACB
:1055C000C3ED187AC4F8A411731C03F01F03A4F8E8
:1055D000AC31A8F80400FEF78FBBB0EE465AFEF7D8
:1055E00021BF0AF021FCCBE496ED007A0C4905EBD3
:1055F0004702B8EEC78A928F21F8172028EE278A33
:10560000FEF765BC22F0FCFF054B23F81700FEF700
:1056100080BC00BFF858002078760020F47300208A
:10562000FC580020A4F84861002B00F06F81D84A94
:105630000227D84BDFEDD86A1968D84B887893F8E1
:1056400000E00B7807EE903AF8EEE77AB0EE007AD9
:1056500067EEA67AF4EEC77AF1EE10FA40F31D83F6
:1056600037EEC77ADFEDCE6AB0EE676AA7EE266A3C
:10567000B0EE467A9FEDCB6AD2ED006A66EE866A9E
:10568000B0EEE66AC4ED5B6A84ED5E6A98B105EE41
:10569000900AB8EEE55ADFEDC05A66EEA64A25EE4E
:1056A000255AF7EE005A75EEC55A64EE864AE4EEC6
:1056B000855A66EEA56ADFEDBC5A4B7927EE257A4E
:1056C00027EE267ACBB1DFEDB46ADFEDB85A26EECD
:1056D000266A06EE903AF8EEE66A26EE266AB4EE00
:1056E000E56AF1EE10FA00F31886F7EE005A35EE8F
:1056F000C66AC5EE866A27EE267ABEF10C0F9FEDCC
:10570000AC8ADFEDAC6A00F08085B4EEC87AF1EEC9
:1057100010FA98BFB0EE478AB4EEE68AF1EE10FABE
:10572000B8BFB0EE668A84ED418A002F00F0E080B9
:10573000B0EE007AF4EEC77AF1EE10FA05DD37EE3E
:10574000C77ADFED976AE7EE267A92ED017ADFED10
:10575000956A27EE267AB0EEC76A84ED5C7A84ED0E
:105760005F6A98B106EE900ADFED8B5AF8EEE66AB2
:1057700027EE075A66EEA56AF7EE005A75EEE65A6E
:1057800025EE065AE5EE265A27EE257ADFED866AE3
:105790008B7967EEA67A67EE877AABB107EE103A9F
:1057A000B8EEC77ADFED7C5ADFED806A27EE067A25
:1057B00027EE257AB4EEE67AF1EE10FA40F3B185E1
:1057C000DFED7D6A67EEA67ABEF10C0F00F0FC8477
:1057D000DFED776A9FED777AF4EEE67AF1EE10FA74
:1057E00088BFF0EE667AF4EEC77AF1EE10FAB8BF31
:1057F000F0EE477A012FC4ED427A79DD4B78DFED88
:10580000666A07EE903AF8EEE77AB0EE007A67EE55
:10581000A67A4B7AF4EEC77AF1EE10FA05DD37EE90
:10582000C77ADFED5F6AE7EE267A92ED027ADFED66
:105830005D6A27EE267AB0EEC76A84ED5D7A84ED64
:10584000606A9BB106EE903ADFED535AF8EEE66AD5
:1058500027EE075A66EEA56AF7EE005A75EEE65A8D
:1058600025EE065AE6EE855A27EE257ADFED4E6ADA
:10587000CB7967EEA67A67EE877A0BB307EE103A1C
:10588000B8EEC77ADFED445ADFED486A27EE067AB4
:1058900027EE257AB4EEE67AF1EE10FA0CDCB5EEDE
:1058A000C07AF1EE10FA01F13E83B7EE006A36EEEF
:1058B000477AC6EE076A01E0DFED3F6A67EEA67A37
:1058C000BEF10C0F00F07684DFED396A9FED397A76
:1058D000F4EEE67AF1EE10FA88BFF0EE667AF4EEB6
:1058E000C77AF1EE10FAB8BFF0EE477AC4ED437A0A
:1058F000BEF1090F00F041849BF82160002E40F0BA
:10590000D7832E4B1968002384F81831890609D5EE
:105910002B4B1B8803F0300323B12A4B1B78DA078B
:1059200002F11680284B1B7823B9284EB378002B40
:1059300041F01683194B1B78072B00F0838400225B
:10594000072B84F800217EF484A9F6F779FC8346BE
:10595000FEF781B91E4B1F4C1A681F4BDFF884807D
:1059600094F80001D2691B88A8F80020A8F802303A
:1059700000287FF438AA8346184DFEF76CB9DFED96
:10598000186AFFF7ECB941023EF54EAFFEF750BF83
:10599000D8590020C0AB00200AD7233CF85800207B
:1059A000D7A368416F12033B00004843A4707D3FBA
:1059B00000C0F94400C0F9C40000C84240550020AE
:1059C000308D0020445500202C5E0020F2A90020DC
:1059D000B0580020E4270020A253002004980020A3
:1059E00000000000FC580020F6F72AFCAC4B0B9A94
:1059F0001B78DFF8B082801A012BA8F8020000F0B3
:105A00004183072B7EF4A4ACF6F71AFC0746FEF799
:105A1000A0BCF6F715FCA34BC01BD880FFF7CCBA8F
:105A2000BEF1000F41F0DE8498ED007ADDED0C6AE6
:105A3000DFF884C225EE877AA6EE867AF0EE676AF2
:105A4000E7EE056ABDEEE67A17EE106A17EE100A69
:105A50009E42A8BF1846B142C8BF084607EE100ACA
:105A6000B8EEC77A012A8CED007A3FF47FAA98ED50
:105A7000047ADDED0D6A25EE877AA6EE867AF0EEE1
:105A8000676AE7EE056ABDEEE67A17EE106A17EE72
:105A9000100A9E42A8BF1846B142C8BF084607EE8A
:105AA000100AB8EEC77A022A8CED017A3FF45EAA9A
:105AB00098ED087ADDED0E6A25EE877AA6EE867AF5
:105AC000F0EE676AE7EE056ABDEEE67A17EE106A59
:105AD00017EE100A9E42A8BF1846B142C8BF08463A
:105AE00007EE100AB8EEC77A032A8CED027A3FF46B
:105AF0003DAA98ED0C7ADDED0F6A25EE877AA6EEC9
:105B0000867AF0EE676AE7EE056ABDEEE67A17EE92
:105B1000106A17EE100A9E42A8BF1846B142C8BFCD
:105B2000084607EE100AB8EEC77A042A8CED037A0D
:105B30003FF41CAA98ED107ADDED106A25EE877A05
:105B4000A6EE867AF0EE676AE7EE056ABDEEE67AC3
:105B500017EE106A17EE100A9E42A8BF1846B1420F
:105B6000C8BF084607EE100AB8EEC77A052A8CEDC2
:105B7000047A3FF4FBA998ED147ADDED116A25EE65
:105B8000877AA6EE867AF0EE676AE7EE056ABDEEE2
:105B9000E67A17EE106A17EE100A9E42A8BF184662
:105BA000B142C8BF084607EE100AB8EEC77A062A07
:105BB0008CED057A3FF4DAA998ED187ADDED126ADA
:105BC00025EE877AA6EE867AF0EE676AE7EE056A3A
:105BD000BDEEE67A17EE106A17EE100A9E42A8BFD5
:105BE0001846B142C8BF084607EE100AB8EEC77A99
:105BF000072A8CED067A3FF4B9A998ED1C7ADDED01
:105C0000136A65EE875AE6EE265AE5EE257AFDEE32
:105C1000E77A17EE900A8342A8BF03468142C8BFC5
:105C20000B4607EE903AF8EEE77ACCED077A002AB9
:105C30007FF49CA9FFF79FB91B4B5A79002A3EF4C9
:105C400076AC1A4A1278002A3EF471AC1B78DFED6C
:105C5000184A07EE903A174BB8EE677A1B8807EEA2
:105C6000902A06EE903AF8EEE77AF8EE666A67EE6A
:105C7000277AB7EE007AC7EEA63AF4EEE43AF1EEF0
:105C800010FA88BFF0EE643AF4EEC73AF1EE10FA7B
:105C9000B8BFF0EE473AFEF74CBCB0EE677AE9E4E5
:105CA000F8580020FC5800202C550020D659002020
:105CB000713DAA3FC0590020FC4F0020BCF1000FED
:105CC00000F00084BEF1000F42F08C80DFF8F08518
:105CD000B9F1000F41F0EC86D8ED006ADDED0C4A19
:105CE000DFF8E0C565EEA66ABDEEC77A17EE101ABA
:105CF000B0EE667AA4EE867AF0EE676AE7EE056AA1
:105D0000BDEEE67A17EE106A17EE100A9E42A8BFA3
:105D10001846B142C8BF084607EE100AB8EEC77A67
:105D2000012A8CED007A3FF421A998ED047ADDED8B
:105D30000D6A25EE877AA6EE867AF0EE676AE7EEC0
:105D4000056ABDEEE67A17EE106A17EE100A9E425B
:105D5000A8BF18468E42B8BF084607EE100AB8EE34
:105D6000C77A022A8CED017A3FF400A998ED087AEF
:105D7000DDED0E6A25EE877AA6EE867AF0EE676A8A
:105D8000E7EE056ABDEEE67A17EE106A17EE100A26
:105D90009E42A8BF18468E42B8BF084607EE100ABA
:105DA000B8EEC77A032A8CED027A3FF4DFA898EDAB
:105DB0000C7ADDED0F6A25EE877AA6EE867AF0EE94
:105DC000676AE7EE056ABDEEE67A17EE106A17EE2F
:105DD000100A9E42A8BF18468E42B8BF084607EE7A
:105DE000100AB8EEC77A042A8CED037A3FF4BEA8F5
:105DF00098ED107ADDED106A25EE877AA6EE867AA8
:105E0000F0EE676AE7EE056ABDEEE67A17EE106A15
:105E100017EE100A9E42A8BF18468E42B8BF084629
:105E200007EE100AB8EEC77A052A8CED047A3FF423
:105E30009DA898ED147ADDED116A25EE877AA6EE1D
:105E4000867AF0EE676AE7EE056ABDEEE67A17EE4F
:105E5000106A17EE100A9E42A8BF18468E42B8BFBD
:105E6000084607EE100AB8EEC77A062A8CED057AC6
:105E70003FF47CA898ED187ADDED126A25EE877A5A
:105E8000A6EE867AF0EE676AE7EE056ABDEEE67A80
:105E900017EE106A17EE100A9E42A8BF18468E42EF
:105EA000B8BF084607EE100AB8EEC77A072A8CED8D
:105EB000067A3FF45BA898ED1C7ADDED136A65EE77
:105EC000875AE6EE265AE5EE257AFDEEE77A17EEDA
:105ED000900A8342A8BF03468142D8BF194607EE05
:105EE000901AF8EEE77ACCED077A002A7FF43EA804
:105EF000FFF741B8D94BD3ED005AFEF712BFAB689C
:105F0000002B3EF47AAF05F1500128469847FEF782
:105F100074BFD348D34AD0F8EC00126844F6206628
:105F2000B042A8BF3046B0F57A7FB8BF4FF47A7060
:105F300080B212F0100FA4F81A01DAF8002001F074
:105F40005A83D20400F1D383C74A1768B7F932C025
:105F5000C64AC74ED2ED037AD4F81C21A6FB000630
:105F6000B609642090FBF6F01428BDEEE77A04EB46
:105F7000420EA8BF142001328242C4F81C2117EE41
:105F8000108AA4BF0022C4F81C2104EB4202AEF820
:105F90002081B2F9202107EE102AB8EEC77A77EEF9
:105FA000C77AFDEEE77ACDED047ABDF9100080EAFC
:105FB000E072A2EBE072624502F3B281AD4A104694
:105FC0004FF07E520260FEF731BFA84AD2ED027A4E
:105FD000B2EE0E7AF0EEE76AF4EEC76AF1EE10FA6E
:105FE00041D5A54B1B885F073DD5A44BA448B3F909
:105FF0000430A44E80FB03703688DB17C3EBA0038C
:106000009B1B9BB218B210F1B30FBCBF03F5B47366
:1060100018B2B328C4BFA0F5B47318B29A4B9B4E04
:106020001B793678002B4FF6FF7318BF0123360714
:106030007EF5E8AE8C4E366810FB03F3307E944E4E
:106040009BB210FB03F386FB03601844DB17C3EB22
:10605000201307EE103AB8EEC77A77EEC77AC2ED92
:10606000027AFEF7CFBE854B854AB3F904308548E6
:1060700082FB0362DB17C3EBA2030380FEF7C2BE01
:10608000DFF84482F6F7DCF8824AD4F8EC31126883
:10609000C4F8EC01C31A9A1A0746A8F80430A8F805
:1060A0000620FEF756B9F6F7CBF80B90FDF75CBF6C
:1060B0001E216C48F3F720FA00283FF422AC6E4B07
:1060C0001B8858063FF51DAC94F88431B34242F06A
:1060D0006E81684BD4ED627AD3ED016A94ED435A38
:1060E000DFED6D5A9FED6D6A27EEC57A68EE277A6F
:1060F000A8EE267AE5EE267AB4EEE57AF1EE10FA0D
:1061000088BFB0EE657AB4EEC67AF1EE10FAF4EE1E
:10611000E57AB8BFB0EE467AF1EE10FA88BFF0EE3D
:10612000657AF4EEC67AF1EE10FAB8BFF0EE467A70
:1061300084ED417AC4ED437AFFF7E3BBB4F8FC1178
:10614000914240F293855649564AD1ED007A92ED3C
:10615000007A5549C4ED807A77EE676AC4ED7E7A9D
:106160000122C4ED7D6A84ED817AD1ED006ADFED14
:106170004F7A84F80822FEF71CB9FDEEC87ADFF8E2
:10618000488117EE903AA8F80460A8F80630FFF7A7
:10619000B3BB474B1B88002B40F08785454A464BD5
:1061A00011781868F6F7DAFED4F8DC21089B9A1A01
:1061B000FDF7D5BFBDEEE77ADFF80C8117EE103A98
:1061C000A8F80430FFF780BB9FED337ADFED336A28
:1061D000DFF8F480F4EEC77AF1EE10FA98BFB0EE73
:1061E000677AFDEEE77AB4EEE67AF1EE10FA17EE92
:1061F000903AB8BFB0EE667A012F84ED427AA8F8E3
:1062000002303FF7FBAAFFF777BBB4EEC87AF1EE96
:1062100010FA98BFB0EE478ABDEEC77AB4EEE68AB0
:10622000DFF8A480F1EE10FA17EE103AB8BFB0EE26
:10623000668A84ED418AA8F80030002F7FF478AA9E
:10624000FFF75ABBF5F7FCFFDFF87C801B4BA0EB98
:1062500009001B78A8F80400FFF771BB404E00202E
:106260006801002044500020A4A80020D859002034
:10627000D34D6210A4000020308D00202455002052
:1062800067666666708E0020EC5100204455002041
:10629000898888881852002000C0F94400C0F9C4D9
:1062A000304F0020C45100204C4F0020000000005F
:1062B000D4950020D6950020D8950020F8580020CD
:1062C000B04E0020FC4F0020FC580020784A79494D
:1062D000D2ED006A784A91ED006A1278C4ED806AC6
:1062E00084ED816A002A40F0BD8476EEC65AF0EE55
:1062F000466ABCEEC76A7149C4ED7D5A16EE102A93
:10630000C4ED7E6AA4F8FC21FF22D1ED006A84F876
:10631000082277EEC77AFEF74CB8DFED696AFFF71F
:10632000EAB9B5EEC07AF1EE10FA00F1F885B7EEF1
:10633000006A36EE477AC6EE076AFFF743BA98ED71
:10634000016A26EE646AB0EE674AA6EE074AB4EE2A
:10635000C45A34EE666AF1EE10FAC8BFB0EE656A50
:10636000012B8CED006A3EF406AE98ED056A26EE30
:10637000646AB0EE674AA6EE074AB4EEC45A34EE39
:10638000666AF1EE10FAC8BFB0EE656A022B8CEDBA
:10639000016A3EF4F0AD98ED096A26EE646AB0EE4B
:1063A000674AA6EE074AB4EEC45A34EE666AF1EEC6
:1063B00010FAC8BFB0EE656A032B8CED026A3EF49A
:1063C000DAAD98ED0D6A26EE646AB0EE674AA6EE85
:1063D000074AB4EEC45A34EE666AF1EE10FAC8BF4A
:1063E000B0EE656A042B8CED036A3EF4C4AD98ED03
:1063F000116A26EE646AB0EE674AA6EE074AB4EE6A
:10640000C45A34EE666AF1EE10FAC8BFB0EE656A9F
:10641000052B8CED046A3EF4AEAD98ED156A26EEC0
:10642000646AB0EE674AA6EE074AB4EEC45A74EE48
:10643000666AF1EE10FAC8BFF0EE656A062BCCED85
:10644000056A3EF498ADD8ED196A66EEE46AB0EEDE
:10645000674AA6EE874AB3EE046AB4EEC45A74EEF5
:10646000466AF1EE10FAC8BFF0EE656A072BCCED74
:10647000066A3EF480ADD8ED1D6A66EEE44AE4EEAD
:10648000877AF4EEC57A77EEC67AF1EE10FAB8BFE5
:10649000F0EE657ACCED077AFEF76DBD9BF8202013
:1064A000C2EB421002EB8002D20092B2FEF7CBBCEC
:1064B00060500020344F0020BC920020484F002044
:1064C0000000C842DFF8D885B9F1000F41F0018122
:1064D000D8ED006ADDED0C4ADFF8C8C565EEA66AA6
:1064E000BDEEC77A17EE101AB0EE667AA4EE867A81
:1064F000F0EE676AE7EE056ABDEEE67A17EE106A1F
:1065000017EE100A9E42A8BF1846B142C8BF0846FF
:1065100007EE100AB8EEC77A012A8CED007A3EF435
:10652000DDAA98ED047ADDED0D6A25EE877AA6EEF8
:10653000867AF0EE676AE7EE056ABDEEE67A17EE58
:10654000106A17EE100A9E42A8BF18468E42B8BFC6
:10655000084607EE100AB8EEC77A022A8CED017AD7
:106560003EF4BCAA98ED087ADDED0E6A25EE877A36
:10657000A6EE867AF0EE676AE7EE056ABDEEE67A89
:1065800017EE106A17EE100A9E42A8BF18468E42F8
:10659000B8BF084607EE100AB8EEC77A032A8CED9A
:1065A000027A3EF49BAA98ED0C7ADDED0F6A25EE97
:1065B000877AA6EE867AF0EE676AE7EE056ABDEEA8
:1065C000E67A17EE106A17EE100A9E42A8BF184628
:1065D0008E42B8BF084607EE100AB8EEC77A042A02
:1065E0008CED037A3EF47AAA98ED107ADDED106A0C
:1065F00025EE877AA6EE867AF0EE676AE7EE056A00
:10660000BDEEE67A17EE106A17EE100A9E42A8BF9A
:1066100018468E42B8BF084607EE100AB8EEC77A91
:10662000052A8CED047A3EF459AA98ED147ADDED32
:10663000116A25EE877AA6EE867AF0EE676AE7EEB3
:10664000056ABDEEE67A17EE106A17EE100A9E4252
:10665000A8BF18468E42B8BF084607EE100AB8EE2B
:10666000C77A062A8CED057A3EF438AA98ED187A96
:10667000DDED126A25EE877AA6EE867AF0EE676A7D
:10668000E7EE056ABDEEE67A17EE106A17EE100A1D
:106690009E42A8BF18468E42B8BF084607EE100AB1
:1066A000B8EEC77A072A8CED067A3EF417AA98ED61
:1066B0001C7ADDED136A65EE875AE6EE265AE5EEA2
:1066C000257AFDEEE77A17EE900A8342A8BF0346CB
:1066D0008142D8BF194607EE901AF8EEE77ACCED62
:1066E000077ABEF1000F7EF446ACFEF7FBB9E04A34
:1066F0001768B7F832C04FEA5C0C29E4DFF8A893BA
:10670000D4ED017A94ED006AB9F80000D9F814309C
:1067100077EEA77AF0EE006AB0EE677AA6EE267AF8
:10672000013804EBC002D6EE267A083A1033F6EEB2
:10673000003A27EE237A67EEA37A84ED207AC4ED3F
:10674000217ACC4CA64604F1800192ED027A92EDBA
:10675000036ADEED036ADEED027A53ED014A13EDC2
:10676000025A37EE674A76EEC65A77EE277AE4EE9B
:10677000845A0138A2F10802E5EE047A0EF1080EFF
:1067800003F1080336EE267A01F10801E4EE877A78
:10679000E5EE475A67EEA37A25EEA37AC1ED007ABB
:1067A00081ED017AD1D1142F7DF461ABF5F748FD6D
:1067B000049BDFF8F882C01AA8F80200D4F8B06190
:1067C000FDF755BBD4F8B481B4F8AC310593C3F1EF
:1067D000200903EB481EA84B5FFA89F903EB8E0EE4
:1067E0005FEA990301F0DE8501331801A349A44A49
:1067F0000EEB000C0EF1100313ED024A13ED035AD9
:1068000013ED016A13ED047A51ED024A51ED035A7A
:1068100051ED016A51ED047A64EE244A65EE255A81
:1068200066EE266A67EE277A10339C4542ED024AEF
:1068300042ED035A42ED016A42ED047A01F1100182
:1068400002F11002D8D18F49A0F11002964401EB59
:10685000020C224419F0030309D0BEEC017AFCECCF
:10686000017A67EE277A013BE2EC017AF5D1059BCC
:10687000002B41F06082142F7DF4F9AAF5F7E0FCBB
:10688000049BDFF82882D4F8B061C01AA8F802008F
:10689000FDF7EDBAD4F8B4917B4A7C4BDFED7C7AFE
:1068A000D3ED008A7B4B4FEAC9010A44F8EE688AAF
:1068B000928809EE102A643AC82AA8BFC82268EE56
:1068C000A78AF8EE497A782AB8BF782268EEA78AB4
:1068D00007EE902A4944B0EE680A03EB8108B8EE4F
:1068E000E78A21F0D9FEB8EEC99AF0EE409AB0EEF0
:1068F000680A21F033FE38EE097A79EE487A28EEFC
:10690000098A67EE877AB7EE006A88EE277A142F35
:10691000F8EE007A77EE076A60EE277A89EEA67ABB
:1069200077EE065A36EE477AC6EE256A67EEA67A05
:1069300027EE267AC8ED006A88ED047AC8ED026A6F
:10694000C8ED017AC8ED037A01F0DF85524B534A56
:1069500009F1010983FB0938A8EBE97808EB48083D
:106960000136A9EB08081778C4F8B061C4F8B481FF
:106970002AE7DFF834913F48D9F80820B9F80C101D
:1069800020F000FD454B1F78142F01F02286D4F82B
:10699000B0610136C4F8B061B2E6DFF8149199F83D
:1069A0000020900801F06A86DFF808C100F10108B4
:1069B0004FEA48180CEB080E0CF12003ACF1700103
:1069C00013ED076A53ED056A13ED037A53ED017A6F
:1069D00053ED025A13ED084A53ED064A13ED045ADB
:1069E00026EE066A66EEA66A27EE077A67EEA77AB3
:1069F000A4EE046A20339E45E4EEA46A01F110017E
:106A0000A5EE057AE5EEA57AF1EEC65AB1EEE66A94
:106A1000F1EEC76AB1EEE77A41ED085A01ED076A77
:106A200041ED066A01ED057ACAD1A8F12008C444F7
:106A300004EB001012F0030318BF0CF1080C0FD088
:106A40005CED017A1CED027A67EEA77A013BE7EE76
:106A5000077A0CF1080CB1EEE77AA0EC017AEFD1DD
:106A6000142F01F0A6850136C4F8B061FDF768B9AE
:106A7000A4A80020E4270020F473002084750020DF
:106A8000F427002074750020F4750020988E0020F3
:106A900027D4D236809F002056555555F8580020EF
:106AA000B04E0020FC4F0020DC730020FC5800207A
:106AB000D673002064280020DFF83C93B9F800E08A
:106AC000D9F804C04FEA5E084FEA880204EB8E064C
:106AD0005FEADE0E04EB020300F0A08010320EF13C
:106AE000010EBA4803EB0E1E324410330CF11007AE
:106AF00006F1100151ED032A51ED043A10ED043A6C
:106B000010ED032A51ED026A11ED016A10ED020A3F
:106B100010ED018A12ED044A12ED035A53ED044AB6
:106B200053ED035A13ED027A53ED017A52ED020A46
:106B300012ED011A73EE238A72EE221A40ED048AD6
:106B400040ED031A70EE268A78EE061A40ED028AAE
:106B500040ED011A74EE848A75EE851A43ED048ABD
:106B600043ED031A77EE208A77EE811A43ED028A0D
:106B700043ED011A73EE633A75EE655A17ED035A49
:106B800032EE623A74EE644A65EE631A17ED044A17
:106B900023EE052A64EE652AE3EE041A10339E45BF
:106BA00024EE843AA3EE842A00F1100007F11007C6
:106BB000A5EE853A01F1100102F11002E4EE852AFA
:106BC00041ED071A01ED082A02ED073A42ED082AC5
:106BD00057ED055A17ED065A70EE666A38EE466AAA
:106BE00030EEC77A71EE677A26EE253A65EEE63A20
:106BF00025EE674A67EE054AE6EE053AA6EE853AC7
:106C0000A7EE254AE7EEA54A01ED063A41ED053A21
:106C100002ED064A42ED054A7FF46CAF1FFA88F890
:106C2000624641466A481EF063F94146D9F804209D
:106C300030461EF05DF9674B1B78142B7FF4BEAD18
:106C4000B4E5F5F7FDFA634B04901F78142F05BFE8
:106C5000DFF8A881D4F8B061D4F8B061A8F800607A
:106C6000FDF753B876EE665AFFF743BB5A4A5B49C5
:106C7000D2ED007A5A4A91ED007A1278C4ED807A0A
:106C800084ED817A002A01F0458377EE676A5549E1
:106C9000C4ED7E7AC4ED7D6AFF22D1ED006ADFED9E
:106CA000597A84F80822FDF784BB4F494B69002BC1
:106CB0003DF455AA4D484E4B008893FBF0F00B680D
:106CC0004FF0010E186081F811E0FDF748BA494F06
:106CD000DFF82C9197ED004A97ED057AD7ED014A40
:106CE00097ED066AD7ED046A97ED035AD7ED025A7D
:106CF00067EE897A09EB8603A4EE277AA4EEA76AE9
:106D000066EEC76AA5EE476AE5EEA76A20EE070AB7
:106D100087ED056AC7ED066A83ED007A29EE088AD9
:106D200021F06EFC69EE288AD7ED0E5AD7ED176A6E
:106D300097ED091AD7ED121A97ED0F5A97ED187AB9
:106D400097ED0A2AD7ED132A97ED0D6AD7ED167A3B
:106D500097ED0C3AD7ED0B3A97ED154AD7ED144A5B
:106D6000E1EE085A002209EB8603E8EEA16A00B2C0
:106D7000C4F89C21A2EE085AC4F8A021C4F8A421AA
:106D8000A8EEA27A26EE656A67EEE67AA3EE655A69
:106D9000A3EE886AA6EEC47AE8EEA47A87ED0E5ACE
:106DA000C3ED205A87ED0F6AC3ED406A87ED177A6D
:106DB000C7ED187AFEF708BC0B494A69002A3DF472
:106DC000FFA90A6813604B74FDF7FAB9F427002095
:106DD000E4270020F858002060500020344F0020A5
:106DE000BC920020484F0020DC950020F495002044
:106DF00020A1070078760020DC730020FC580020DA
:106E0000F473002000000000B5F93C306A6207EE20
:106E1000903A0122F8EEE77AEB66C5F88820002365
:106E2000012FC5ED1F7AC5ED1E7AC5F8803001F03F
:106E30009C82B7427DF4AAAEB5F93E302B6707EECF
:106E4000903A00220123F8EEE77AAA62C5F89C3056
:106E50000023012FC5ED247AC5ED237AC5F89430BF
:106E600001F07F82B7427DF4C1AEB5F940306B6767
:106E700007EE903A00220123F8EEE77AEA62C5F8BD
:106E8000B0300023012FC5ED297AC5ED287AC5F869
:106E9000A8307DF4DBAE1FED258AB9F1030F46D093
:106EA000BAF1000F09D007EE90AAF8EEE77AF4EEF7
:106EB000C87AF1EE10FA01F1E683BA4A6B6F1268F4
:106EC00094F8B811A8F8060003EB560393FBF6F606
:106ED0000023EE6293621363D36231B1B24B1B881D
:106EE00023F40063002B7DF4B3AEB04B1B6813F4A6
:106EF000003341F02E82AE491A46C85C012803F1E6
:106F00000C0300F0A1850132152AF6D1FDF7A0BED1
:106F1000A84B9B7B002B3EF487A9FDF77ABFF7EEC9
:106F2000006AFEF74FBCF7EE006AFEF7C7BCB0EE92
:106F3000480A21F065FB00B2B2E7B4F84861013EAF
:106F400036B2002EA4F848617EF76EAB9A4AFDF780
:106F5000CDBFB4F81A2102F57A7292B2FDF773BF71
:106F6000964F3A78013A0A2A1CD8DFE812F06501F8
:106F70008E01CB00AA009200760062005100410110
:106F800005010B008E4A8F4952680968C8328A424F
:106F900003D31DF079FA28B1B378032B01F0818473
:106FA00001233B70F378002B3EF4C4AC864B1B7876
:106FB000D80740F14A81DFF80C82D4F89821D8F83C
:106FC00000309A4200F24D813B78012B3EF4B2AC86
:106FD00094F89421002A3EF4ADAC0B2B0DD801227D
:106FE0009A4040F6030112EA01060CD112F4C06F78
:106FF00003D0093B012B41F22E85714BD8F80020BC
:107000005A600B233B70002384F89431FEF792BC46
:107010001DF018FA0CF078FA0028C3D01DF034FAED
:107020000028BFD0694A6A4B12681A600A233B7075
:10703000B8E71DF007FA674B002105208DE8030033
:10704000A3F10802029153200CF052FF0028A9D1AD
